:020000040000FA
:10000000884600201104000019040000310200009D
:100010001D0400001F040000210400000000000077
:1000200000000000000000000000000023040000A9
:10003000250400000000000027040000290400003F
:10004000190B00002B0400005D0E00002B040000C3
:100050002B0400002B040000810700002B0400008B
:100060002B0400002B0400002B0400002B040000D4
:100070002B0400002B0400002B0400002B040000C4
:100080002B040000290B00002B0400002B040000AF
:100090002B0400002B0400002B0400002B040000A4
:1000A0002B0400002B0400002B0400002B04000094
:1000B0002B0400002B0400000000000000000000E2
:1000C0002B0400002B0400002B0400002B04000074
:1000D0002B0400002B0400002B040000B50E0000D0
:1000E0002B0400002B0400002B0400000000000083
:1000F000000000002B040000000000002B040000A2
:1001000000000000000000000000000000000000EF
:1001100000000000000000000000000000000000DF
:1001200000000000000000000000000000000000CF
:1001300000000000000000000000000000000000BF
:1001400000000000000000000000000000000000AF
:10015000000000000000000000000000000000009F
:10016000000000000000000000000000000000008F
:10017000000000000000000000000000000000007F
:10018000000000000000000000000000000000006F
:10019000000000000000000000000000000000005F
:1001A000000000000000000000000000000000004F
:1001B000000000000000000000000000000000003F
:1001C000000000000000000000000000000000002F
:1001D000000000000000000000000000000000001F
:1001E000000000000000000000000000000000000F
:1001F00000000000000000000000000000000000FF
:10020000DFF80CD000F070FA00480047917200004F
:100210008846002000B583B002900091019244F21C
:10022000010071466A4601F045F803B000BD0000C8
:10023000094B1EF0040F1CBFEFF309801847EFF3C2
:1002400008800649064A884201D8904202D88D4665
:100250004FF00000184700003509000088460020D4
:100260008826002030B450E8012F93B2C48923447B
:100270008489A34228BF1B1B0489A34202BFBFF38A
:100280002F8F002007E0C3EA020340E80134002C6E
:10029000E9D14FF001000A6030BC704750E8012FEF
:1002A000C2EA024240E801210029F7D1704730B488
:1002B00050E8022F1FFAA2F3C488A34202BFBFF383
:1002C0002F8F00200DE0C48923448489A34228BFD6
:1002D0001B1BC2EA034340E80234002CE8D14FF074
:1002E00001000A6030BC704750E8022FC2EA224287
:1002F00040E802210029F7D17047034653E8022F56
:10030000D988B2EB324F4FF0000017BF92B241EAEA
:10031000014142EA014104E05A68B2EB324F08BFA2
:10032000012043E80212002AE8D1704730B40446A5
:1003300054E8000F0D4644E80053002BF8D1156037
:1003400030BC704730B4044654E8000F40EA010561
:1003500044E80053002BF7D1156030BC704730B42F
:10036000044654E8000F00EA010544E80053002B5E
:10037000F7D1156030BC704730B4044654E8000F24
:1003800080EA010544E80053002BF7D1156030BC2A
:10039000704730B4044654E8000F00EB010544E810
:1003A0000053002BF7D1156030BC704730B40446C1
:1003B00054E8000FA0EB010544E80053002BF7D1EF
:1003C000156030BC704770B404464FF0000054E82C
:1003D000006F0D68AE4207BF44E80023012044E8E7
:1003E00000630E60002B1CBF0020F0E770BC70475C
:1003F00030B4044654E8000F88422CBF451A054625
:1004000044E80053002BF5D1156030BC7047000064
:100410000648804706480047FEE7FEE7FEE7FEE79E
:10042000FEE7FEE7FEE7FEE7FEE7FEE7810C0000E1
:10043000010200000048704738FC0000A0F14101B3
:10044000192900D8203070472DE9FE4399461546FA
:100450008846074601AC022942D3002D40D0002037
:100460000290A8F101004FF0FF36009022E000FB5F
:10047000057201FB057011464A469047002805DCCD
:1004800054F82600304444F8260013E060682A46F9
:1004900000FB057154F8040C00FB057007E00B78B5
:1004A00090F800C001F801CB00F8013B521E002A71
:1004B000F5D1764254F8040C61688842D7DC4B468B
:1004C0002A463846FFF7C0FF54F8040C4B46A8EB09
:1004D0000001401C00FB05702A46491EFFF7B4FFCF
:1004E000BDE8FE8310B5431A934209D283188818D9
:1004F00003E010F8011D03F8011D521EF9D210BDD2
:1005000040EA01039B0703D009E008C9121F08C095
:10051000042AFAD203E011F8013B00F8013B521E15
:10052000F9D210BDD2B201E000F8012B491EFBD276
:1005300070470022F6E710B513460A4604461946EE
:10054000FFF7F0FF204610BD30B505462A460B46A2
:1005500012F8010B13F8014B08B1A042F8D01CB1FE
:10056000002802D06D1CF1E7284630BDCAB2401EFB
:1005700010F8011F8A4202D00029F9D100207047EB
:10058000421C10F8011B0029FBD1801A704710B5DE
:10059000002200E0521C835C8C5CA34201D1002B42
:1005A000F8D1D8B2E1B2401A10BD034611F8012BC0
:1005B00000F8012B002AF9D11846704730B50546DE
:1005C0000020034600E05B1C934205D2EC5CC85C53
:1005D000201A01D1002CF6D130BD2DE9F04791460B
:1005E0000F4680460446002614F8015B2DB1FFF744
:1005F00021FF0068405DC007F6D12B2D02D02D2DC4
:1006000018D0641E4A463946204600F01EF827B12D
:100610003968A14201D1C7F8008071054FF002048A
:100620000BD54042002803DD00F0AEFD0460A007BA
:10063000BDE8F08746F48066E4E70028F8DA00F0C9
:10064000A3FD04606FF00040F2E72DE9F05F824601
:100650000078002715468B460AF10104B946302878
:1006600001D09DB113E014F8010B0127782803D0C5
:10067000582801D045B10AE00DB1102D07D100274F
:10068000102514F8010B02E0082500E00A250026D9
:10069000B0460EE005FB080005FB06F1012701EB63
:1006A00010461FFA80F8B6F5803F00D3B94614F81B
:1006B000010B294600F02AF80028EBDABBF1000F05
:1006C00005D00FB1641E00E05446CBF80040B9F1EC
:1006D000000F06D000F058FD02210160C81EBDE8E1
:1006E000F09F48EA0640FAE7064C074D06E0E0684E
:1006F00040F0010394E8070098471034AC42F6D369
:10070000FFF782FD641B0100841B01003A2800D220
:10071000303820F02002412A01D3A2F1370088426C
:1007200001D34FF0FF30704770B58C1810F8015BA3
:1007300015F0070301D110F8013B2A1106D110F87A
:10074000012B03E010F8016B01F8016B5B1EF9D17E
:100750002B0705D40023521E0DD401F8013BFAE704
:1007600010F8013BCB1A921C03E013F8015B01F86F
:10077000015B521EF9D5A142D8D3002070BD000004
:100780002DE9F04F00268DB0DFF8A081B146049628
:100790004FF48075012437460596284609F076FF08
:1007A00038B1D8F80403204203D0284609F064FF8A
:1007B00026432D1D64007F1CADB2082FEDD34FF4EE
:1007C000BE74204609F062FF48B1204609F054FF8C
:1007D00046F0004604AA0221002009F017FF544CFD
:1007E00016F0FF0F15D00127002537420DD008EB7A
:1007F0008501D1F81005D1F81015C0F3052054F883
:100800002520C1F3014102B190477F006D1C082DE6
:10081000EBD3002E7EDA0020CDF82890411E0DF19A
:10082000100B07AACDF82C9042F82010401C9146DE
:100830000228F9D300252E46A11911F8607F91F9FD
:10084000000027F0C008401C40D007A9404607F030
:100850009BF940B34FEA971A404602F0CDFC54F89A
:1008600020701FB1BAF1030F03D006E0BAF1030FF5
:100870002CD10AA9404607F08FF902A8CDF80880CC
:1008800009F020FE029900EB8100D0F8000704A9CE
:10089000C0F301400290404607F076F90028029824
:1008A00002D0022802D011E003280FD1BAF1030FC1
:1008B00008D10298022833D00221404609F0EAFD0F
:1008C0006D1CEDB217B151464046B847761C042E58
:1008D000B2D3002D21D001AA0221002009F096FEFA
:1008E00000205A460DF1040152F8206051F82030E2
:1008F000B34217D000200AAE4FEA090351F8207026
:1009000042F8207056F8207043F82070401C0228EE
:10091000F4D300E001E0002D8CD10DB0BDE8F08FE4
:100920000321CAE7401C0228DED3F6E7006000403E
:10093000EC1900201CB581460AF0A4FA0AF03CF834
:100940000028FBD137484E460768374C01256068C0
:10095000002821D0208835A105EB0040B2690AF0BB
:1009600059F96068002817D0D6E90201CDE90001E5
:100970002088D6E9002305EB004032A10AF062F995
:10098000606848B1F0690090D6E9042320883BA153
:1009900005EB00400AF04DF92248001D0068800771
:1009A00007D5606828B120883E4905EB00400AF071
:1009B0002DF9DFF8F480002605FA06F038420AD057
:1009C00058F826203AB1606828B1208837A105EB95
:1009D00000400AF01FF9761C1A2EEDD338060AD50E
:1009E000606840B10F480C300268208832A105EBE6
:1009F00000400AF00FF938040AD5606840B1094890
:100A000010300268208834A105EB00400AF002F99A
:100A10000448C8300068C00700D000BE484600F057
:100A200069F8000028ED00E0180500204841524414
:100A3000204641554C542061742030782530385878
:100A400000000000202052303A2020307825303835
:100A500058202052313A2020307825303858202034
:100A600052323A2020307825303858202052333AFC
:100A700020203078253038580000000020205231E6
:100A8000323A2030782530385820204C523A2020F5
:100A900030782530385820205053523A203078256D
:100AA0003038580000070100500200204361757380
:100AB000653A2025732E00004D656D4D616E6167AE
:100AC00065204661756C7420416464726573733A85
:100AD0002030782530385800427573204661756C97
:100AE0007420416464726573733A2030782530381D
:100AF00058000000BFF34F8F05480168054A01F414
:100B0000E06111430160BFF34F8F00BFFDE70000BC
:100B10000CED00E00400FA0510B50BF049FEBDE84D
:100B200010400BF06BBD000002490248091F096824
:100B30000068084748020020044900EB400001EB30
:100B4000C000416D806D081A70470000FC23002032
:100B500000F064BA70B5064614460D46002001F058
:100B60001BFD22462946304600F006F804460020C8
:100B700001F040FD204670BD2DE9F0471B4D0746B2
:100B8000164628780C4608B900F048FA07EB4700EB
:100B900005EBC007A046D7E91595002448374D4519
:100BA00011D9B868441BB44200D334467868224651
:100BB00041194046FFF796FCB868361B2544A0440F
:100BC000A84200D10025A9EB0500B04200D206469C
:100BD0003EB17868324641194046FFF783FC344401
:100BE000354404B13D612046BDE8F087FC23002078
:100BF00070B50B4B0646144618780D4608B900F040
:100C00000DFA002001F0C8FC22462946304600F0CB
:100C100009F80446002001F0EDFC204670BD0000FC
:100C2000FC23002070B50E46144900EB400001EB98
:100C3000C0051446E86A183520B101280FD00228F3
:100C400005D113E0284600F01DFAA04201D200248D
:100C500011E022463146284600F061FA0BE02846B2
:100C600000F010FAA042F4D20446F2E731462846DA
:100C700000F028FA0446204670BD0000FC23002046
:100C800030B54FF0805000228300D0F83011C3F807
:100C90000C21C3F81021624B1A60624B1B68624C36
:100CA0002360604B1B1D1B68241D23605D4B0833B4
:100CB0001B68241D23605B4B0C331B68241D2360C1
:100CC000584B10331B68241D2360564B14331B688C
:100CD000241D2360534B18331B68534C203423606E
:100CE000504B1C331B68241D23604E4B20331B6864
:100CF000241D23604B4B24331B68241D2360494B68
:100D000028331B68241D2360464B2C331B68241D8D
:100D10002360444B30331B68434C40342360414BC9
:100D200034331B68241D23603E4B38331B68241D5D
:100D300023603C4B3C331B68241D2360394B4033FC
:100D40001B68241D23600124082902D1D0F8343106
:100D500013B1082904D006E0354B3449196005E089
:100D6000D0F8343113B1082904D006E0314BFB210F
:100D7000196005E0D0F8343113B1082908D00EE02D
:100D800090F858322C48016863F30301016002E0D7
:100D9000D0F834311BB929494FF400700860284855
:100DA0000168C90702D06FF00101016025480168A0
:100DB00041F470010160BFF34F8FBFF36F8F4FF0AD
:100DC0001021D1F80002002803DBD1F8040200282A
:100DD00022DA1D4B1C601D480468002CFCD0122434
:100DE000C1F800420568002DFCD0C1F8044201683A
:100DF0000029FCD01A6001680029FCD0BFF34F8F96
:100E000010487C380168124A01F4E0611143016026
:100E1000BFF34F8F00BFFDE70F490E48086030BD9C
:100E2000380500400404001020C50040488103003C
:100E30008C56004018F50040E40E004040960240F9
:100E40000004004088ED00E004E5014000E40140BA
:100E50000400FA050090D0037003002010B5054C83
:100E6000206818B904A12B2001F07AFC2068BDE8A5
:100E700010400047C40100202E2E5C2E2E5C2E2E2A
:100E80005C2E2E5C2E2E5C2E2E5C6D6F64756C6558
:100E9000735C6E7266785C647269766572735C739B
:100EA00072635C7072735C6E7266785F7072732EC0
:100EB000630000002DE9F05F5448D0F8045300248B
:100EC0002E464FF0010913E096FAA6F0B0FA80F72B
:100ED000B80000F5807080460BF092FA28B14046C9
:100EE0000BF096FA09FA07F0044309FA07F0864373
:100EF000002EE9D108F060FB002869D0444AD07880
:100F0000F0BBA00264D5434940F2A978C1F8008043
:100F1000081D036813F0FF0C02D0036803EA0C0CF1
:100F200040F2AA7AC1F800A0036813F0FF0301D0D1
:100F30000668334040F2AB7BC1F800B0066816F09B
:100F4000FF0601D007683E4040F2AC770F600768AB
:100F500017EA0C0709D0D2F810C04CEA070CC2F807
:100F600010C0C1F800800760076840F2AD770F60DD
:100F700007681F4009D0136943EA0743136100E083
:100F800026E0C1F800A00760036840F2AE730B6072
:100F9000036833400BD0DE0701D044F40004DE06C2
:100FA00001D544F00104C1F800B003600068106985
:100FB00030F0011102D005F080710C4310F0011FD8
:100FC00006D0690504D520F0011044F48064106156
:100FD000C4F3C05624F400044F46DFF83C8009E017
:100FE00094FAA4F0B0FA80F558F82500804707FA83
:100FF00005F08443002CF3D10DF012FE002E03D037
:10100000BDE8F05F05F0ACB8BDE8F09F00700240AD
:101010009401002000780240A8F3000010B5124CA3
:1010200002202061606111A0A06104F17800E061FC
:101030004FF4007020620020A06260620BA1A164E6
:10104000E06204F51E71E1641021A065C4E914108A
:10105000E06509A1E01DFFF7A8FA08A12046FFF707
:10106000A4FA2020A07110BDFC2300205465726DED
:10107000696E616C000000005254540053454747AC
:10108000455200000269C1688A4203D88068401A4C
:10109000104400E0501A401E70470000C11700EBDA
:1010A000D161074B4A1153F8222021F01F01411A48
:1010B00001208840024201D0012070470020704783
:1010C00000E100E02DE9F047C4681746894606466E
:1010D0004FF000083069A04201D9051B02E0B16859
:1010E000201A0D1AB0686D1E001BA84200D80546D4
:1010F000BD4200D33D4670682A4620444946FFF76A
:10110000F1F9B0687F1B2C44A844A944A04200D147
:101110000024F460002FDDD14046BDE8F0872DE9C2
:10112000F04104468846D4E90207C51BE1686068BF
:1011300016460844B54206D94146FFF7D3F9B81917
:10114000E060BDE8F0812A464146FFF7CBF9761B07
:1011500008EB050132466068FFF7C4F9E660F0E786
:101160000FB4084B10B504A902AA039800F01FF8A9
:10117000044602A9002000F085F8204610BC5DF866
:1011800014FB000085120000004870477403002023
:1011900002E008C8121F08C1002AFAD17047704740
:1011A000002001E001C1121F002AFBD170472DE988
:1011B000F84F9946924688460546002706E02528BE
:1011C0000AD051464A4690476D1C7F1C287800285B
:1011D000F5D13846BDE8F88F002315F8011F1846F1
:1011E0002E2915D115F8011F04232A290DD06FF0DF
:1011F0002F022978A1F13004092C09D800EB8000D6
:1012000002EB400008446D1CF3E758F8040B6D1C1A
:101210002A78002ADDD0632A07D0732A0FD010461F
:1012200051464A4690477F1C2AE018F8042B8DF857
:10123000002000218DF801106E46012103E058F8CE
:10124000046B4FF0FF315A074FF0000401D409E05E
:10125000641C84420BDA8C42FADB325D002AF7D13F
:1012600005E0641C8C42FCDB305D0028F9D127448A
:1012700004E016F8010B51464A469047641EF8D226
:101280006D1CA3E70A68531C0B6010707047800741
:1012900001D00020704701207047C3688B4206D8F8
:1012A00011440069491E814201D801207047002085
:1012B000704700002DE9FE4315460F46804672B682
:1012C00009F0E0FD09F078FB0028FBD16FF48041C4
:1012D000224C18EB01004FF0010622D00128606873
:1012E00014D030B120883A4606EB00401CA109F02A
:1012F00091FC21480068C00700D000BE2A4603B018
:1013000039464046BDE8F04300F064B80028F0D00C
:1013100020882B8806EB004018A16A6809F081FC40
:10132000E7E760680028E4D0A8680AF0BBFE03463F
:10133000D5E90001CDE900100297208816A106EB3F
:101340000040AA6809F088FC60680028D1D0208895
:101350001BA106EB004009F059FCCAE784050020F8
:10136000554E4B4E4F574E204641554C54206174BC
:101370002030782530385800F0ED00E041535345D7
:101380005254494F4E204641494C454420617420F7
:1013900025733A25750000004552524F522025759D
:1013A000205B25735D2061742025733A25750D0A35
:1013B00050432061743A203078253038780000009E
:1013C000456E64206F66206572726F722072657060
:1013D0006F72740008B501238DF800309DF800305D
:1013E000144B186059609A606FF48041401807D020
:1013F00001280FD1DA60D86800889861D86807E0C2
:101400001A611869806858611869006898611869DC
:101410004068D861186858689868D8681869586929
:101420009869D86972B600BF9DF800000028FBD10A
:1014300062B608BDA81A0020014804F0F6BA000000
:10144000D401002070B514460E46050004D10B49A6
:1014500040F2C51001F084F93CB12868012EC46047
:101460000AD000218160002070BD04494FF4E37070
:1014700001F076F9072070BD0121F3E74004010077
:1014800038B50E4808235822416800910C4900687D
:1014900006F075F900280FD10A4A69460A4804F097
:1014A000C9FA040008D10121074804F09AFB064953
:1014B000012008390870204638BD000054F40000AF
:1014C000C81A002085D60000D401002070B5164649
:1014D0000D46040004D10C4940F2D51001F040F94A
:1014E0000A48854201D9072070BD0948266104F0E9
:1014F0009CFA28446060A06800B1A5602146BDE860
:10150000704000200CF0C0BF4004010017FCFF0039
:10151000D401002010B5040004D106494FF4F57041
:1015200001F01EF9002021462076BDE81040012080
:101530000CF0AABF4004010070B505460648446897
:1015400007E02946204601F0D1FF204600F022FAAC
:101550000446002CF5D170BDF401002070B50A4896
:1015600045680EE02E7A002405E02146284600F06A
:1015700015FE641CE4B2B442F7D3284600F00AFA20
:101580000546002DEED170BDF40100202DE9F0419B
:101590000E4840F2AB67456814E02E7A00240BE059
:1015A00000222146284600F05DFE18B108A1384609
:1015B00001F0D6F8641CE4B2B442F1D3284600F03E
:1015C000E9F90546002DE8D1BDE8F081F4010020DD
:1015D0002E2E5C2E2E5C2E2E5C2E2E5C2E2E5C2E45
:1015E0002E5C636F6D706F6E656E74735C6C696298
:1015F0007261726965735C757362645C6170705F5F
:10160000757362642E63000070B5064609480625AE
:1016100044680AE03146204601F068FF0546062886
:1016200005D1204600F0B6F90446002CF2D1284638
:1016300070BD0000F40100202DE9FC4115460F00AB
:10164000064604D11E494FF47C7001F089F83046FB
:1016500001F010F90446007DC00715D0002000F00D
:101660009BFFE06E98B1A84200D805462A4638464E
:10167000A16EFEF737FFE06E401BE066A06E656767
:101680002844A066002405E00820BDE8FC81A0698C
:1016900028B11124002000F0ADFF2046F5E7C4E991
:1016A0000675304604F0A7F906498969CDE90014AA
:1016B000694600F0A3FB0400ECD19224EAE70000A5
:1016C000CC040100B4F4000010B501F0D3F8406F71
:1016D00010BDFEB515460E46044601F0CBF8007D60
:1016E00010F0010F0AD0204604F07CF9002100968A
:1016F000CDE90151694600F0CDFBFEBD0820FEBDDD
:10170000F8B5040004D138A140F2EF4001F028F808
:10171000606820B934A14FF49E6001F021F8606840
:10172000006820B930A140F2F14001F019F82068BA
:10173000006820B12CA140F2F24001F011F808F04D
:10174000C7F810B908F0CEF820B927A140F2F6404A
:1017500001F006F800250FE0002705E0007800F012
:1017600061FB08B11120F8BD3946781CC7B230467C
:1017700000F0C0F80028F1D12946681CC5B2204607
:1017800000F0E0F80600E7D100250DE0002703E0B7
:101790000078214600F04CFB3946781CC7B2304631
:1017A00000F0A8F80028F3D12946681CC5B22046ED
:1017B00000F0C8F80600E9D1194D40F21C5607E0C8
:1017C000A04203D108A1304600F0CAFF286805688E
:1017D00028680028F4D113482C60694640690090BD
:1017E000204601F083FEF8BD2E2E5C2E2E5C2E2EA0
:1017F0005C2E2E5C2E2E5C2E2E5C636F6D706F6ED9
:10180000656E74735C6C69627261726965735C7534
:101810007362645C6170705F757362642E63000054
:10182000F801002068F400002DE9F04F87B04FF078
:1018300000081D46934689460446DDF840A046460A
:10184000CDF80C8000E0761C606801230022476818
:10185000214603A8B8470028F5D140468DF80080FE
:101860000027B84601903BE0606801236A46D0F843
:1018700004C0214601A8E0476068012305AAD0F80A
:1018800004C0214601A8E0479DF8141049451AD12B
:10189000D84514D19DF80000CAF8000005F8010BE6
:1018A0006A1C85F8009060689DF800302146456804
:1018B00001A89B1EA847002007B0BDE8F08F08F1E3
:1018C000010000F0FF0860689DF800300022D0F8A9
:1018D00004C0214601A89B1EE0479DF80000074474
:1018E000B742C1D30520E7E70148406870470000D0
:1018F000F401002070B50D46040004D106494FF4F0
:101900008E7000F02DFF6078A84201D8002070BDD5
:10191000A0782044284470BD8804010070B50D46AD
:10192000040004D106494FF48E7000F019FF60786E
:10193000A84201D8002070BDA0782044284470BD82
:101940008804010070B50D46040003D10649E92062
:1019500000F006FF207AA84201D8002070BD05EBF8
:1019600045000934204470BD8804010070B50D465F
:10197000040003D10649E92000F0F2FE207AA842D3
:1019800001D8002070BD05EB45000934204470BD2E
:101990008804010010B5040004D104494FF4F97023
:1019A00000F0DEFE2068006810BD00000421000089
:1019B00010B5040004D104A14FF4F97000F0D0FE7A
:1019C0002068006810BD00002E2E5C2E2E5C2E2E8E
:1019D0005C2E2E5C2E2E5C2E2E5C636F6D706F6EF7
:1019E000656E74735C6C69627261726965735C7553
:1019F0007362645C6170705F757362642E6800006E
:101A000002484078002800D001207047F4010020EF
:101A10002DE9F041484E0D460246097806243078FB
:101A200001270F2964D2DFE801F063080C0E632060
:101A30004863636363252D363F0003200CF0F6FFF7
:101A400056E0002454E03C48001D05F0DAFE28B1C1
:101A50003A480760BFF36F8FBFF34F8F307800288D
:101A6000EFD137A140F20B4009E0104600F0A4F896
:101A700004463DE00028E4D031A140F2164000F0D9
:101A80006FFEDEE7012804D02DA140F21C4000F0DB
:101A900067FE002005E03948006810F0010F0AD009
:101AA00002200CF0C3FFCCE7022804D224A14FF49B
:101AB000866000F055FE0120F3E7E878032817D090
:101AC000A87830B1802804D01DA140F23E4000F03B
:101AD00047FE1949E87808310A6832B100230B60E3
:101AE00049689047040006D000E00E2407F054FF38
:101AF0002046BDE8F0810CF091FF28B1A8780028BD
:101B0000F6D107F00CFFF3E71D480078082810D144
:101B10001B48001D007800070BD1194808300078D9
:101B200010F0F00F05D116480C30007810F0F00FCF
:101B3000DED007F0F1FEDBE7140200205C7002400B
:101B40002E2E5C2E2E5C2E2E5C2E2E5C2E2E5C2ECF
:101B50002E5C636F6D706F6E656E74735C6C696222
:101B60007261726965735C757362645C6170705FE9
:101B7000757362645F636F72652E630038040040A2
:101B8000E00F00F0024A0146D2E9000210470000CF
:101B9000681B002070B50C46054607F0B7FEA8424A
:101BA00001D0102070BD0348D4E90012C0E9021230
:101BB000002070BD140200207FB5054605208DF879
:101BC000000006240DF1010007F0BEFE0CF026FF18
:101BD0002949002008609DF8010010F01F0006D080
:101BE00001280FD0022826D0032833D106E0694609
:101BF00028460BF085FF044606282AD16846FFF7E1
:101C000003FD25E09DF8050003A900F007FB050092
:101C100008D06A469DF80C1000F0BCFA044606286D
:101C200002D016E0102415E06A469DF80C102846F4
:101C30000CF0C0F80CE09DF80500010705D06946DE
:101C400000F080F80446062803D168460CF002F83C
:101C5000044624B107F0A0FE04B0204670BD0CF08D
:101C6000DDFE30B107F052FE0028F5D107F057FE37
:101C7000F2E707F051FEEFE71C020020FEB5C08836
:101C800014460E46A04201D2054600E015468442A5
:101C900007D2802007F0B6FAB4FBF0F100FB114048
:101CA00068B100200096CDE90150002000F074FCDE
:101CB0006946802000F0EEF8040002D006E0012022
:101CC000F0E705498020FFF765FF0446002000F09B
:101CD00091FC2046FEBD0000E4F4000008B1402164
:101CE0000160014870470000BC1B002010B507F0E0
:101CF00001FE20B104A140F26F3000F031FDBDE8DB
:101D0000104007F081B800002E2E5C2E2E5C2E2E87
:101D10005C2E2E5C2E2E5C2E2E5C636F6D706F6EB3
:101D2000656E74735C6C69627261726965735C750F
:101D30007362645C6170705F757362642E6300002F
:101D400007F0A4B810B50C46010600F00F02092AEE
:101D500008D200F009F8006820B12146BDE8104023
:101D600001F0C4BB102010BD10B5010600F00F0437
:101D700008D5092C04D309A140F2611000F0F0FC51
:101D8000144808E0092C04D304A140F2671000F0C5
:101D9000E7FC1048483000EBC40010BD2E2E5C2E2E
:101DA0002E5C2E2E5C2E2E5C2E2E5C2E2E5C636FF7
:101DB0006D706F6E656E74735C6C6962726172696E
:101DC00065735C757362645C6170705F7573626487
:101DD0002E630000201B002010B5044600F00F0009
:101DE000082805D2204607F035F9204607F08EFA7C
:101DF0002046BDE8104007F051B9000070B50C4610
:101E0000054607F09BF918B105480078022801D073
:101E1000082070BD21462846BDE8704007F096B9FD
:101E2000F401002010B5FFF79FFF006810BD00000F
:101E300070B50D460646FFF797FF0446056015B1DD
:101E40006868006808E00EB1802E04D103A140F25A
:101E50008B1000F085FC0020606070BD2E2E5C2E83
:101E60002E5C2E2E5C2E2E5C2E2E5C2E2E5C636F36
:101E70006D706F6E656E74735C6C696272617269AD
:101E800065735C757362645C6170705F75736264C6
:101E90002E63000070B50C46054607F04FF918B1E7
:101EA00005480078022801D0082070BD2146284648
:101EB000BDE8704007F0BABAF40100200149096892
:101EC00008470000B01B002070B57D4C05466068D7
:101ED00020B97CA140F2C33000F042FC03F0CEFBFD
:101EE000072804D277A140F2CA3000F039FC2878E4
:101EF000092872D007DC16D2DFE800F07085A98CC3
:101F000096B2B715DA00812814D006DC0A28F0D082
:101F10000F28EED0802806D13CE082281FD08328ED
:101F200043D084284AD0BDE8704066A140F2AB405F
:101F300000F016BC7148FFF725FE7048FFF7FCFA69
:101F40000D200DF043F8A06810B96D48007A00B17B
:101F5000012007F025FDFFF701FB012073E0FFF7EB
:101F6000FDFA07F073FD00200CF0D6F86348401C22
:101F7000FFF7E2FA6148401CFFF704FE0E200DF067
:101F800025F8207800F0EEFA00283BD0BDE870403C
:101F900006F06ABD2078052803D0062803D007285C
:101FA00030D102204FE008204DE02078032829D1CD
:101FB00007F096FD002825D0042044E0207803286F
:101FC00005D107F08DFD10B104200CF0A5F807F045
:101FD00057FE002816D0062035E06AE000200CF0FD
:101FE000F5FFA46840F20E260AE02946204601F0DB
:101FF0007DFA1CB943A1304600F0B2FB206844686A
:10200000002CF2D170BDFFF7A9FA02200CF084F881
:10201000012003E005200CF07FF803200CF0D6FF30
:102020002846FFF7AFFD46E003200CF0CFFF334812
:10203000801CFFF7A7FD3148801CFFF77DFA207850
:102040000628AED10720BDE870400CF065B803202B
:102050000CF062F802200CF0B9FF2846FFF76CFA8A
:102060002846BDE87040FFF78DBDA878FFF77CFEDD
:102070000446006820B913A140F2874000F070FBCD
:10208000606820B90FA14FF4916000F069FBD4E9BA
:102090000002294690470028B4D0A8780107B1D0A3
:1020A00000F00F010829ADD2BDE8704007F0FCB880
:1020B00008200CF08BFF2846BDE87040FFF73CBAC3
:1020C000F40100202E2E5C2E2E5C2E2E5C2E2E5C1B
:1020D0002E2E5C2E2E5C636F6D706F6E656E74734A
:1020E0005C6C69627261726965735C757362645C71
:1020F0006170705F757362642E63000079F4000094
:10210000B01B00202E2E5C2E2E5C2E2E5C2E2E5C04
:102110002E2E5C2E2E5C636F6D706F6E656E747309
:102120005C6C69627261726965735C757362645C30
:102130006170705F757362642E680000FFF7BEBE49
:1021400010B520B104A140F2272000F009FBBDE842
:1021500010400F48FFF7B2BE2E2E5C2E2E5C2E2EA6
:102160005C2E2E5C2E2E5C2E2E5C636F6D706F6E5F
:10217000656E74735C6C69627261726965735C75BB
:102180007362645C6170705F757362642E630000DB
:1021900068F40000114601F0A9B9000070B50446CA
:1021A00040680D46C2680AB120469047207AA8428E
:1021B00004D20CA140F2BF2000F0D2FA29462046FA
:1021C000FFF7C0FB05464678002408E02146284674
:1021D000FFF790FB007806F00DFF641CE4B2B442F8
:1021E000F4D370BD2E2E5C2E2E5C2E2E5C2E2E5C1B
:1021F0002E2E5C2E2E5C636F6D706F6E656E747329
:102200005C6C69627261726965735C757362645C4F
:102210006170705F757362642E6300002DE9F04198
:1022200080460F480E46456816E02F7A00240DE0E0
:1022300021462846FFF786FB0178414504D106B1C7
:1022400034702846BDE8F081641CE4B2BC42EFD390
:102250002846FFF79FFB0546002DE6D10020F1E759
:10226000F401002070B50446406815460E468368A8
:102270001BB120469847062809D1207AB04204D2E3
:102280000E494FF4287000F06BFA0DB1072070BDB5
:1022900031462046FFF756FB05464678002408E005
:1022A00021462846FFF726FB0078FFF795FD641CC2
:1022B000E4B2B442F4D3002070BD0000E421000079
:1022C000034600205A681269002A01D018461047B8
:1022D000704700002DE9F843044606F073FC20B96E
:1022E0002FA14FF4367000F03BFA3B4807F0AEFAEE
:1022F000002850D139490870486088604821384822
:10230000FEF717F9364848214830FEF712F93448ED
:10231000344D80304CB194E80E00103080E80E004F
:102320002F489030016821B105E005F12C010EC95C
:10233000F3E72D490160002006F09AFC30B18528B2
:1023400004D017A240F20631FDF764FF274E0024A7
:102350000DE0002703E000783146FFF769FD3946BC
:10236000781CC7B24046FFF7C5FA0028F3D12146D2
:10237000641CE4B23046FFF7E5FA5FEA0008E8D1F2
:10238000686800906946304601F0B0F8040004D057
:1023900007F068FC2046BDE8F8830020FBE700005A
:1023A0002E2E5C2E2E5C2E2E5C2E2E5C2E2E5C2E67
:1023B0002E5C636F6D706F6E656E74735C6C6962BA
:1023C0007261726965735C757362645C6170705F81
:1023D000757362642E6300003D210000F40100204B
:1023E000201B002068F40000C91E000024F5000036
:1023F00040B1012808D0022809D007A140F20E20E0
:1024000000F0AEB9124804E01148001D01E0104888
:102410000830FFF753BD00002E2E5C2E2E5C2E2EB2
:102420005C2E2E5C2E2E5C2E2E5C636F6D706F6E9C
:10243000656E74735C6C69627261726965735C75F8
:102440007362645C6170705F757362642E63000018
:1024500082F4000010B507F045FA10B107F038FA21
:1024600008B1082010BD054806F012FC20B104A2F6
:102470004FF45871FDF7CEFE002010BD90F400001F
:102480002E2E5C2E2E5C2E2E5C2E2E5C2E2E5C2E86
:102490002E5C636F6D706F6E656E74735C6C6962D9
:1024A0007261726965735C757362645C6170705FA0
:1024B000757362642E63000010B507F009FA20B945
:1024C00009A140F2763000F04BF915480168C1F3DC
:1024D000400121B1BDE810401248FFF7EFBC016890
:1024E00011F0010FF2D110BD2E2E5C2E2E5C2E2E7F
:1024F0005C2E2E5C2E2E5C2E2E5C636F6D706F6ECC
:10250000656E74735C6C69627261726965735C7527
:102510007362645C6170705F757362642E63000047
:10252000380400406DF40000034808B5806800904E
:102530006846FFF7C3FC08BD68F40000074918B1FE
:10254000052803D30020704708687047044A105CD0
:102550000028FAD051F82000704700002C0200201B
:10256000B0F50000092808D2DFE800F007070507EA
:102570000705050505000120704700207047092860
:1025800008D2DFE800F0070705070707070705007F
:10259000012070470020704710B50AF05FFF012846
:1025A00003D004A11D2000F0DBF8BDE8104000F0CE
:1025B0004FB800002E2E5C2E2E5C2E2E5C2E2E5C34
:1025C0002E2E5C2E2E5C636F6D706F6E656E747355
:1025D0005C6C69627261726965735C7574696C5C6C
:1025E0006170705F7574696C5F706C6174666F7236
:1025F0006D2E630010B50AF031FF012803D004A14D
:102600002B2000F0ADF8BDE8104000F029B8000024
:102610002E2E5C2E2E5C2E2E5C2E2E5C2E2E5C2EF4
:102620002E5C636F6D706F6E656E74735C6C696247
:102630007261726965735C7574696C5C6170705FFE
:102640007574696C5F706C6174666F726D2E630077
:1026500072B602480168491C0160704740020020C0
:1026600003490868401E086000D162B67047000048
:102670004002002070B5054608680C46411C04D095
:1026800007F0B0FF206807F0F1FE6068411C02D03F
:10269000002107F0D9FE2968A069C1F82405607DF2
:1026A000227D29681043C1F86C05D4E9001228681E
:1026B000C0F81425C0F80C15207D012814D1A0689D
:1026C000411C02D0002107F0BFFEE068411C04D08D
:1026D00007F088FFE06807F0C9FED4E90212286815
:1026E000C0F80825C0F8101570BD70B5054608681B
:1026F0000C46411C04D007F07FFF206807F0C0FEA5
:102700006068411C02D0002107F0A7FE2968A0697B
:10271000C1F82405607D217D2A680843C2F86C0554
:10272000D4E900122868C0F80C15C0F81425207DE3
:10273000012814D1A068411C02D0002107F08DFEB1
:10274000E068411C04D007F057FFE06807F098FEEE
:10275000D4E902122868C0F80825C0F8101570BD29
:102760001CB56A46ADF800000191002144F2020058
:10277000FEF7A0FD1CBD102802D31038C0B2704770
:1027800040F08000704700002DE9F0470546C61C68
:1027900090460F464FF001090020FFF7FDFE1B4C4D
:1027A00020683860D4E90001401AA16804F21C478F
:1027B000081A0EE00121384605F02CF804F076FCEA
:1027C0000146384605F026F8D4E90001401AA16810
:1027D000081A401C8642EDD8B8F1000F03D005203E
:1027E00065F3891002E0062065F39F50A268216816
:1027F000114004EB8101C860206830442060002053
:10280000FFF7F8FE4846BDE8F0870000D81F00201B
:1028100030B482680468531C8360A154D0E901126B
:102820008A4202D330BC07F093BA30BC7047000034
:10283000034803C8814201D101207047002070473E
:10284000D81F00204360CA699A420DD38A6902608A
:10285000886918448861086F18440867C869C01AF5
:10286000C86100D00120704701F1280202600020F9
:102870008B67704710B5040003D106493920FFF774
:102880006FFF206818B903493A20FFF769FF2068F5
:10289000083010BDCC04010070B50C46060004D110
:1028A000224940F2B720FFF75BFF24B91F494FF4DC
:1028B0002E70FFF755FF207800250F2833D2DFE870
:1028C00000F033083333320C1132320832333333F1
:1028D0003300304600F0D3FB26E0214630460BF0B3
:1028E00003FA0FE0304602F0B6FD0146A07800255D
:1028F000814219D00106E1784FF0030004D531B9C7
:1029000001210CE005460FE021B101290CD003297B
:10291000F8D109E0304600F0C3FB054600213046FF
:102920000CF046FB00E00625284670BDCC040100F3
:102930002DE9FF5F05460198DFF8F0931F46017A05
:1029400089F800101646019800F042FB804625B930
:10295000F74940F2E920FFF703FF29684FF0000A2A
:1029600040F21F325446A1F21F304FF0020B914249
:1029700056D04CDC40F20132A1F20130914272D0CB
:1029800029DC40F2F120A1F2F12281426CD015DC69
:1029900040F2EE22A1F2EE2391426ED009DC4FF418
:1029A0003B73E1B3994270D0A1F50071ED395ED16E
:1029B0007AE0012B74D0022B59D19BE0092A70D008
:1029C00004DC012A6ED0022A51D1B7E00A2A6AD06B
:1029D0000F2A4CD1DDE00E2871D00EDC07286ED016
:1029E00006DC01286CD005286BD006283FD116E103
:1029F0000C2867D00D283AD138E11538092836D28D
:102A0000DFE800F0F535353535F4F3F2F100132841
:102A10006FD010DCA0F10300102828D201E02EE0D6
:102A200079E1DFE800F0F0EFEEEDEC2424EBEAE9E9
:102A3000E82424E7E6E537280CD00CDC292878D0F8
:102A400004DC142876D0282811D125E22D2872D054
:102A500032280CD150E244286ED006DC3E286CD0DF
:102A60003F2804D16FE29FE04CE04928F4D00020D9
:102A7000C5F800A004B0BDE8F09F24E005E00821FF
:102A80002971002F01D82B607FE20EB129793170B6
:102A90000B2101242971012F06D840F2ED2073E2A9
:102AA0001CE059E03AE062E00EB12979315598F81E
:102AB0001410641C2971BC4205D32A6065E2BAE097
:102AC0007FE0A1E0C7E00EB129793155641C85F89B
:102AD00004B0BC4202D340F2EF2055E20EB1297996
:102AE0003155641C85F804B0BC4203D34FF43C70EC
:102AF0004AE2A6E10EB129793155641C85F804B08B
:102B0000BC42CCD20EB12879305598F81900641C1B
:102B10002871BC4202D340F2F22035E20EB128798E
:102B20003055641C85F804A0BC4207D340F2F32062
:102B30002AE2BCE191E1CDE117E2F9E10EB1287999
:102B4000305589F801A0641C35E209202871BC4287
:102B500002D340F2FA2017E20EB128793055042052
:102B6000641C2871BC4202D340F2FB200CE20EB17F
:102B70002879305599F80110641C0198FEF7F6FE8B
:102B8000C9F8040000782871BC4202D34FF44070A9
:102B9000FAE10EB128793055641C85F804A0BC42D6
:102BA00002D340F20130EFE10EB128793055D9F867
:102BB0000400641CBC424078287102D340F2023009
:102BC000E2E10EB128793055D9F8040098F81410D4
:102BD000641C0078814233D185F804B0BC4213D321
:102BE00040F20630D0E18BE07FE073E067E054E034
:102BF0001BE10FE103E1F7E0EBE0DFE0D3E0C7E04A
:102C0000B9E0ADE0A1E095E00EB128793055641C43
:102C100085F804B0BC4202D340F20730B4E10EB1F3
:102C20002879305598F81900641C2871BC4202D3E9
:102C30004FF44270A8E10EB128793055641C25E0AC
:102C400098F8161081421CD10A202871BC4202D388
:102C500040F20D3098E10EB128793055641C85F8AA
:102C600004A0BC4202D340F20E308DE10EB12879AF
:102C70003055641C85F804A0BC42DCD340F20F3010
:102C800082E12B4940F21330FFF76AFD85F804A07A
:102C9000BC4202D340F2163076E10EB128793055AD
:102CA000D9F8040098F81410641C007881426ED1A1
:102CB00005202871BC4202D340F21B3064E10EB102
:102CC000287930552420641C2871BC4202D34FF46B
:102CD000477059E10EB128793055641C85F804A07D
:102CE000BC4202D340F21D304EE10EB1287930557E
:102CF0001020641C2871BC4202D340F21E3043E114
:102D00000EB1287930550120641C2871BC4202D3D1
:102D100040F21F3038E10EB1287930550520641C8F
:102D20002871BC4206D340F222302DE10802002077
:102D3000CC0401000EB1287930552420641C287180
:102D4000BC4202D340F223301EE10EB12879305547
:102D50000120641C2871BC4202D34FF4497013E176
:102D60000EB1287930550320641C2871BC4202D36F
:102D700040F2253008E10EB12879305598F8160058
:102D8000641C2871BC4203D340F22630FCE069E0A9
:102D90000EB1287930550420641C2871BC4202D33E
:102DA00040F22930F0E00EB1287930552420641C1F
:102DB0002871BC4202D340F22A30E5E00EB12879F6
:102DC0003055641C85F804B0BC4202D340F22B306D
:102DD000DAE00EB128793055641C85F804B0BC42A5
:102DE00002D34FF44B70CFE00EB128793055052057
:102DF000641C2871BC4202D340F22F30C4E00EB1F3
:102E0000287930552420641C2871BC4202D34FF429
:102E10004C70B9E00EB1287930550620641C287139
:102E2000BC4202D340F23130AEE00EB128793055C9
:102E300098F81400641C2871BC4202D340F232306E
:102E4000A2E00EB12879305598F81600641C28715C
:102E5000BC4202D340F2333096E00EB128793055AF
:102E6000641C08E098F81610814204D057494FF4CA
:102E70004F70FFF775FCD9F804104846497889F877
:102E80000210514689F803A08CE007202871BC424B
:102E900002D340F2473077E00EB128793055052053
:102EA000641C2871BC4202D34FF452706CE00EB126
:102EB0002879305599F80310641CD9F80400FEF7FE
:102EC0002DFDC9F8080000782871BC4202D34FF4E8
:102ED000537059E00EB128793055D9F8040098F8AC
:102EE0001410641C007881420BD103202871BC426D
:102EF00002D340F2513047E00EB128793055641CBE
:102F00000FE098F81610814206D185F804B0BC4253
:102F1000F2D340F2563037E02C4940F25A30FFF7F6
:102F20001FFC40202871BC4202D340F25D302BE0F0
:102F30000EB128793055641C85F804A0BC4202D338
:102F400040F25E3020E00EB128793055D9F8040007
:102F500098F81410641C007881420BD1102028715D
:102F6000BC4202D340F263300EE00EB128793055F6
:102F7000641C11E098F81610814208D185F804A06D
:102F8000BC42F2D34FF45A702860012072E50F4919
:102F90004FF45B70FFF7E4FB99F803104846491CB7
:102FA00089F803108278C9B29142FFF46EAF41787C
:102FB000491C89F8011099F8011099F80000814224
:102FC000FFF4C3AD40F27330DEE70000CC04010033
:102FD00010B5040003D103492C20FFF7C1FB2046A4
:102FE00010BD0000CC04010070B50546144808F07F
:102FF000BFFB30B9134800684068D0E900210020C9
:103000009047402210491148FEF716FB38B192282C
:1030100015D0BDE870400E4A4B21FDF7FBB828469D
:10302000FEF752FB044602460749054808F056FBE6
:103030008442DBD006494220FFF792FBD6E770BD01
:10304000001E0100BC020020281D002028F80000FE
:103050001C0F010010B508B1032010BD0846FFF792
:1030600009FC0178202901D0062010BDD0F80210FB
:10307000C160C1880182017A8174002010BD10B541
:10308000FFF7A6FFFFF7F6FB002181828161016255
:10309000C16601674167816700F12801816610BD43
:1030A0002DE9FC478146FFF793FFFFF7E3FB04465A
:1030B000484602F0A0FC07462F4800268068CDE96C
:1030C0000004E069B0B1D4F878804546404500D2AC
:1030D00005462A4604F12801A069FDF703FA206F8E
:1030E0002844C4E91C60A8EB0500E066601928309C
:1030F000A06627E0206F60672667E666216A304693
:1031000021B1626AA161C4E907202CE0A06130E02E
:1031100004F11802616A82E84300E26E1AB38A423F
:1031200015D3A36E0A461946FDF7DCF9E16EE06996
:10313000091AE166A16E0144A16660670021484654
:103140000BF036FF206A0028E2D1A66111E0A16EE3
:10315000FDF7C8F9E06E2067E169091AE161A1692C
:103160000818A06105D069463846FEF747FEBDE85D
:10317000FC870020FBE70000B4F400004360CA694C
:103180009A4204D38A6902600B67CB6103E001F1C4
:10319000280202608B6700207047000070B504466B
:1031A00081B1012905D002291CD1BDE87040FFF78B
:1031B0001BBF0D4800684068D0E90021BDE87040A1
:1031C00001201047FEF780FA0546024607490848E5
:1031D00008F084FA854203D006496C20FFF7C0FA54
:1031E0002046E2E770BD0000BC020020281D002040
:1031F000001E01001C0F01000249084490F9300034
:1032000070470000EC19002070B5816804464A8BB5
:10321000002A4DD0888B00284AD0121A084495B253
:1032200000F120016A1C1F30FDF75CF9A068818B5A
:10323000491E8183A068418B491E41838DB30822BA
:103240001C49206906F044FD204604F070FA81888C
:10325000C088814211D1A06817A2818B4318082130
:103260002046203305F068F8204600F0BDF92946D5
:103270002046BDE8704002F08BBA204600F020FAEC
:10328000204600F0B1F9A0680BA2818B43180821F9
:103290002046203305F050F82046BDE8704000F08D
:1032A000D9B92069BDE87040044A03A106F010BDF9
:1032B00070BD0000E834000025730000F4F7000042
:1032C00070B504468068428B818B521A15042D0C10
:1032D00048D0084400F121012A462030FDF702F9C8
:1032E000A068418B491E4183204604F020FA818862
:1032F000C08881420CD1A0681BA2818B4318082191
:103300002046203305F018F84FF47076C4B913E066
:10331000204600F0D5F9204600F066F9A06812A218
:10332000818B431808212046203305F005F82046FC
:10333000BDE8704000F08EB90CA13046FFF710FADE
:10334000206918B909A13046FFF70AFA154A06A103
:10335000206906F0BDFC6D1EA9B22046BDE8704094
:1033600002F016BA70BD0000257300002E2E5C2EF0
:103370002E5C2E2E5C2E2E5C2E2E5C2E2E5C636F11
:103380006D706F6E656E74735C6C69627261726988
:1033900065735C636C695C6E72665F636C692E63F7
:1033A00000000000F8F700002DE9F04104468068B5
:1033B0000F46D0F84813828B11F00106418BA1EB28
:1033C00002039DB24FF4BF730BD0994201D9002D77
:1033D0007ED0A068818B0844002180F8207066B1FF
:1033E00013E099427CD8002DF3D0831803F120011B
:1033F0002A46481CFDF776F8EBE7A068428B521C82
:1034000092B24283A068203281544DB3204604F02A
:103410008EF98188C08881420ED1A06831A2818B4B
:10342000431808212046203304F086FFA81B81B2F0
:10343000204602F0ADF921E0204600F041F9A068F5
:1034400028A2818B431808212046203304F074FF02
:10345000204600F0FFF80121204602F0ABFA0DE013
:103460003EB1A068428B521C92B24283A0682032C7
:1034700081543A461CA1206906F02AFCA168888B79
:10348000401C8883204602F070F90028204603D0B3
:10349000BDE8F04102F088B903F0D8F900281FD048
:1034A000204604F044F90546C088A988401A401E09
:1034B00081B2204602F0FAF8204602F075F9E88859
:1034C000A988401A81B2204602F080FA288800E0DC
:1034D00006E0401E81B22046BDE8F04102F06ABA23
:1034E000BDE8F081257300002563000070B50D462E
:1034F000040003D10BA1E120FFF732F9606818B98D
:1035000008A1E220FFF72CF96068006818B905A14E
:10351000E320FFF725F96068294602682046BDE8E8
:10352000704010472E2E5C2E2E5C2E2E5C2E2E5CB4
:103530002E2E5C2E2E5C636F6D706F6E656E7473D5
:103540005C6C69627261726965735C757362645CFC
:103550006170705F757362642E63000009B10620AC
:10356000704700207047000041680A6041684B6066
:103570000149086000207047BC02002070B51C00A3
:1035800015460E4603D10649A020FFF7E9F82A4662
:103590003146044808F0B4F92060002070BD0000F6
:1035A0001C0F0100001E01000020704770B51C00B8
:1035B00015460E4603D10A49AD20FFF7D1F82A4639
:1035C00031460848FEF785F838B1082805D011289B
:1035D00002D100202060002070BD2560FBE70000C4
:1035E0001C0F010028F8000070B504004FF4B275FC
:1035F00003D108A12846FFF7B3F8206918B905A13F
:103600002846FFF7ADF82069BDE870400F4A10A1C9
:1036100006F05EBB2E2E5C2E2E5C2E2E5C2E2E5CBB
:103620002E2E5C2E2E5C636F6D706F6E656E7473E4
:103630005C6C69627261726965735C636C695C6E13
:1036400072665F636C692E6300000000ECF7000097
:103650002573000070B504004FF4B87503D108A1BC
:103660002846FFF77DF8206918B905A12846FFF71D
:1036700077F82069BDE870400F4A10A106F028BB1A
:103680002E2E5C2E2E5C2E2E5C2E2E5C2E2E5C2E74
:103690002E5C636F6D706F6E656E74735C6C6962C7
:1036A0007261726965735C636C695C6E72665F639C
:1036B0006C692E6300000000E3F700002573000032
:1036C00070B504004FF4B57503D108A12846FFF783
:1036D00047F8206918B905A12846FFF741F8206985
:1036E000BDE870400F4A10A106F0F2BA2E2E5C2EF3
:1036F0002E5C2E2E5C2E2E5C2E2E5C2E2E5C636F8E
:103700006D706F6E656E74735C6C69627261726904
:1037100065735C636C695C6E72665F636C692E6373
:1037200000000000E0F70000257300002DE9F04FD5
:103730004FF000099FB005464E464C46CDF85090DC
:1037400001F03CFE284603F0B1F9A868CA464FF4E0
:10375000C07100F5D070FCF7ECFEA86800F1200104
:10376000428B00F5D070FCF7BDFEA86800F5D07064
:103770000AF0ECFBA86800F5D07000F09FFCA96887
:10378000401CC883284601F09DFF284601F0EDFF4C
:1037900010B9284602F008F8AA680C2304A912A858
:1037A000203203F01BFE0346129840B15BB170A2B9
:1037B0000221284604F0C0FD1FB0BDE8F08F284666
:1037C00001F0F2FFF8E7704970480027A1EB00080C
:1037D0000DF1100B13E008D36DA0009071A202212F
:1037E0002846049B04F0A8FDE6E700EBC7046068E8
:1037F00001685BF82900FCF7CAFE20B17F1C634812
:10380000B7EBD80FE7D9207820B168A140F6820045
:10381000FEF7A6FF4FF00008CDF870806068C7681B
:103820000FB1A9684860606809F101044FF0000910
:1038300080680390129884425CD25BF8240069A1EE
:10384000FCF7A5FED0B15BF8240067A1FCF79FFE52
:10385000A0B15BF824000BF007FCB8B10020139076
:1038600013A800905BF8243022462846039901F003
:1038700033FE02283ED013998A4439E0A868D0F874
:10388000481341F00201C0F8481333E018A84A4633
:10389000009009F101091CAB2146039801F000FBDF
:1038A000B9F1000F26D01C9820B301685BF8240002
:1038B000FCF76DFE0028BDD11C98C168A1B1BAF11A
:1038C000000F0BD0284601F0FDFE284601F04DFF09
:1038D00010B9284601F068FF45A23CE0A9F10101BA
:1038E000DDF80C802646149180684FF000090390A3
:1038F000641C9FE7BAF1000F10D0A86800F5D071E2
:10390000C28B2030FCF7EEFDA9680C23C88B4883DE
:10391000AA6804A912A8203203F060FDB8F1000FD4
:1039200012D018A800901CAB31464046149A01F002
:10393000B7FAA9681C980BEB860248601299C36815
:10394000891B284698470AE027B104AA28461299FD
:10395000B84704E032A20221284604F0EDFCA86832
:10396000D0F8481321F00201C0F8481324E7000002
:103970006E6F74207465726D696E617465643A204F
:1039800025630D0A00000000141C0100841B0100C7
:103990003A20636F6D6D616E64206E6F7420666F88
:1039A000756E6400257325730D0A00002E2E5C2EA3
:1039B0002E5C2E2E5C2E2E5C2E2E5C2E2E5C636FCB
:1039C0006D706F6E656E74735C6C69627261726942
:1039D00065735C636C695C6E72665F636C692E63B1
:1039E000000000002D6800002D2D68656C7000003F
:1039F0004572726F723A2072657175657374656491
:103A0000206D756C7469706C652066756E63746981
:103A10006F6E20657865637574696F6E730D0A004B
:103A2000506C6561736520737065636966792061A8
:103A300020737562636F6D6D616E642E0D0A0000F8
:103A40008068D0F84803C0F3C000704710B58AB052
:103A5000032401231A4600211948009404F046FE6D
:103A600018B1184AB521FCF7D5FB1549202254316D
:103A700001A8FCF737FD06200190082002900020E5
:103A80008DF818000E4801231A4601A91C30009435
:103A900004F02CFE18B10B4ABE21FCF7BBFB084812
:103AA00001231A4600213830009404F01FFE00283C
:103AB00003D0044AC221FCF7ADFB0AB010BD0000E0
:103AC00028F200009C3E00002DE9F0410446C06849
:103AD0008EB00D460026C068324601A907F090FD61
:103AE00018B100200EB0BDE8F0816DB1019807F06B
:103AF00098FAA168D1F83803401CC1F8380300F0E7
:103B00000700012879D10126204603F010FE054662
:103B10008088012804D9401E81B2204601F056FF5A
:103B20002888012804D9401E81B2204601F030FEC9
:103B30002046FFF759FD2EB131A20221204604F0A4
:103B4000FBFB5AE04FF0010800230C2202A9019868
:103B500007F076FA04980590BDF80C00ADF818004F
:103B6000BDF80E00ADF81A008DF81D8002980C27E4
:103B700000F00300012802D0022818D032E0029899
:103B80003B46860AC0F3C2008DF81C00029808A9C3
:103B9000C0F38315AA00019807F052FA206900903B
:103BA00005AB2A4608A9304607F080F91AE00298CA
:103BB000850DC0F3C2008DF81C00082D01D22E46E1
:103BC00000E008263B46324608A9019807F038FA7B
:103BD0003744AD1B05AA314608A8236907F04AF807
:103BE000002DEAD1019807F01CFAE068002201A933
:103BF000C06807F005FD0028A6D0012072E700008C
:103C00004C6F7374206C6F6773202D20696E637224
:103C100065617365206C6F67206261636B656E64BC
:103C20002071756575652073697A652E0D0A00002F
:103C30002DE9F0411E4617460D46040000D01DB97F
:103C400009A1EA20FEF78CFD606818B906A1EB20F7
:103C5000FEF786FD606833463A4601680C692946DE
:103C6000A446BDE8F04160472E2E5C2E2E5C2E2E21
:103C70005C2E2E5C2E2E5C2E2E5C636F6D706F6E34
:103C8000656E74735C6C69627261726965735C63A2
:103C90006C695C6E72665F636C692E630000000085
:103CA00070B5044640680E460025007A38B1A06819
:103CB0000068FDF72FFC08B108281AD10025BEB90D
:103CC0006068007A50B90B4A0021A068FDF7BAFB82
:103CD000616805004FF00100087209D1A068224612
:103CE00040F6CD410068FDF7F1FB0546FCF730FFDB
:103CF000284670BDBDE2000010B541680A60416809
:103D00004B60406800210172FCF722FF024901204C
:103D10000870002010BD0000C002002070B51C001B
:103D200015460E4603D106A16620FEF719FD2A4668
:103D300031460020FCF70EFF2060002070BD00001F
:103D40002E2E5C2E2E5C2E2E5C2E2E5C2E2E5C2EAD
:103D50002E5C636F6D706F6E656E74735C6C696200
:103D60007261726965735C636C695C7274745C6EB9
:103D700072665F636C695F7274742E63000000008A
:103D800080680068FDF7C6BB2DE9F05F5FEA0308B5
:103D900015460E4603D11DA17420FEF7E1FC2B4809
:103DA0000068C0070FD0DFF8A8B000244FF0050A64
:103DB000B14600BF09EB04012A460020FCF718FFBA
:103DC000060003D011E0C8F8005018E09BF800008E
:103DD00088B10A271F494FF47A4088477F1EF9D1DE
:103DE000AAF101005FEA000A0CD001218BF8001053
:103DF0003444AD1BDED1002CE5D0C8F800400020D3
:103E0000BDE8F09F00218BF80010F4E72E2E5C2E09
:103E10002E5C2E2E5C2E2E5C2E2E5C2E2E5C636F66
:103E20006D706F6E656E74735C6C696272617269DD
:103E300065735C636C695C7274745C6E72665F63FC
:103E40006C695F7274742E6300000000F0ED00E096
:103E5000C002002071F8000010B50F4804F0A4FD66
:103E600018B10EA2A321FCF7D5F90B481C3004F0C1
:103E70009BFD18B109A2A821FCF7CCF906483830FF
:103E800004F092FD002805D0BDE8104003A2AC214B
:103E9000FCF7C0B910BD000028F200002E2E5C2EE9
:103EA0002E5C2E2E5C6D61696E2E63007CB5002643
:103EB0000446019601AB012269462046FFF7B8FE91
:103EC000019800281CD09DF800007F28F2D807F048
:103ED00085FBA068417821B1012964D0022966D10F
:103EE0006AE0217E9DF80050A9420DD1408B002848
:103EF000204606D0FFF71AFC0221204600F0CAF83F
:103F00007CBD01F051FCF7E7092D1CD004DC002D2D
:103F1000D0D0082D04D11FE01B2D12D07F2D24D02E
:103F2000FCF788FA0068405D10F03E0FC2D02046D2
:103F3000FFF786FD9DF8001000B32046FFF734FA26
:103F4000B8E7012136E02046FFF77AFD0028B1D01E
:103F5000204600F0B9F8ADE72046FFF771FD0028D4
:103F6000A8D02046FFF750F9A4E72046FFF768FDE8
:103F700000289FD02046FFF7A3F99BE7A268508B4B
:103F8000B0F5BF7F96D8908B1318401C908383F8B0
:103F90002010A068818B084480F82060A068418BC5
:103FA000491C418386E79DF800105B2901D0002160
:103FB00000E0022141707DE7002141702046FFF7BB
:103FC0003FFD00289CD09DF8000041380C28B7D256
:103FD000DFE800F007090E2D064C065006060654D1
:103FE00068E7012100E00021204602F043FC61E780
:103FF000204603F09CFB054600886988884203D16F
:10400000A988EA8891429BD0698988424FF00101D2
:10401000204606D101F04AFB6989204601F0B8FB31
:1040200001E001F0C7FCA068818B491C15E0204627
:1040300003F07DFB05460088297B491C884202D19C
:10404000A988012987D001284FF00101204606D018
:1040500001F09EFBA068818B491E81832AE701F055
:10406000B5FC6989204601F0A5FCF3E7204601F084
:1040700029FB1FE7204601F04EFB1BE7A068D0F8A4
:10408000482301219143D0F8482361F30002C0F88E
:1040900048230FE78268022911700CD18268002141
:1040A00082F82010826891838268518302A20321E2
:1040B000036804F041B9704725730000002801D05F
:1040C000FCF75EBA704700002DE9F04FA5B04FF045
:1040D00000080546CDF83480CDF83080806847462A
:1040E000418BA1F27F11494289B25FEA010B71D085
:1040F000828B00F1200100F5D070FCF7F3F9A8687D
:104100000024818B084480F8A041FCF793F92090AB
:104110000168A8680C23828B0244D27F895CC0F8B6
:104120004443AA6801F001090EA91FA802F5D07244
:1041300003F054F90E98FFF7C1FF86B2A2460A9425
:1041400007941F9921B101EB0900401EB8426BD8BA
:10415000B9F1000F01D0002605E00EA850F82700A5
:10416000FFF7ACFF86B200241BA822460090641C17
:104170000AAB3946504600F093FE0A9800287CD0DE
:1041800001680EA8324650F82700FCF717FA0028FD
:10419000079802D00028E7D06FE0E0B10A980068E5
:1041A000FFF78CFF0C9980B2884200D90C90BBF1CC
:1041B000000F2BD021A8009007AB4246394650464D
:1041C00000F06EFE0A98006883190798006881194C
:1041D000002015E042E0601E0D900A980068FFF78D
:1041E0006DFF80B20C90801B58450FDA80B20CE056
:1041F00011F800C0624506D1401C0004000C10D02C
:104200001A5C002AF4D1834500D983460A98B4F198
:1042100001080790A8D267A20421284604F08CF870
:104220002BE04FF6FF70EEE700241BA8224600901B
:10423000641C0AAB3946504600F032FE4CB10A9875
:1042400000280BD00EA850F827000AF00DFFA0B9E7
:1042500007E058A20421284604F06EF825B0BDE816
:10426000F08F0A9801680EA850F82700FCF78FF924
:104270000028DAD10A98D0F808A0BAF1000F09D0C6
:104280000A9838B11F997F1CBFB201EB0900874221
:10429000FFF457AF07980028E0D00D9841464045FD
:1042A00056D19AF8000038B11BA80A46009007AB17
:1042B0003946504600F0F4FD07980068FFF7FEFE0F
:1042C000B04206D007985A4600688119284601F086
:1042D00069F920980368A868818B421892F8202019
:1042E0009A5CD20715D0408B8142B7D2284603F0A2
:1042F0001EFAA9688488888B401C8883284603F0AE
:1043000016FA8088A0421FD10121284601F052FBF5
:10431000A4E7D0F84813C90711D0D0F8481321F00A
:104320000101C0F8481320212846FFF73DF8A8688E
:10433000D0F8481341F00101C0F848138EE720215E
:104340002846FFF731F889E7284601F02DFA85E77E
:10435000002128460C9A08F0CBFF0DF16C090D9C4A
:104360000EE00AAB224639465046CDF8009000F0E8
:1043700097FD0A980C9A0168284608F0B9FF641C5A
:104380004445EED917A2032128462B6803F0D4FF39
:10439000AB6816A208212846203303F0CDFF28463B
:1043A00001F0D2FA07985A4600688119284601F0B0
:1043B000F9F853E75461622066756E6374696F6E35
:1043C0003A20636F6D6D616E647320636F756E74F8
:1043D0006572206F766572666C6F7765642E0D0A64
:1043E000000000000D0A2573000000002573000086
:1043F00070B505460C0004D107A14FF41260FEF71A
:10440000AFF9002D06D0A068D0F8481341F0200184
:10441000C0F8481370BD00002E2E5C2E2E5C2E2E90
:104420005C2E2E5C2E2E5C2E2E5C636F6D706F6E7C
:10443000656E74735C6C69627261726965735C63EA
:104440006C695C6E72665F636C692E6300000000CD
:1044500000238B540A460068194603F06DBF000024
:1044600070B5044640680D4690F8280030B1A06849
:104470000068FDF74FF808B108280CD1012685B176
:10448000606904F05BFC616800220831606904F037
:1044900011FC08B1062070BD606880F8296000201A
:1044A00070BD606890F8280048B9074A0021A068EC
:1044B000FCF7C8FF6168002881F82860F0D1204629
:1044C000BDE8704009F0D0B93DE3000070B5044686
:1044D00040680D460260606800224360606880F8B2
:1044E0002820606880F82920606820220830FBF7C7
:1044F000F9FF2C61074A2946606904F0DBFB0500DF
:1045000005D1E06807F092FC206907F08FFC28468F
:1045100070BD0000D1E500002DE9F0411C001646F9
:104520000F46054603D106A1D220FEF719F92660F1
:1045300022463946E868BDE8F04107F08DBB00002F
:104540002E2E5C2E2E5C2E2E5C2E2E5C2E2E5C2EA5
:104550002E5C636F6D706F6E656E74735C6C6962F8
:104560007261726965735C636C695C756172745CBD
:104570006E72665F636C695F756172742E630000B2
:1045800010B50446406904F0D9FBA0680068BDE896
:104590001040FCF7BFBF00002DE9FC411D0016468E
:1045A0000F46044603D11AA1E620FEF7D9F82E6083
:1045B0002A463946206907F09BFB050025D1606932
:1045C000234A0178515C19B1001D08F0A5FD02E0F5
:1045D0000C3008F097FBC0B9FF20009001236A4619
:1045E00001A9206907F0DEFB78B900980199C2B2F1
:1045F000606904F093FB0546606890F8290020B1DB
:104600001DB92069009907F0B9FB2846BDE8FC8177
:104610002E2E5C2E2E5C2E2E5C2E2E5C2E2E5C2ED4
:104620002E5C636F6D706F6E656E74735C6C696227
:104630007261726965735C636C695C756172745CEC
:104640006E72665F636C695F756172742E630000E1
:10465000800100202DE9F8431F46144688460500D6
:1046600002D0B8F1000F03D11EA1BB20FEF778F8ED
:104670006868006818B91BA1BC20FEF771F8002615
:1046800028E000BF686808EB06016B460268D2F8B4
:104690000CC02246E04718B112A1C620FEF760F810
:1046A0000098844203D20FA1C720FEF759F8009862
:1046B0000644241A70B9A868017803290AD000BFFB
:1046C000D0F848138906FBD5D0F8481321F0200113
:1046D000C0F84813002CD5D1002F01D000983860C5
:1046E000BDE8F8832E2E5C2E2E5C2E2E5C2E2E5CCA
:1046F0002E2E5C2E2E5C636F6D706F6E656E747304
:104700005C6C69627261726965735C636C695C6E32
:1047100072665F636C692E630000000070B5084C20
:10472000050009D010342168002907D008682060EE
:10473000496828468847F6E70834F4E770BD00006A
:10474000A0170020054A012120B1012805D1917050
:10475000FFF7E4BF51700020FAE77047A017002070
:104760003EB5044603F0BCFF38B103B02046BDE8B7
:1047700030400022114603F03DBE06490648CDE90F
:1047800000010346029105A20821204603F0D4FD52
:104790003EBD0000901F0100000000004170706CE1
:1047A00069636174696F6E20616464726573733AE2
:1047B00025642028307825303858292C2073697AD0
:1047C000653A2025642028307825303858290D0A8C
:1047D00000000000F8B514460E46050004D121A1E2
:1047E0004FF48770FDF7BCFFA86818B1686808B17E
:1047F000286820B91BA140F20F10FDF7B1FF012E70
:1048000003D0284603F066FF30B12846BDE8F840E3
:1048100001221B4903F0EEBD022E08D0236801B02F
:104820002846BDE8F04017A2022103F085BD1CA177
:104830006068FBF7ACFE68B11AA16068FBF7A7FEE1
:1048400040B16068009019A202212846236803F055
:1048500073FDF8BD2846BDE8F8401BA2082103F00F
:104860006BBD00002E2E5C2E2E5C2E2E5C64656DC2
:104870006F5F636C695F636D64732E63000000009B
:1048800004F2000025733A20626164207061726155
:104890006D6574657220636F756E740D0A0000009B
:1048A0002D7400002D2D74657374000025733A205B
:1048B000756E6B6E6F776E20706172616D65746579
:1048C000723A2025730D0A0044756D6D7920746568
:1048D0007374206F7074696F6E2E0D0A00000000F3
:1048E000012904D0136804A2022103F025BD09495F
:1048F000002048607047000025733A206261642000
:10490000706172616D6574657220636F756E740D90
:104910000A00000000000020012904D0136804A24E
:10492000022103F009BD0949012008707047000009
:1049300025733A2062616420706172616D657465EF
:104940007220636F756E740D0A0000000000002075
:10495000012904D0136804A2022103F0EDBC094927
:10496000002008707047000025733A2062616420BF
:10497000706172616D6574657220636F756E740D20
:104980000A0000000000002070B514460D460646DF
:10499000012902D003F09EFE30B13046BDE87040E0
:1049A0000022114603F026BD2368022D01D904A27E
:1049B00000E00AA23046BDE87040022103F0BCBC12
:1049C00025733A2062616420706172616D6574655F
:1049D0007220636F756E740D0A00000025733A2013
:1049E000706C6561736520737065636966792073A7
:1049F0007562636F6D6D616E640D0A002DE9F0479D
:104A000014460D46814603F065FE30B14846BDE8C8
:104A1000F0470022114603F0EDBC022D07D04846B6
:104A20002368BDE8F04728A2022103F085BCDFF827
:104A3000B48098F80100142801D32BA206E0606826
:104A4000FBF79EFD86B2212E02D32DA2022132E079
:104A5000002567680AE000BFFBF7ECFC0068795DA1
:104A6000405C10F0380F2BD06D1CEDB2B542F3D383
:104A7000284E002505EB451030446168FBF787FDA3
:104A800000281FD06D1CEDB2142DF3D398F801103F
:104A9000454601EB4110491C88F8011030441EA125
:104AA0006268FCF75DFB1D4B212269781948FBF712
:104AB000CBFC1BA208214846BDE8F04703F03CBCF4
:104AC0001FA2C3E72EA2C1E725733A2062616420CA
:104AD000706172616D6574657220636F756E740DBF
:104AE0000A00000000000020636F6D6D616E64209D
:104AF0006C696D697420726561636865640D0A0094
:104B0000746F6F206C6F6E6720636F6D6D616E6484
:104B10000D0A0000900500202573000071E00000E0
:104B2000636F6D6D616E642061646465642073758C
:104B3000636365737366756C6C790D0A0000000021
:104B400062616420636F6D6D616E64206E616D657E
:104B5000202D20706C6561736520757365206F6E04
:104B60006C7920616C7068616E756D6572696361E6
:104B70006C20636861726163746572730D0A000072
:104B80006475706C69636174656420636F6D6D61D9
:104B90006E640D0A000000002DE9F84314460D462E
:104BA000804603F097FD30B14046BDE8F84300224F
:104BB000114603F01FBC022D03D014A2022123686A
:104BC0001DE00025184F194E09E000BF05EB451008
:104BD00038446168FBF7DBFC70B16D1CEDB2707896
:104BE0008542F3D36068009011A2022140462368F9
:104BF00003F0A2FBBDE8F883636814A2082101B0AA
:104C00004046BDE8F04303F097BB000025733A200F
:104C100062616420706172616D6574657220636F9A
:104C2000756E740D0A000000900500200000002041
:104C300025733A20756B6E6F776E20706172616DAF
:104C4000657465723A2025730D0A000064796E61FF
:104C50006D696320636F6D6D616E643A2025730D1D
:104C60000A0000002DE9F04117460C468046012954
:104C700002D003F02FFD30B14046BDE8F0410022E4
:104C8000114603F0B7BB022C02D01BA23B6811E017
:104C90000024204E204D08E004EB44103044796895
:104CA000FBF775FC60B1641CE4B268788442F3D30E
:104CB0007B681AA24046BDE8F041022103F03CBBEC
:104CC000132C14D06878001B00EB401204EB441046
:104CD000304400F12101FBF705FC687816A2401E64
:104CE00068704046BDE8F041082103F025BB002074
:104CF00086F87302F1E7000025733A2062616420B0
:104D0000706172616D6574657220636F756E740D8C
:104D10000A00000090050020000000206469642063
:104D20006E6F742066696E6420636F6D6D616E6472
:104D30003A2025730D0A0000636F6D6D616E64206B
:104D400072656D6F766564207375636365737366F2
:104D5000756C6C790D0A0000F8B514460D460746CF
:104D600003F0B8FC30B13846BDE8F84000221146E7
:104D700003F040BB012D08D0236801B03846BDE8E0
:104D8000F04013A2022103F0D7BA184D687838B169
:104D900017A20821384603F0CFFA00241A4E13E078
:104DA0003846BDE8F84019A2042103F0C5BA00BF97
:104DB00004EB44103044009023461DA208213846DD
:104DC00003F0BAFA641CE4B268788442F0D3F8BD08
:104DD00025733A2062616420706172616D6574654B
:104DE0007220636F756E740D0A00000000000020D1
:104DF00044796E616D696320636F6D6D616E6420CF
:104E00006C6973743A0D0A0090050020506C65615E
:104E100073652061646420736F6D6520636F6D6DD1
:104E2000616E64732066697273742E0D0A0000004F
:104E30005B2533645D2025730D0A000010B5044620
:104E400003F04EFC30B120460022BDE81040114670
:104E500003F0D0BA1F21BDE8104002A20320FBF7E7
:104E6000D9B900002E2E5C2E2E5C2E2E5C2E2E5CD0
:104E70002E2E5C2E2E5C636F6D706F6E656E74737C
:104E80005C6C69627261726965735C636C695C63B6
:104E90006C695F7574696C735F636D64732E630016
:104EA0002DE9F05F1C000A9F15468846064603D18F
:104EB00021A1FF20FDF754FC27B91FA14FF48070FA
:104EC000FDF74EFC4FF00009B8F1000F0BD026B3F0
:104ED000307840B372683946284690473868E0B168
:104EE0002760BDE8F09F22492248A1EB0008B5EBFE
:104EF000D80F15D2DFF880A0002683460AE000BF55
:104F00000BEBC607786801685AF82500FBF73FFBF2
:104F100020B1761CB6EBD80FF2D301E0786808E038
:104F2000C4F80090DDE7706800EB05100168002907
:104F3000F6D02060D5E700002E2E5C2E2E5C2E2EA3
:104F40005C2E2E5C2E2E5C2E2E5C636F6D706F6E51
:104F5000656E74735C6C69627261726965735C63BF
:104F60006C695C6E72665F636C692E6300000000A2
:104F7000141C0100841B0100780300202DE9F0417E
:104F800015460F46044603F0ABFB30B12046BDE8A2
:104F9000F0410022114603F02DBA0126214C7F1E5C
:104FA0000ED0012F14D06068022F22D0002837D0F5
:104FB00020881DA106EB0040BDE8F04105F026BEAB
:104FC000606800282CD0208823A106EB0040F3E77E
:104FD0006068002824D00A2200216868FBF7FDFAE7
:104FE0000246208821A106EB0040BDE8F04105F013
:104FF00011BE002814D00A220021A868FBF7EDFAA0
:1050000007460A2200216868FBF7E7FA0246208873
:105010003B4606EB0040BDE8F0411AA105F001BE99
:10502000BDE8F08184050020746573742065727298
:105030006F72206D6573736167652077697468208E
:105040006D6F7265207468616E20332061726775C0
:105050006D656E7473000000746573742065727200
:105060006F72206D6573736167650000746573749A
:10507000206572726F72206D6573736167653A2087
:105080002564000074657374206572726F72206D00
:105090006573736167653A2025642025640000000C
:1050A0002DE9F04115460F46044603F019FB30B1D7
:1050B0002046BDE8F0410022114603F09BB90226CC
:1050C000214C7F1E0ED0012F14D06068022F22D0F9
:1050D000022837D320881DA106EB0040BDE8F0412F
:1050E00005F094BD606802282CD3208823A106EB2C
:1050F0000040F3E76068022824D30A220021686890
:10510000FBF76BFA0246208822A106EB0040BDE8BF
:10511000F04105F07FBD022814D30A220021A868BF
:10512000FBF75BFA07460A2200216868FBF755FA8D
:10513000024620883B4606EB0040BDE8F0411CA13A
:1051400005F06FBDBDE8F0818405002074657374BF
:10515000207761726E696E67206D65737361676534
:105160002077697468206D6F7265207468616E20A5
:105170003320617267756D656E7473007465737446
:10518000207761726E696E67206D65737361676504
:105190000000000074657374207761726E696E6739
:1051A000206D6573736167653A2025640000000017
:1051B00074657374207761726E696E67206D6573B4
:1051C000736167653A2025642025640010B50446A4
:1051D00003F080FA30B120460022BDE810401146AD
:1051E00003F008B9054A0721204603F0A5F8204638
:1051F000BDE8104002A2082103F09EB8ECFE0000BA
:10520000202020202020202020202020202020209E
:105210004E6F726469632053656D69636F6E647568
:1052200063746F7220202020202020202020202046
:1052300020200D0A0D0A0000F8B515460E460400A0
:1052400003D117A12520FDF78BFAA06818B160687B
:1052500008B1206818B912A12620FDF781FA012EA5
:1052600003D0204603F036FA30B12046BDE8F840BE
:105270000022114603F0BEB8022E08D02B6801B000
:105280002046BDE8F0400DA2022103F055B8686841
:10529000009011A2022120462B6803F04DF8F8BDC2
:1052A0002E2E5C2E2E5C2E2E5C64656D6F5F636C03
:1052B000695F636D64732E630000000025733A20FC
:1052C00062616420706172616D6574657220636FE4
:1052D000756E740D0A00000025733A20756E6B6EB2
:1052E0006F776E20706172616D657465723A20250A
:1052F000730D0A002DE9F04116460D4607460124BC
:1053000008E000BF56F8243007A20821384603F011
:1053100013F8641CAC42F5D33846BDE8F04103A253
:10532000082103F009B80000257320000D0A0000D1
:10533000F8B516460D460746012409E056F8240044
:105340000090234604A20821384602F0F5FF641CB1
:10535000AC42F3D3F8BD0000617267765B25645DF3
:10536000203D2025730D0A0001A2022102F0E4BFB6
:105370004E696365206A6F6B65203B290D0A00004A
:1053800010B5044603F0ACF930B120460022BDE868
:105390001040114603F02EB8BFF34F8F0548016847
:1053A000054A01F4E06111430160BFF34F8F00BF74
:1053B000FDE700000CED00E00400FA052DE9F041E6
:1053C00085680646002495F82000002811D0A046E4
:1053D000FBF730F80746006804F1200104F10104EE
:1053E000695CA4B2415CC90705D0002CF4D185F8F2
:1053F0002080BDE8F081641E2404240C0FD0688B4B
:10540000021B04F12000291805F12000521CFBF7B3
:1054100069F8B168488B001B4883B1688883B2681B
:105420003D68538BD0181F300446002102E0491C10
:1054300089B2401E0778EF5DFF07F8D18442D8D0CB
:105440005B1A203302F80380B268508B401A5083F5
:10545000B1688883CDE710B50021FCF787FA0021F9
:10546000FCF75CFA007810BD2DE9F04107461546BF
:1054700088460846FEF722FE84B2B868661CC18BD7
:105480003144B1F5C07F07D9124A0421384602F0F1
:1054900053FF0020BDE8F081294600F5D070FBF7EE
:1054A00053F8051EF6D0FEF709FE82B228192946E8
:1054B000401C521CFBF716F8224641462846FBF7D3
:1054C00011F820202855B868C18B3144C1830120D0
:1054D000E0E70000C80E01002DE9FF4F002787B06C
:1054E0009A46DDF850B006463C46B84602250DF116
:1054F00008090197DDE908013A467F1C01ABCDF8A8
:105500000090FFF7CDFC019888B101680022504659
:1055100001F028F848B90198524601683046FFF773
:10552000A3FF5FEA000802D0641C002FE2D15CB345
:10553000CBF80040B0685546514600F5D070FBF7F7
:1055400003F804462846FEF7B9FD85B2C4B1B06839
:1055500000F5D070A04206D214F8010C202802D128
:105560006D1CADB2641E2046FEF7A8FD421BB0685C
:10557000521CC18B491BC18361192046FAF7B2FF47
:10558000B8F1000F01D0002500E001250BB028463E
:10559000BDE8F08F40684968884201D80120704713
:1055A000002070472DE9F04115460F00044604D154
:1055B00023A140F28650FDF7D3F8A068418B828B7F
:1055C0008B1A29449EB2B1F5C07F37D2002D35D059
:1055D000104400F1200105F120021044721CFAF77A
:1055E00081FFA0682A46818B084439462030FAF7AB
:1055F00079FFA0682030FEF761FDA1681EA24883F4
:10560000A068818B431808212046203302F094FEC5
:10561000A068818B29448183204600F0A6F818B940
:10562000204601F013F910B1204600F0BDF8002E1D
:1056300004D02046BDE8F04100F086B9BDE8F08115
:105640002E2E5C2E2E5C2E2E5C2E2E5C2E2E5C2E94
:105650002E5C636F6D706F6E656E74735C6C6962E7
:105660007261726965735C636C695C6E72665F63BC
:105670006C692E630000000025730000EFF30580C5
:10568000C005C00D10D0103840B2002806DA00F076
:105690000F0000F1E02090F8140D03E000F1E0208D
:1056A00090F80004400970470F207047002904D08B
:1056B0000A46006901A104F00BBB70471B5B25641F
:1056C0004200000070B5054602F031F8044600883B
:1056D0006188884203D1A088E18888421AD0E18895
:1056E000A088814204D9081A81B22846FFF7DEFF5C
:1056F00020886188884205D9401A81B2284600F086
:1057000047F804E0081A81B2284600F053F9A86867
:10571000418B818370BD70B5054602F008F80446E0
:105720000188007B401C814202D1A08801281BD047
:10573000A088012804D9401E81B2284600F046F90D
:105740002088217B884206D9401A401E81B2284613
:1057500000F01EF805E0081A401C81B2284600F04F
:1057600029F9A9680020888370BD10B50446006837
:10577000FEF7A4FC0146A068828B408A1144B1FB6D
:10578000F0F200FB121008B1002010BD012010BD86
:10579000002904D00A46006901A104F099BA7047B3
:1057A0001B5B25644400000070B504004FF4BB751A
:1057B00003D108A12846FCF7D3FF206918B905A139
:1057C0002846FCF7CDFF2069BDE870400F4A10A1C4
:1057D00004F07EBA2E2E5C2E2E5C2E2E5C2E2E5CBD
:1057E0002E2E5C2E2E5C636F6D706F6E656E747303
:1057F0005C6C69627261726965735C636C695C6E32
:1058000072665F636C692E6300000000E6F70000BB
:10581000257300002DE9FC47002604468DF804603E
:1058200080684FF4C07A3546B146B046514600F51F
:10583000D070FAF77EFE4349206904F049FA2069E6
:1058400004F086FA00276B46012201A92046FEF7E4
:10585000EFF90098D8B19DF804001B2806D0A16884
:1058600091F8A0111B29EED152281FD0A26808F58B
:10587000D071505408F101001FFA80F8B8F1090FF7
:105880000AD9A168042081F8A091BDE8FC872D49C0
:105890004FF6C0100D31884700980028D3D17F1CE7
:1058A000BFB2B7F57A7FCED30D20EEE7A16808F539
:1058B000D0704A4601F80090A16891F8A1015B28D8
:1058C00003D081F8A0210B20DFE7022057466FF0BC
:1058D0002F0309E005EB850503EB4505401C6544F6
:1058E00080B2ADB2B8420AD200F5D07C11F80CC03B
:1058F000BCF13B0FEED1401C80B2B84209D30C2062
:10590000C3E700BF06EB860603EB46066644B6B265
:10591000F1E700F5D07C11F80CC0BCF1000FF1D11B
:10592000FA20FA2E01D9088100E00E81FA2D02D961
:10593000A168888101E0A0688581A06880F8A02125
:105940000020A2E704F8000070B5054601F0EFFE64
:1059500004468088E188884201D1012600E00026C3
:105960002846FFF702FF18B9284600F06FFF10B174
:105970002846FFF719FF1EB160882188401A12E0FF
:10598000E088A188401A81B2284600F01FF82088DC
:105990006188884206D9401A81B22846BDE8704025
:1059A00000F008B8081A81B22846BDE87040FFF739
:1059B000EFBE0000002904D00A46006901A104F0EE
:1059C00087B970471B5B256443000000002904D0A1
:1059D0000A46006901A104F07BB970471B5B25648E
:1059E0004100000010B50121FBF7C0FF0021FBF7CB
:1059F00095FF007810BD10B50121FBF7B7FF01211D
:105A0000FBF78CFF007810BD10B50021024801F0B3
:105A100017FF80F3100010BDF42300204FF4A07294
:105A200002EB810189B200F099BC0068D0F804054E
:105A3000704700002DE9F04715460E46040003D1DB
:105A400038492F20FCF78CFE1EB936493020FCF770
:105A500087FE1DB933493120FCF782FE6079324957
:105A6000DFF8C480DFF8C49041F82050617908F174
:105A7000040808EBC100007958B1D9F804000824E3
:105A800002284CD3B9F80000022101EB004028A104
:105A900043E035882768B5F5805F03D32DA1FD204D
:105AA000FCF75EFEC7F80855B67894F90450082E46
:105AB00003D334A14520FCF753FE002D4FEA4610D6
:105AC00006DA05F00F0101F1E02181F8140D03E081
:105AD00005F1E02585F8000494F90410012201F095
:105AE0001F0302FA03F04909890001F1E021C1F81E
:105AF0008002C1F80001617908EBC1010A71617986
:105B000048F83140D9F804000024032807D3B9F835
:105B10000000032101EB004026A105F077F82046A4
:105B2000BDE8F087E405010044020020DC04002009
:105B300052544320696E7374616E636520616C72A8
:105B40006561647920696E697469616C697A6564FC
:105B50002E0000002E2E5C2E2E5C2E2E5C2E2E5C37
:105B60002E2E5C2E2E5C6D6F64756C65735C6E7290
:105B700066785C68616C2F6E72665F7274632E6803
:105B8000000000002E2E5C2E2E5C2E2E5C2E2E5C35
:105B90002E2E5C2E2E5C696E746567726174696F5F
:105BA0006E5C6E7266785C6E7266785F676C756547
:105BB0002E6800005254433A20696E697469616C22
:105BC000697A65642E00000090F90400012100F05C
:105BD0001F0291404009800000F1E020C0F800124F
:105BE00070470A46022100F0A5BB4FF4827100F015
:105BF000B5BB000010B5040003D104496120FCF7D7
:105C0000AFFD20680121016010BD0000E405010026
:105C100010B5040003D104496720FCF7A1FD2068FA
:105C20000121416010BD0000E40501002DE9F843A9
:105C3000994616460F46050003D12E498620FCF7EB
:105C40008FFD29684FF480344FF4A070BC4000EB06
:105C5000870080B226F07F46C1F808432968C1F862
:105C60004843296800220A5008580090286800EB31
:105C70008701D1F84005C1F840652968D1F80415BD
:105C80001D4F401A20F07F404FF0040801280CD12E
:105C90007868042805D3398808EB014017A104F07F
:105CA000B5FF23494FF4046088472868C0F844438F
:105CB0002968D1F80435F01A20F07F40020201D59E
:105CC00040F07F40C9F1000290420EDD02280CDC5A
:105CD0007868042806D33988324608EB014015A1BC
:105CE00004F09FFF0D20BDE8F883C1F804430020B5
:105CF000F9E70000E4050100DC0400205254433AB7
:105D00002044656C617920696E74726F6475636597
:105D1000642064756520746F207269736B206F66F0
:105D2000207072652D666972696E672E0000000032
:105D300031F600005254433A2057696E646F77651C
:105D40006420636F6D70617265207365742074697F
:105D50006D656F757420286162735F76616C75651F
:105D60003A25642C20636F756E7465723A25642938
:105D70002E00000070B50C00054604D10AA140F2C7
:105D80007510FCF7EDFC0F48417800208D4209D2D8
:105D90000D4AE06005EB4511A06011440BA0C4E979
:105DA000001070BD206070BD2E2E5C2E2E5C2E2E3D
:105DB0005C64656D6F5F636C695F636D64732E63B4
:105DC00000000000000000209005002053686F775D
:105DD0002064796E616D696320636F6D6D616E64BF
:105DE000206E616D652E00001FB514461A4AD06101
:105DF0000020019002900390886801908888ADF897
:105E00000800086800F00302012A07D0022A15D012
:105E1000124940F27720FCF7A3FC1FBDC0F3C2007B
:105E20008DF80C000C4801AB20300090086821462A
:105E3000C0F38312800A05F039F81FBDC0F3C20019
:105E40008DF80C000868044B810D203301AA204610
:105E500004F010FF1FBD0000C80200203015010033
:105E600010B50446010600F00F00092804D306A16E
:105E70004FF42B70FCF774FC6FEA0460C10F2046EE
:105E800061F31F1010BD00002E2E5C2E2E5C2E2EF6
:105E90005C2E2E5C2E2E5C2E2E5C636F6D706F6EF2
:105EA000656E74735C647269766572735F6E726638
:105EB0005C757362645C6E72665F6472765F757344
:105EC00062642E630000000070B50546000605F010
:105ED0000F0402D5092C09D301E0092C08D307A12E
:105EE00040F29920FCF73CFC280601D5134801E05C
:105EF0001248903800EB041070BD00002E2E5C2E6E
:105F00002E5C2E2E5C2E2E5C2E2E5C2E2E5C636F55
:105F10006D706F6E656E74735C64726976657273B2
:105F20005F6E72665C757362645C6E72665F6472EB
:105F3000765F757362642E630000000044180020D1
:105F400010B50446010600F00F00092804D30349E8
:105F50004FF41F70FCF704FC204610BDE0EB00007E
:105F60002DE9FC4180461F4615460E4600240D488B
:105F700001F04DFC38B11120BDE8FC8106EB043086
:105F800005F0E8FA641CAC42F8D1064801F036FC92
:105F9000CDE90057334600220221404600F0AEF919
:105FA0000020E9E7C402002010B508F0F3FD8020CE
:105FB000FFF78AFF817B0124032902D000680028B3
:105FC00009D18020FFF74CFF8440E143BDE8104039
:105FD000014801F025BC10BDA0010020812006F081
:105FE000E7B8822006F0E4B8832006F0E1B8842008
:105FF00006F0DEB8852006F0DBB8862006F0D8B8BB
:10600000872006F0D5B8882006F024B938B508F006
:10601000C1FD0020FFF758FF817B0124032905D033
:10602000006868B1BDE8384003F079BC0020FFF794
:1060300017FF8440E143BDE838400A4801F0F0BB57
:106040000020FFF70DFF8440E143064801F0E8FB24
:1060500005480449C0680C3900904968684688477B
:1060600038BD0000A001002060F30000012006F010
:1060700033B9022006F030B9032006F02DB9042010
:1060800006F02AB9052006F027B9062006F024B943
:10609000072006F021B9000038B5082408F07AFD81
:1060A0002046FFF711FF817B032915D000680028E7
:1060B00012D12046FFF7D4FE01218140C943074891
:1060C00001F0AEFB06480549406900900C398DF897
:1060D000024049686846884738BD0000A00100209A
:1060E00060F3000070B5154804680460BFF36F8F5B
:1060F000BFF34F8FBFF36F8FBFF34F8F03F05CFA87
:1061000038B10F48016921F0011201F00111144367
:10611000016101266CB194FAA4F0B0FA80F528462A
:10612000FCF729FB06FA05F18C43294608F0CEFE60
:10613000F0E7BDE8704008F073BD00006C740240E9
:106140009401002010B5054CA078FFF789FE0146A8
:10615000A078BDE8104008F0B9BE0000940100200E
:10616000F8B51A4800681A4DC6B2A878FFF778FE4D
:10617000012404FA00F12889EA68C04380B2104380
:10618000014202D0A87808F019FE06F08000A8703D
:106190000020FFF765FE04FA00F68020FFF760FE9E
:1061A00004FA00F006430A48F1430C3001F038FBD2
:1061B0008020FFF755FE8440A86804430548AC6082
:1061C000006A0090696868468847F8BD807402409C
:1061D0009401002060F3000038B5002000900B48C7
:1061E0000068ADF802008820FFF73AFE012505FAA5
:1061F00000F40820FFF734FE054985402C438868E9
:1062000004438C6049686846884738BD2075024061
:106210009401002070470000F8B51C480568284626
:1062200006F002F9BFF36F8FBFF34F8F184E194C72
:10623000E80506D501206070706A009061686846C4
:106240008847A8054FF0000705D56770B06A009031
:10625000616868468847680516D56078002813D0BD
:1062600006F0ECF820B10CA140F2C540FCF778FA3A
:106270006770194901200860582006F0E7F8F06AB5
:106280000090616868468847F8BD000000740240CD
:1062900060F30000940100202E2E5C2E2E5C2E2E2A
:1062A0005C2E2E5C2E2E5C2E2E5C636F6D706F6EDE
:1062B000656E74735C647269766572735F6E726624
:1062C0005C757362645C6E72665F6472765F757330
:1062D00062642E630000000008750240054908B59D
:1062E00000204870887004484068009049686846FB
:1062F000884708BD9401002060F300002DE9F043B9
:1063000087B00446DDE90E8980681D4616460F46B3
:1063100000280BD018216846FAF70BF902A88DF86F
:10632000007080E86003A1686846884707B0BDE850
:10633000F083000070B516460C46050003D10649EF
:10634000B920FCF70DFA2868C0F84443002E02D0AB
:106350002868C0F8044370BDE405010038B50C4658
:10636000050003D10749CA20FCF7FAF9286801594A
:1063700029B10021015100590090012038BD0020B1
:1063800038BD0000E405010010B58168D1F848135C
:10639000C1F3400119B10022114602F02BF8BDE80B
:1063A000104004F05DBA000010B5134804F06EFA16
:1063B00018B1124AFD21F9F72DFF0221104804F00F
:1063C0006DF9012414EBE07003D10C4A2102F9F7B6
:1063D00021FF0B48032144720C3004F05FF914EBE9
:1063E000E07004D1054A40F20711F9F713FF0448A1
:1063F0000C30447210BD000008F900009C3E000003
:10640000080000203EB505468068D0F84803C0F378
:10641000400020B100221146284601F0EBFF002089
:106420000290012400906A4601A902A804F054FADF
:1064300038B1002C04D006A20221284601F07CFFCE
:106440003EBDDDE900212846FFF7CEFC0024EAE747
:10645000466C617368206C6F6720656D7074790D90
:106460000A0000007CB505468068D0F84803C0F3F8
:10647000400020B100221146284601F0BBFF14A2C3
:106480000821284601F058FF164C4FF48056230B84
:106490001B0315A208212846009601F04DFF200B92
:1064A0001D4C40421DA2216901EB0031CDE90016CF
:1064B000642041430B0B0821284601F03DFFA369EE
:1064C00002B02846BDE8704020A2082101F034BF88
:1064D000466C617368206C6F6720737461747573A8
:1064E0003A0D0A008F2F010009092D204C6F6361BE
:1064F00074696F6E2028616464726573733A20302A
:1065000078253038582C206C656E6774683A2025E1
:1065100064290D0A00000000C802002009092D208E
:1065200043757272656E742075736167653A256490
:10653000252520282564206F662025642062797433
:1065400065732075736564290D0A000009092D2003
:1065500044726F70706564206C6F67733A202564B5
:106560000D0A00004023AFF300802DE9F0471646E6
:106570000C4605005BD0ACB3B3F1010902D2032095
:10658000BDE8F087884615F8010B314600F0A3F806
:10659000C7B23F2F11D003DC3FB12A2F7DD122E0BB
:1065A0005B2F69D05C2F78D182E0F00602D520788D
:1065B0002F283ED02078A8B9E2E7207890B12F2884
:1065C00002D02E2803D06DE0B00730D46AE0700707
:1065D00068D544452BD0B00764D514F8010C2F289A
:1065E00025D05FE023E0287801E015F8010F31465F
:1065F00000F071F8C0B22A28F7D021782E2909D1ED
:10660000710707D5444512D0B10703D514F8011C12
:106610002F290CD010B12F280DD023E0B00708D5BA
:10662000F00606D42F212046F9F7A0FF08B101207B
:10663000A6E70020A4E7B00714D52F212046F9F7DC
:1066400095FF04009FD1F2E74B464246214628467B
:10665000FFF78BFF012893D12F2F01D1B007E6D48C
:10666000641C01E026F004082078314600F033F87D
:1066700010F0FF07E8D1DAE720780028D7D02F28DC
:1066800001D1B107D3D4314600F025F80146324696
:10669000284606F095FF002800E014E0C7D0411C12
:1066A00002D00546641C6EE720785B28BFD1F9E76D
:1066B000F00708D115F8010B314600F00CF810F086
:1066C000FF0700D16D1E14F8010B314600F003F8EE
:1066D000B842E8D0ABE710B5044608070AD5F9F789
:1066E000A9FE0068005DC00604D52046BDE8104044
:1066F000F9F7A4BE204610BD2DE9F05F17460E0045
:10670000814670D013B1B9B2FFF754F90024F9F7FC
:1067100091FE8246006800E0641C315D415CC9075F
:10672000FAD100253046FDF7C9FCD9F80810001B46
:106730004A8AD11B814228D306EB040805E000BF3A
:1067400018F805100A290CD06D1C8542F8D33119B0
:10675000D9F8100003F0BCFA4846BDE8F05FFFF737
:1067600023B8D9F8100003F0F3FA414600232A4673
:106770004846FDF76FFF2C444846641CFFF714F8A9
:10678000B9B24846FFF716F9E1E78B46DAF8001090
:1067900006EB040818F805000B5CDB0702D0AB46DB
:1067A0000A2804D0E819904201D26D1CF2E7D9F80A
:1067B000100003F0CDFA414600235A464846FDF743
:1067C00049FF5C44DAF8000000E0641C315D415C84
:1067D000C907FAD14846FEF7E7FFB9B24846FFF7C6
:1067E000E9F89EE7FFE7BDE8F09F000010B504461A
:1067F00014480021027862B1012A09D12278022AC4
:1068000006D1114AA3686FF30B02934200D10170C5
:1068100010BD2278012AFBD162684AB18169491C06
:10682000816160690028F3D0BDE8104004F0F9BB35
:10683000D0E904231A44C0E904210021406800F093
:10684000E7FBEEE7C80200208F2F010010B50446D9
:106850000068FDF733FC0146A068428B408A114472
:10686000B1FBF0F200FB121008B1002010BD0120B6
:1068700010BD0000FEB50026044600960196029663
:106880008068E9B3D0E9D0128A4273D0D0F83C03D3
:1068900000286FD02046FEF73EFFA068D0F8445392
:1068A000002D6AD000230A226946284604F0C8FB5E
:1068B000A168BDF808500098C1F84403A0680023FF
:1068C0000A22D0F84403694604F0BAFBA168BDF877
:1068D00008200A23D1F844032031521C04F0B0FBF5
:1068E000A168BDF808008883A168BDF80800488346
:1068F000BDF80800A84202D22046FCF775FE00E071
:106900000BE0A3682CA208212046203301F014FDDF
:106910002046FEF72AFF70BB45E0D0F8440300286C
:1069200049D02046FEF7F7FEA06800230A22D0F8DF
:106930004403694604F084FBA0680199C0F844133D
:10694000A0680029458BB9D100F5D070FDF7B6FBE2
:106950000028A06805D000F5D0712030F9F725FE99
:1069600001E080F82060A0682030FDF7A7FBADF8BB
:106970000800B5E71FE01BE0FFE72030FDF79EFBB6
:106980000504A0682D0CD0F83C13C0F84413A0688F
:1069900006D000F1200100F5D070F9F706FE8DE772
:1069A00080F8A0618AE72046FFF750FF002802D058
:1069B0002046FEF7F9FEFEBD25730000FEB50D0072
:1069C000044604D11E4940F2DD40FBF7C9FEA16830
:1069D0000026D1F83C0338B300230A22694604F0AC
:1069E0002FFB0195A06800230A22D0F83C036946DA
:1069F00004F02CFB0196A068D0F83C130091408B6A
:106A0000ADF80800A068C0F83C5300230A2269468C
:106A1000284604F01BFBA1680A2328464A8B203134
:106A2000521C04F013FBFEBDC1F83C53A068C0F833
:106A3000405300960196A068408BADF80800E4E74B
:106A4000ECE10000FEB504468068D0F84063002EFB
:106A500028D000230A226946304604F0F1FAA168E2
:106A600001980025C1F84003009501952B460A22A4
:106A700069463046029504F0E9FA304604F0B2FA6D
:106A8000A168D1F8400370B100230A22694604F0DE
:106A9000D7FA0095A06800230A22D0F8400369467F
:106AA00004F0D4FAFEBDC1F83C53FEBDFEB5044669
:106AB00080682030FDF702FB0504A0684FF0000657
:106AC0002D0CC0F8446333D0A068D0F83C03E0B18B
:106AD00000230A22694604F0B3FABDF80820AA424E
:106AE00013D1A0680A2300F5D071D0F83C03521CE2
:106AF00004F0A6FAA06800F5D0712030F9F747FD40
:106B00000028A06880F8A06112D000260B35294625
:106B1000606904F037FA0100204604D003B0BDE8F4
:106B2000F040FFF74BBFFFF78DFF761C082EEED32A
:106B3000FEBD00000149416000207047FCF80000E4
:106B40002DE9FC5F0E008346DDE90C47C6F100002D
:106B500098469246814600D40846012503E000BFCE
:106B600090FBFAF06D1C5045FADAA84500D945466D
:106B700024B1002E01DB780700D5641EB80702D5CA
:106B8000B8F1000F0AD0F80708D13CB1A54205D2F0
:106B900020215846641EFBF73BFEF6E7002E02DA82
:106BA0004E462D2102E0780703D52B215846FBF7EE
:106BB0002FFE07F0030002280BD1B8F1000F08D117
:106BC0003CB1A54205D230215846641EFBF720FE99
:106BD000F6E7CDE90047434652463146584607F0AE
:106BE000C3FEBDE8FC9F000070B50E460546006878
:106BF0004FF48E7105F065FA4FF4A271286805F024
:106C000060FA28681549C0F804132868000B44B2DC
:106C1000082E03D312A14520FBF7A2FD7007000E3A
:106C2000002C06DA04F00F0101F1E02181F8140DC7
:106C300003E004F1E02484F8000428680121000B3B
:106C400040B200F01F0291404009800000F1E020B6
:106C5000C0F88012C0F8001170BD00008000020072
:106C60002E2E5C2E2E5C2E2E5C2E2E5C2E2E5C2E5E
:106C70002E5C696E746567726174696F6E5C6E72AA
:106C800066785C6E7266785F676C75652E6800006A
:106C900070B50E46044600684FF4887105F022FA7C
:106CA0004FF49071206805F01DFA4FF4927120683E
:106CB00005F018FA4FF4A271206805F013FA206865
:106CC0001549C0F804132068000B45B2082E03D301
:106CD00012A14520FBF744FD7007000E002D06DAD7
:106CE00005F00F0101F1E02181F8140D03E005F139
:106CF000E02585F8000420680121000B40B200F077
:106D00001F0291404009800000F1E020C0F880128D
:106D1000C0F8001170BD0000100302002E2E5C2E82
:106D20002E5C2E2E5C2E2E5C2E2E5C2E2E5C696E22
:106D3000746567726174696F6E5C6E7266785C6EA2
:106D40007266785F676C75652E68000010B5024644
:106D500000201268930702D0530702D410BD5007D9
:106D600019D502F00300012807D002280BD00D49E5
:106D70004FF49170FBF7F4FC0BE0C2F383100B6847
:106D8000C01C184404E00323086803EB925210442B
:106D90000860012010BD086800EB9253C2F389100F
:106DA000401CEEE78415010002480068002800D06E
:106DB00001207047C40200200268134602E08A42A4
:106DC00004D01268002AFAD10B60016070470000FD
:106DD0001CB5012905D08168D1F84813C1F34001E1
:106DE00031B102B00022BDE81040114601F002BBF3
:106DF000536804A1CDE90013136808A2022101F031
:106E00009BFA1CBD20756E6B6E6F776E2070617281
:106E1000616D657465723A200000000025733A25A3
:106E20007325730D0A0000002DE9F74F82B0154657
:106E300002980F004FF00006C068007A009058D00A
:106E4000072248A12868F9F7B9FB78B1082247A1C1
:106E50002868F9F7B3FB002830D02B6845A20298C8
:106E600005B00221BDE8F04F01F066BA012F02D053
:106E7000022F08D008E0029805B044A2BDE8F04F08
:106E8000022101F059BA0126DFF81881002400BF61
:106E900058F824100A226868F9F790FB10B1641CB6
:106EA000052CF5D3052C06D004F0FF090224002E92
:106EB00054D0002419E03CA26B68D0E7012F4FF0BA
:106EC0000009F6D0012449E04A462146009800F026
:106ED000B8FB48B90021204603F0C6FF03463AA29A
:106EE0000221029801F028FA641C03F06BFFA04213
:106EF000EAD805B0BDE8F08F4FF0000A55F824B08D
:106F000003F060FF8046002609E00021304603F0D0
:106F1000ABFF20225946F9F751FB90B1761C46454C
:106F2000F3D3464506D155F8243030A20221029809
:106F300001F002FA4A465146009800F082FB10B177
:106F40000BE0B246EDE70021504603F08DFF03460B
:106F50001DA20221029801F0EFF9641CBC42CBD3C0
:106F6000C7E70000656E61626C650000646973616B
:106F7000626C6500556E6B6E6F776E206F70746912
:106F80006F6E3A2025730D0A0000000042616420F4
:106F9000706172616D6574657220636F756E742EB9
:106FA0000D0A000000030020556E6B6E6F776E2097
:106FB0007365766572697479206C6576656C3A20C4
:106FC00025730D0A000000004C6576656C20756E17
:106FD000617661696C61626C6520666F72206D6FAD
:106FE00064756C653A2025730D0A0000556E6B6E52
:106FF0006F776E206D6F64756C653A25730D0A00AE
:10700000C068012141727047C06800214172704719
:107010007CB50D460646214C26E040201F4A6061A3
:1070200014321F49019800F047FBE8B10198009025
:10703000D4E904131A4A1B4803F0CAF808B155B141
:107040000BE0002D1BD0D4E9040108442061019815
:1070500003F0E7FF08E0042812D0102817D01249E7
:1070600040F21710FBF77CFB002201A9304604F028
:10707000C7FA0028D1D009480C3000F0BFFB7CBD16
:10708000019803F0CEFFA069401CA061F3E70198CE
:1070900003F0C7FF01202070E6E70000C8020020CF
:1070A000C81D0020C0030020301501002DE9FF415C
:1070B0000026264800F0A8FB2448001F074600F0E1
:1070C000A3FB234C60680090A56800E00098694627
:1070D000284004EB80000C30FFF738FE0028F5D183
:1070E00001AA009901EA050304EB8303491CDB684C
:1070F00042F82030401C00910328F2D3019800F0A0
:10710000030001281AD002280ED012494FF4AF70A4
:10711000FBF726FB384600F074FB08B1009860606E
:1071200004B03046BDE8F0810198032101EB905096
:107130000099BDF80A6001EB900005E00198BDF8E8
:107140000A60C0F3831008440090E3E7F0230020B6
:10715000D81F0020841501002DE9FE4F814603F061
:1071600031FE0746D9F80C0090F80880407A20B923
:107170001FA20221484601F0DFF822A324A2082121
:10718000484601F0D9F82AA20821484601F0D4F86F
:10719000002429E001231A462146404603F01CFE44
:1071A0008246002301222146404603F015FE054693
:1071B000042801D2064600E004260121204603F0FF
:1071C00053FE0346AE4201D229A200E027A229487D
:1071D00050F8261050F82A008DE8070026A2082152
:1071E000484601F0A9F8641CBC42D3D3BDE8FE8F29
:1071F0004C6F6773206172652068616C74656421EF
:107200000D0A00006D6F64756C655F6E616D6500E1
:10721000252D343073207C2063757272656E742066
:107220007C206275696C742D696E200D0A00000067
:107230002D2D2D2D2D2D2D2D2D2D2D2D2D2D2D2D7E
:107240002D2D2D2D2D2D2D2D2D2D2D2D2D2D2D2D6E
:107250002D2D2D2D2D2D2D2D2D2D2D2D2D2D2D2D5E
:107260002D2D2D2D2D2D2D2D2D2D0D0A0000000045
:107270002A00000000030020252D343073207C20DC
:10728000252D3773207C20257325730D0A000000FF
:107290004FF4004421462F4803F042FD20B12EA2B6
:1072A00040F22111F8F7B6FF01F072FC20B12AA2DA
:1072B0004FF49371F8F7AEFF002001F089FCFAF764
:1072C000DFF820B124A24FF49571F8F7A3FF264A06
:1072D00001212648FAF7B6F820B11FA240F22D117D
:1072E000F8F798FF2148002221460068FAF7EEF8E7
:1072F00020B119A24FF49871F8F78CFFFCF7A6FBA8
:1073000007F004FEFCF7A8FDFFF74EF8184C606884
:1073100003280FD32088052505EB004015A103F0B5
:1073200075FC6068032805D320881DA105EB00408B
:1073300003F06CFC03F040FB0C48183001F0CEFA6F
:107340000A48343001F0CAFA0848503001F0C6FA51
:10735000F0E70000391400002E2E5C2E2E5C2E2E3D
:107360005C6D61696E2E630079E2000010F200002E
:1073700084050020436F6D6D616E64204C696E65FD
:1073800020496E74657266616365206578616D7011
:107390006C6520737461727465642E0D0A000000C0
:1073A000506C6561736520707265737320746865D5
:1073B00020546162206B657920746F2073656520AD
:1073C000616C6C20617661696C61626C6520636FD1
:1073D0006D6D616E64732E0D0A0000002DE9FF4F84
:1073E0004FF0000881B014468B468146C246C0F873
:1073F00000802578002D71D0F9F71CF80090006806
:10740000405DC00702D004F801AB84E0D9F8000069
:107410008300401CC9F800004BF8034015E02678B3
:10742000002E78D0B8F1000F05D1222E10D0272ED3
:107430000ED05C2E1ED0B04514D12046FCF73EFE87
:107440000246611C2046F9F74DF84FF00008E6E7C8
:107450002046FCF733FE0246611C2046F9F742F84D
:10746000B046DCE7B8F1000F50D05C2E6AD16078EE
:10747000404508D12046FCF721FE0246611C20460B
:10748000F9F730F85EE030281CD100270225605D56
:10749000A0F13001072906D86D1C41EAC701EDB201
:1074A000CFB2052DF3D3022D0CD92046FCF706FEF2
:1074B000421B61192046491E921CF9F713F804F883
:1074C000017BACE778281ED100270225605DA0F182
:1074D0003001092903D841EA07100DE021E0A0F1AD
:1074E0006101052901D8573804E0A0F141010529BF
:1074F00007D8373840EA07106D1CEDB2C7B2042D2B
:10750000E4D3022DD1D8B8F1000F1BD10098006848
:10751000805DC00716D0D9F8001004988142FFF4AE
:1075200068AFD9F800000C2804D907A140F25B40ED
:10753000FBF716F9D9F8002040464BF822A005B019
:10754000BDE8F08F641C6AE72E2E5C2E2E5C2E2E7A
:107550005C2E2E5C2E2E5C2E2E5C636F6D706F6E1B
:10756000656E74735C6C69627261726965735C6389
:107570006C695C6E72665F636C692E63000000006C
:107580002DE9F05FC7888A46191D1646B1FBF7F250
:10759000B1FBF7F507FB121999193944C91CB1FB66
:1075A000F7F104464079C9B2DDF828B0884206D226
:1075B00017499420FBF7D4F801E024686D1E002DD4
:1075C000FBD1A846A7EB0905B5421AD81CE000BFBD
:1075D000BBF1000F06D004EB09010AEB08002A46B4
:1075E000091D05E004EB09000AEB08012A46001D0D
:1075F000F8F778FF2468761B4FF00009A844B742DB
:1076000001D9354600E03D46002EE1D1BDE8F09FAE
:10761000B40F010033B581B00546002409E0002213
:107620006946284603F0ECFF18B9009803F0F9FC0E
:10763000641C02A9284604F0A7F90028EFD12046CF
:107640003EBD70B5144600230D4606461A4603F0AB
:10765000C3FB844201D9002070BD22462946304632
:1076600003F0E0FB012070BD30B5024669B103F0C4
:10767000A9FB0021084C0BE001EB410304EB830361
:1076800015685B88AB4202D11160002030BD491CF7
:107690008142F1D3052030BDD403002010B50C4643
:1076A0000021E16061600349A160012103F0DCFB7E
:1076B000206010BD2CFB00002DE9FE43002416467F
:1076C0000D460C2780460094019423463A466946AD
:1076D000029403F0B5FC009845F8040B019845F8B6
:1076E000040B029845F8040B009800F003000128F1
:1076F00003D0022806D0346017E00098C0F383104E
:10770000840004E00098800D06F0FEF804463B4635
:1077100022462946404603F093FC30680C34A042D0
:1077200003D301203460BDE8FE830020FBE770B581
:107730008468006804F10805FCF7C0FCC1B2297335
:10774000A08B6A890844B0FBF2F302FB13035B1CB5
:107750002B80A08B0844B0FBF2F35B1CAB80608BEA
:107760000844B0FBF2F35B1CEB80608B0844B0FB79
:10777000F2F102FB1101491C6980284670BD10B569
:1077800031B1B2FBF3F403FB14241CB1092010BD8A
:107790000E2010BD01600021416081608281C381A3
:1077A000084610BD70B50C460546F8F75BFD00288D
:1077B00002D021882868084470BD10B50A8849881D
:1077C0008A4203D1F8F790FD012010BD002010BDC2
:1077D00070B50C460546F8F76AFD002802D06188AE
:1077E0002868084470BD10B50A8849888A4203D1C8
:1077F000F8F754FD012010BD002010BD002100F05D
:107800000FB8002100F012B8012100F01EB80121CC
:1078100000F011B808B56A46F8F7BBFD009808BD3E
:1078200008B56A46F8F79BFD009808BD08B56A469A
:10783000F8F795FD08BD08B56A46F8F783FD08BD61
:1078400008B56A46F8F772FD08BD08B56A46F8F74C
:1078500079FD009808BD08B56A46F8F7A7FD0098BD
:1078600008BD000070B5040003D113A1FE20FAF793
:1078700077FF00252846FAF78FFE206862680168C6
:10788000914214D9491E01600D781CB919A1C2207A
:10789000FAF766FF208BE16805FB00152068217A66
:1078A0000278891A0279C9B28A4200D20171002095
:1078B000FAF7A0FE284670BD2E2E5C2E2E5C2E2ED2
:1078C0005C2E2E5C2E2E5C2E2E5C636F6D706F6EA8
:1078D000656E74735C6C69627261726965735C6217
:1078E000616C6C6F635C6E72665F62616C6C6F631F
:1078F0002E6300002E2E5C2E2E5C2E2E5C2E2E5C17
:107900002E2E5C2E2E5C636F6D706F6E656E7473C1
:107910005C6C69627261726965735C62616C6C6FE8
:10792000635C6E72665F62616C6C6F632E630000F5
:1079300070B50C46050004D110A140F22110FAF7F1
:107940000FFF24B90DA14FF49170FAF709FF002041
:10795000FAF722FE1DB91849CF20FAF701FFE868AF
:107960002A68211A288BB1FBF0F11068431C1360C0
:107970000170BDE870400020FAF73CBE2E2E5C2E50
:107980002E5C2E2E5C2E2E5C2E2E5C2E2E5C636FBB
:107990006D706F6E656E74735C6C69627261726932
:1079A00065735C62616C6C6F635C6E72665F626172
:1079B0006C6C6F632E630000F478000010B5040057
:1079C00002D0206830B901E00E2010BD17A1D920E7
:1079D000FAF7C6FE606818B914A1DA20FAF7C0FEFB
:1079E000A06818B911A1DB20FAF7BAFEE06818B94F
:1079F0000EA1DC20FAF7B4FE208B18B90BA1DD2014
:107A0000FAF7AEFE207A61682268401AC0B21160AF
:107A100004E0226811684B1C13600870401EC0B25D
:107A2000F7D221680020087110BD00002E2E5C2EB8
:107A30002E5C2E2E5C2E2E5C2E2E5C2E2E5C636F0A
:107A40006D706F6E656E74735C6C69627261726981
:107A500065735C62616C6C6F635C6E72665F6261C1
:107A60006C6C6F632E6300002DE9F04F81468068D7
:107A700089B0D0F84803C0F3400038B109B0484697
:107A8000BDE8F04F0022114600F0B4BC012907D92F
:107A900009B04846BDE8F04F24A2022100F04CBCDA
:107AA00027492848081A1C21B0FBF1F8002538E0C6
:107AB0002448C5EBC50110EB81044FF0000AB4F86F
:107AC00018B0D4E90101A1EB000604D11EA140F2D7
:107AD0001F10FAF745FE2068077924B91AA140F271
:107AE0002F10FAF73DFE2068217A0078081AC0B2FC
:107AF000642117FB01F1B1FBF6F2642110FB01F1E7
:107B0000B1FBF6F16369CDE90210CDE90462CDE97C
:107B10000676CDE900BA1B4A0821484600F00CFC65
:107B20006D1C4545C4D309B0BDE8F08F42616420A7
:107B3000617267756D656E7420636F756E74000099
:107B4000AC1D01003C1D01002E2E5C2E2E5C2E2E45
:107B50005C2E2E5C2E2E5C2E2E5C636F6D706F6E15
:107B6000656E74735C6C69627261726965735C6284
:107B7000616C6C6F635C6E72665F62616C6C6F638C
:107B80002E680000940B0100C20800F007030120DA
:107B9000895C98400840704710B5C20800F00703A0
:107BA000885C01249C402043885410BD70B5154664
:107BB0008268D2F84843C4F3400424B11A462946E7
:107BC00000F018FC06E039B1516804A20B680221EC
:107BD00000F0B2FB012070BD002070BD25733A207B
:107BE00077726F6E6720706172616D657465722067
:107BF000636F756E740D0A0070B50D46040004D1F4
:107C000022A140F65640FAF7ABFDA06818B16068B3
:107C100008B1206820B91DA140F65740FAF7A0FD31
:107C2000022D0CD1A068D0F84803C0F3400030B159
:107C30002046BDE870400022114600F0DBBB40F654
:107C40005F451CB911A12846FAF78AFD206918B9C9
:107C50000EA12846FAF784FD1A4A1BA1206902F0FA
:107C600037F84FF446651CB908A12846FAF778FDA5
:107C7000206918B905A12846FAF772FD2069BDE808
:107C80007040104A10A1093202F022B82E2E5C2E4C
:107C90002E5C2E2E5C2E2E5C2E2E5C2E2E5C636FA8
:107CA0006D706F6E656E74735C6C6962726172691F
:107CB00065735C636C695C6E72665F636C692E638E
:107CC0000000000000F800002573000070B50D46AC
:107CD000040004D113A140F66540FAF741FDA06805
:107CE00018B1606808B1206820B90EA140F666405E
:107CF000FAF736FD012D07D0022D0CD1A068D0F87F
:107D00004803C0F3400030B12046BDE87040002277
:107D1000114600F06FBB2046BDE870400FA2022163
:107D200000F00ABB2E2E5C2E2E5C2E2E5C2E2E5CBE
:107D30002E2E5C2E2E5C636F6D706F6E656E74738D
:107D40005C6C69627261726965735C636C695C6EBC
:107D500072665F636C692E6300000000506C6561A1
:107D6000736520737065636966792061207375623D
:107D7000636F6D6D616E642E0D0A00001CB50129E4
:107D800005D002290BD014D94FF0010112E002B046
:107D90004FF00002BDE81040114600F02BBB5368C5
:107DA00008A1CDE9001313680CA2022100F0C4FA67
:107DB0001CBD002102B00023BDE810401A46FFF7A9
:107DC000F5BE000020756E6B6E6F776E207061726D
:107DD000616D657465723A200000000025733A25D4
:107DE0007325730D0A00000010B50446012901D067
:107DF000012100E0002100231A46FFF7D7FE0028EA
:107E000008D1A168C1F83803E068C068BDE8104037
:107E100003F03ABD10BD00003EB50446012901D073
:107E2000012100E0002100231A46FFF7BFFE0028D1
:107E300018D1E068C06803F0FDFCC0B2642110FBFB
:107E400001F2E168C9688968B2FBF1F2D2B200922E
:107E5000CDE90101A06804A20821D0F838332046FA
:107E600000F06AFA3EBD00004C6F7374206C6F67BF
:107E7000733A2025750D0A4D6178206C6F6720716B
:107E800075657565207574696C697A6174696F6E62
:107E90003A2025752525205B25752F25755D0D0A52
:107EA000000000007CB515460E46040004D118A160
:107EB00040F68640FAF754FCA06818B1606808B133
:107EC000206820B912A140F68740FAF749FC012E3C
:107ED00003D0022E09D0012108E002B02046BDE8FF
:107EE00070400022114600F085BA002100231A4696
:107EF0002046FFF75BFE002809D1696812A0CDE992
:107F0000000117A2022120462B6800F015FA7CBD63
:107F10002E2E5C2E2E5C2E2E5C2E2E5C2E2E5C2E9B
:107F20002E5C636F6D706F6E656E74735C6C6962EE
:107F30007261726965735C636C695C6E72665F63C3
:107F40006C692E630000000020756E6B6E6F776E9B
:107F500020706172616D657465723A2000000000E6
:107F600025733A257325730D0A00000010B50446E9
:107F7000012901D0012100E0002100231A46FFF76A
:107F800015FE002806D1A068D0F8481321F004019E
:107F9000C0F8481310BD10B50446012901D00121D5
:107FA00000E0002100231A46FFF700FE002806D15A
:107FB000A068D0F8481341F00401C0F8481310BD80
:107FC0007CB514460D460646022901D9012100E080
:107FD000002100231A46FFF7E9FD002811D1022DE8
:107FE00005D03046FBF72CFD60B10BA30BE06168B8
:107FF0000AA0CDE900010FA202213046236800F05B
:108000009BF97CBD0EA302B03046BDE870400DA2C6
:10801000082100F091B900006F6E000020756E6BB2
:108020006E6F776E20706172616D657465723A2053
:108030000000000025733A257325730D0A00000027
:108040006F6666004563686F207374617475733A78
:108050002025730D0A00000010B50446012901D047
:10806000012100E0002100231A46FFF79FFD0028B0
:1080700006D1A068D0F8481321F00801C0F84813D1
:1080800010BD10B50446012901D0012100E00021F6
:1080900000231A46FFF78AFD002806D1A068D0F811
:1080A000481341F00801C0F8481310BD7FB50D46D4
:1080B000040004D123A140F6CC40FAF751FBA0689C
:1080C00018B1606808B1206820B91EA140F6CD4003
:1080D000FAF746FB012D01D0012100E00021002329
:1080E0001A462046FFF762FD002829D1A068002625
:1080F000D0F8405305B301E0082E1DD200230A2218
:1081000001A9284602F09CFFBDF80C20A1680A23B3
:10811000284601F5D071521C02F092FFA068334648
:1081200000F5D0700090029D761C14A20821204614
:1081300000F002F9002DDFD1A168002081F8A00134
:108140007FBD00002E2E5C2E2E5C2E2E5C2E2E5C13
:108150002E2E5C2E2E5C636F6D706F6E656E747369
:108160005C6C69627261726965735C636C695C6E98
:1081700072665F636C692E63000000005B253364E8
:108180005D2025730D0A00007CB515460E460400DF
:1081900004D120A140F63250FAF7E2FAA06818B1F3
:1081A000606808B1206820B91AA140F63350FAF788
:1081B000D7FA012E03D0022E18D9012117E0A168A9
:1081C000204601F11002123105F0D2FF00281FD025
:1081D000A16850201DA24882A1681820088202B020
:1081E0002046BDE87040042100F0A6B8002100231D
:1081F0001A462046FFF7DAFC002809D1696822A058
:10820000CDE9000126A2022120462B6800F094F857
:108210007CBD00002E2E5C2E2E5C2E2E5C2E2E5C45
:108220002E2E5C2E2E5C636F6D706F6E656E747398
:108230005C6C69627261726965735C636C695C6EC7
:1082400072665F636C692E63000000004E6F2072DF
:108250006573706F6E73652066726F6D20746865EC
:10826000207465726D696E616C2C20617373756D1D
:1082700065642038307832342073637265656E200F
:1082800073697A650D0A000020756E6B6E6F776EEC
:1082900020706172616D657465723A2000000000A3
:1082A00025733A257325730D0A00000070B5044646
:1082B000012901D0012100E0002100231A46FFF727
:1082C00075FC002817D140F62B551CB90AA1284689
:1082D000FAF746FA206918B907A12846FAF740FAD2
:1082E000134A14A1206901F0F3FCA16850204882D0
:1082F000A1681820088270BD2E2E5C2E2E5C2E2EBA
:108300005C2E2E5C2E2E5C2E2E5C636F6D706F6E5D
:10831000656E74735C6C69627261726965735C63CB
:108320006C695C6E72665F636C692E6300000000AE
:1083300016F80000257300000FB4F8B5044608983D
:108340000E4620B91DA140F65120FAF709FA24B9CA
:108350001AA140F65220FAF703FAA06818B1606833
:1083600008B1206820B915A140F65320FAF7F8F9B2
:1083700009A80090A068D0F84813490717D5817D57
:10838000B14214D0C58A3146204606F045FE6A4601
:108390002069089901F008FDE9B2204606F03CFE8C
:1083A000290A204606F01AFEF8BC5DF814FB6A465E
:1083B0002069089901F0F8FCF6E700002E2E5C2EEB
:1083C0002E5C2E2E5C2E2E5C2E2E5C2E2E5C636F71
:1083D0006D706F6E656E74735C6C696272617269E8
:1083E00065735C636C695C6E72665F636C692E6357
:1083F000000000002DE9F04F89B090460D460400C2
:1084000004D191A140F6D220FAF7AAF9A06818B1D8
:10841000606808B1206820B98BA140F6D320FAF734
:108420009FF99748FBF74AFE064695483338FBF715
:1084300045FE301A1FFA80F9914892A22038009028
:10844000A0680821406803682046FFF775FFA06810
:1084500040680068FBF732FE064689482038FBF783
:108460002DFE304482B2A068002340684168204657
:10847000FEF742F985A208212046FFF75DFFB8F11B
:10848000000F22D00DB300261DE000BF06EB460A08
:1084900005EB8A0BDBF80400FBF710FE074655F8E6
:1084A0002A00FBF70BFE391849450BD9DBF804000D
:1084B000FBF704FE074655F82A00FBF7FFFD38449A
:1084C0001FFA80F9761C4645E0D36D483338FBF738
:1084D000F5FD4844801C1FFA80F9694800904B461E
:1084E0006DA208212046FFF727FF09F1030087B29C
:1084F000079000233A466AA12046FEF7FDF8002DBA
:1085000051D000264DE000BF06EB460A05EB8A0B72
:1085100055F82A00DBF8043063B348B3584965A224
:108520003339CDE9001008212046FFF705FF09F196
:1085300002000090DBF80400FBF7C0FD074655F889
:108540002A00FBF7BBFD07444D483338FBF7B6FD67
:1085500039180098401A801E81B22046FDF72AFA89
:108560003A225749206901F0B3FB0098401C0AE009
:10857000009301E040B100904B4647A208212046FD
:10858000FFF7DAFE079887B2DBF8081029B100235D
:108590003A462046FEF7B0F802E02046FDF704F91F
:1085A000761C4645B0D3A06840688068002847D054
:1085B000814600200646054603AF02902A466D1C00
:1085C00002AB012148460097FCF76AFC029850B1C3
:1085D0000068FBF773FDB042F0D902980068FBF722
:1085E0006DFD86B2EAE7012D2AD036A20821204689
:1085F000FFF7A2FE0025B8462A466D1C02AB0121FA
:108600004846CDF80080FCF74BFC0298002817D0B4
:10861000B11C8FB2006800903B461FA20821204683
:10862000FFF78AFE0298FF1CBAB2416821B100230D
:108630002046FEF761F8DFE72046FDF7B5F8DBE7F7
:1086400009B0BDE8F08F00002E2E5C2E2E5C2E2E81
:108650005C2E2E5C2E2E5C2E2E5C636F6D706F6E0A
:10866000656E74735C6C69627261726965735C6378
:108670006C695C6E72665F636C692E63000000005B
:108680001CF8000025732573000000004F7074690A
:108690006F6E733A0D0A00002020252D2A733A00D0
:1086A00053686F7720636F6D6D616E642068656CD1
:1086B000702E000020202573257325730000000014
:1086C000E8340000537562636F6D6D616E64733AD8
:1086D0000D0A00008068D0F84803C0F340007047DE
:1086E0008068D0F84803C0F3400070472DE9F0419E
:1086F0001E46DDF8188015460F46040004D10DA172
:1087000040F69410FAF72CF82A463946204600F035
:108710002DF805000CD15EB14146E06801F0BEFFC6
:10872000002802DA0420BDE8F081E06801214172EE
:108730002846F8E72E2E5C2E2E5C2E2E5C2E2E5C0C
:108740002E2E5C2E2E5C636F6D706F6E656E747373
:108750005C6C69627261726965735C636C695C6EA2
:1087600072665F636C692E63000000002DE9F047BC
:1087700015460E46040004D143A140F63610F9F721
:10878000EFFFA06818B1606808B1206820B93EA169
:1087900040F63710F9F7E4FF207E0A2806D00D28AE
:1087A00004D039A140F63810F9F7DAFFE068234623
:1087B000434A4461606801680F683146B847002841
:1087C0005FD1606920B930A140F64710F9F7C8FFC2
:1087D000606902F024FC002853D1A168C1F83C0371
:1087E000A168C1F840034FF45371A068F7F7A1FEE8
:1087F000A068D0F8481341F02001C0F84813A068E1
:10880000D0F8481365F38201C0F84813A068D0F887
:10881000481341F00801C0F84813A1680120294F0E
:108820000870A168502040F663194882A16818209A
:10883000002408822448254940F6641A0D1A80460F
:1088400013E000BF18EBC40603D10FA14846F9F7A7
:1088500087FF7068006818B90BA15046F9F780FFD0
:108860007068006847F82400641CB4EBD50FE9D3A6
:10887000072D05D9E908164B04223846F7F7E4FD21
:108880000020BDE8F08700002E2E5C2E2E5C2E2EE0
:108890005C2E2E5C2E2E5C2E2E5C636F6D706F6EC8
:1088A000656E74735C6C69627261726965735C6336
:1088B0006C695C6E72665F636C692E630000000019
:1088C000F143000078030020841B0100141C010008
:1088D000B5E000000023FBF7BDBE000010B50400AA
:1088E00004D122A140F61B20F9F73AFFA06818B185
:1088F000606808B1206820B91CA140F61C20F9F777
:108900002FFFA068102100F55270FEF79EFFA068AF
:108910000078F8B101281DD002281BD12046FBF7B2
:10892000C5FA00212046FBF7CFF898B11DA203211C
:1089300020462368FFF700FD2046FBF781F848B189
:10894000A36818A2082120462033FFF7F5FC204633
:10895000FCF7FAFF206901F0FBF9A068BDE81040C0
:108960006FF0100100F55270FEF75ABF2E2E5C2EEC
:108970002E5C2E2E5C2E2E5C2E2E5C2E2E5C636FBB
:108980006D706F6E656E74735C6C69627261726932
:1089900065735C636C695C6E72665F636C692E63A1
:1089A000000000002573000070B5040004D117A179
:1089B00040F6EA10F9F7D4FEA06818B1606808B173
:1089C000206820B911A140F6EB10F9F7C9FEA068A4
:1089D0000078012801D0082070BD606801688A68AD
:1089E0000021904705000FD10821204606F014FB16
:1089F0000121204606F0F2FA12A1206901F068F97F
:108A000002212046FBF746FB284670BD2E2E5C2E29
:108A10002E5C2E2E5C2E2E5C2E2E5C2E2E5C636F1A
:108A20006D706F6E656E74735C6C69627261726991
:108A300065735C636C695C6E72665F636C692E6300
:108A4000000000000D0A0A0000F1804000680028C4
:108A500000D00120704708B500F18040002101607E
:108A60000068009008BD000010B5104C207820B9B7
:108A70000FA140F21F10F9F773FE606820B90CA136
:108A80004FF49070F9F76CFE0020F9F785FD6068EF
:108A9000401E6060606818B903F046FD00206070F9
:108AA000BDE810400020F9F7A5BD0000A017002088
:108AB0002E2E5C2E2E5C2E2E5C2E2E5C2E2E5C2EF0
:108AC0002E5C696E746567726174696F6E5C6E723C
:108AD00066785C6C65676163795C6E72665F647210
:108AE000765F636C6F636B2E6300000070B5184C8B
:108AF0000546207818B917A1FE20F9F731FE6078F5
:108B000038B115B16968002088470020F9F744FDA5
:108B10000CE00020F9F740FD25B10D48294608304A
:108B2000FEF74AF9606808B903F0CEFC6068401CA3
:108B300060600020F9F75EFD6068002806D1BDE89E
:108B4000704004A14FF48D70F9F70ABE70BD0000AB
:108B5000A01700202E2E5C2E2E5C2E2E5C2E2E5C5E
:108B60002E2E5C2E2E5C696E746567726174696F5F
:108B70006E5C6E7266785C6C65676163795C6E7260
:108B8000665F6472765F636C6F636B2E63000000D8
:108B900070B50A4C207808B185250CE00020A06053
:108BA00060602061E060064803F0F6FC054603F0D3
:108BB00059FC01202070284670BD0000A01700203D
:108BC000454700000148007870470000A0170020CA
:108BD00070B5174C0546207818B916A1C120F9F7D1
:108BE000BFFDA07838B115B1696801208847002021
:108BF000F9F7D2FC0CE00020F9F7CEFC25B10C48C7
:108C000029461030FEF7D8F8E06808B903F022FDD5
:108C1000E068401CE0600020F9F7ECFCE068002808
:108C200005D1BDE8704003A1DD20F9F799BD70BD05
:108C3000A01700202E2E5C2E2E5C2E2E5C2E2E5C7D
:108C40002E2E5C2E2E5C696E746567726174696F7E
:108C50006E5C6E7266785C6C65676163795C6E727F
:108C6000665F6472765F636C6F636B2E63000000F7
:108C700010B500B9044803F05DFD002802D1034A95
:108C80000121117010BD000050F300007C01002094
:108C900010B5044600F007F8204603F01FFE03F06D
:108CA00016FE002010BD10B503F00AFEBDE810400E
:108CB00003F01EBEF0B505460478154889B0164687
:108CC00040F82420124A08690832A2F10C0742F841
:108CD0002400487F385520226846F7F703FC0494A7
:108CE0002878385C48B10EB10A4A00E00022694693
:108CF000281D04F079F809B0F0BD0EB1064A00E075
:108D00000022694605F10C0003F06CFEF3E7000059
:108D10008401002035E80000DDE6000030B403786F
:108D2000054CE35C1BB130BC001D04F077B930BCCE
:108D30000C3003F065BF0000800100200178044A78
:108D4000515C11B1001D04F0F5B90C3003F0EABF1D
:108D50008001002003490248C1F804037047000065
:108D600004148001007002402DE9F0411D461746B1
:108D700006460C46AA4204D213A140F2C310F9F7EA
:108D8000EFFC206838B103F0A1FC20B90EA14FF42C
:108D9000E270F9F7E5FC6068A84204D20021716036
:108DA0002168316007E075602168401B31606060B8
:108DB000216829442160AF4203D110B10120BDE8F0
:108DC000F0810020FBE700002E2E5C2E2E5C2E2E64
:108DD0005C2E2E5C2E2E5C2E2E5C636F6D706F6E83
:108DE000656E74735C647269766572735F6E7266C9
:108DF0005C757362645C6E72665F6472765F7573D5
:108E000062642E630000000010B50D4C207820B97C
:108E10000CA140F2EF60F9F7A3FC00F017FE19492E
:108E2000D1F80403C1F80803174900200860BFF314
:108E30006F8FBFF34F8F05F0ADFE0120207010BD86
:108E4000940100202E2E5C2E2E5C2E2E5C2E2E5C8D
:108E50002E2E5C2E2E5C636F6D706F6E656E74735C
:108E60005C647269766572735F6E72665C7573625C
:108E7000645C6E72665F6472765F757362642E63A3
:108E80000000000000700240007502402DE9F0472C
:108E9000DFF8049199F80000012804D03FA140F2C6
:108EA0008C60F9F75DFC4FF40068404603F0BCFAB3
:108EB00000F05CFB494E4A4D49F2753450B1002038
:108EC000F9F76AFB29680320002952D0306000209E
:108ED000F9F790FB0020F9F75FFB2968404FC020AD
:108EE000143700294AD038600020F9F783FB3D4948
:108EF00001200860BFF36F8FBFF34F8F3A480168BE
:108F00000905FCD5404603F08FFA0020F9F744FB31
:108F10002868A846002580B33D600020F9F76AFB69
:108F200000F024FB50B10020F9F736FBD8F8001010
:108F3000404669B335600020F9F75CFB2B4940F2ED
:108F4000E37008604020091D0860BFF36F8FBFF316
:108F50004F8F244980201C3108604C4640F2FF109E
:108F6000C4E9020505F016FEA57002202070BDE8D8
:108F7000F0872C6030602C60A9E703E02C6038603B
:108F80002C60B1E7C8F800403D60C8F80040C4E775
:108F9000046035600460CEE7940100202E2E5C2E24
:108FA0002E5C2E2E5C2E2E5C2E2E5C2E2E5C636F85
:108FB0006D706F6E656E74735C64726976657273E2
:108FC0005F6E72665C757362645C6E72665F64721B
:108FD000765F757362642E630000000014ED064036
:108FE00000EC064000750240007402400078024028
:108FF00005F0E4BE70B5054605F0E0FE2846FCF736
:109000009FFF044600F00F00092804D30E4940F2E8
:10901000B640F9F7A5FB04F00F0122064FF001005E
:1090200001D50A4A01E0094A121D136888408343AA
:109030001360BFF36F8FBFF34F8F284600F0BAF96C
:109040000349C1F8080370BD309C00001075024050
:109050000070024070B5010600F00F050446092DAE
:1090600004D30C4940F28240F9F77AFB082D04D36F
:10907000084940F28340F9F773FB07480460BFF3E7
:109080004F8F44F480710160BFF36F8FBFF34F8F38
:1090900070BD0000309C00000C75024070B50546A4
:1090A00000F088F92149C1F80403284603F048F884
:1090B00000283AD12846FCF743FF044600F00F0091
:1090C000092804D31A4940F2A540F9F749FB04F0F6
:1090D0000F0021064FF0010401D5164901E01549A2
:1090E000091D0A6804FA00F002430A60BFF36F8F9B
:1090F000BFF34F8F280718D0280616D405F00F00AD
:10910000082812D20020F9F747FA284600F024FD7B
:109110002846FCF7A5FE84400748C168A143C1600A
:10912000BDE870400020F9F765BA70BD00700240DC
:10913000309C0000107502409401002010B5FCF72F
:10914000FFFEBDE8104002F0FBBF00002DE9F0413A
:109150000E460746FCF784FE054626B918A140F6E0
:109160005600F9F7FDFA0020F9F716FA244C3807F3
:1091700004D1A078874201D010241BE02089E16847
:10918000C04380B20843012101FA05F5284201D00D
:1091900011240FE03846FCF797FE00218160326809
:1091A0000260726842608173E0680543E5600C46C6
:1091B00005F0D8FE0020F9F71DFA2046BDE8F08141
:1091C0002E2E5C2E2E5C2E2E5C2E2E5C2E2E5C2ED9
:1091D0002E5C636F6D706F6E656E74735C64726924
:1091E000766572735F6E72665C757362645C6E72D4
:1091F000665F6472765F757362642E6300000000C0
:109200009401002010B5FCF75FFE808910BD0000BE
:1092100070B50C00054602D0601E044204D011A1B6
:1092200040F29B70F9F79CFA05F00F0008280CD368
:109230001C480068C1B2802904D04FF48060A0426D
:109240000AD204E04FF40070F9E7402C04D905A1DC
:1092500040F29D70F9F784FA2846FCF735FE8481C8
:1092600070BD00002E2E5C2E2E5C2E2E5C2E2E5CF1
:109270002E2E5C2E2E5C636F6D706F6E656E747338
:109280005C647269766572735F6E72665C75736238
:10929000645C6E72665F6472765F757362642E637F
:1092A000000000001C75024010B5FCF749FE0446A2
:1092B00000F00F00082804D3064940F2CF40F9F728
:1092C0004FFA054944F480700860BFF36F8FBFF315
:1092D0004F8F10BD309C00001875024010B5FCF790
:1092E0002FFE00F00F01082901D3002010BD020657
:1092F000054800EB810002D5D0F8200401E0D0F849
:1093000044040128F1D110BD0070024010B5FCF7F3
:1093100017FE044600F00F00082804D3054940F268
:10932000D740F9F71DFA04480460BFF36F8FBFF30D
:109330004F8F10BD309C00001875024070B5044678
:10934000000604F00F0502D5092D09D301E0092D0F
:1093500008D307A140F26310F9F702FA200601D5FD
:10936000134801E01248123030F8150070BD0000BB
:109370002E2E5C2E2E5C2E2E5C2E2E5C2E2E5C2E27
:109380002E5C636F6D706F6E656E74735C64726972
:10939000766572735F6E72665C757362645C6E7222
:1093A000665F6472765F757362642E63000000000E
:1093B0000CF4000070B50546000605F00F0402D558
:1093C000092C09D301E0092C08D307A14FF4C6707A
:1093D000F9F7C6F9280601D5134801E0124809300B
:1093E000015D0120884070BD2E2E5C2E2E5C2E2E3D
:1093F0005C2E2E5C2E2E5C2E2E5C636F6D706F6E5D
:10940000656E74735C647269766572735F6E7266A2
:109410005C757362645C6E72665F6472765F7573AE
:1094200062642E630000000030F400002DE9F0417A
:109430000D460646FCF714FD044625B930A140F25E
:10944000E770F9F78DF90020F9F7A6F83C483107E5
:1094500004D181788E4201D0102438E00189804601
:10946000C943C06889B201270143A740394201D0EE
:1094700011242CE03046FCF727FD044606F00F00CF
:10948000310600EB40002AD52E4901EB8006286802
:1094900003F01CF90028287A4FEAC07004D008B104
:1094A000294803E0294801E0B8B12948206095E83F
:1094B000070086E807000020C4E90160A073D8F81F
:1094C0000C1004460F43C8F80C7005F04BFD00204B
:1094D000F9F790F82046BDE8F0811E48E6E7194903
:1094E0006C3101EB8006286838B103F0EFF820B941
:1094F00003A14FF40460F9F733F91748D6E70000E9
:109500002E2E5C2E2E5C2E2E5C2E2E5C2E2E5C2E95
:109510002E5C636F6D706F6E656E74735C647269E0
:10952000766572735F6E72665C757362645C6E7290
:10953000665F6472765F757362642E63000000007C
:1095400094010020D4180020B9970000359700003E
:109550008D960000ED950000698D000010B5FCF7B8
:10956000EFFCBDE8104002F01FBF000010B500F096
:1095700013F858B107480078C0F30310012805D14B
:109580000448001D007810F0F00F01D0002010BD3D
:10959000012010BDE80F00F006480078082804D12B
:1095A0000448001D0078000701D00020704701200A
:1095B00070470000E00F00F010B5FFF7EDFF50B16D
:1095C0000748007810F0F00F05D10548001D00781D
:1095D00010F0F00F01D0002010BD012010BD0000E0
:1095E000E80F00F000487047AC1900202DE9F04169
:1095F000804616460C46086803F068F820B112A1B0
:109600004FF40B70F9F7ACF865681F4FB54200D9FD
:109610003546402D04D90CA140F23620F9F7A0F8C8
:109620002A4638462168F6F75DFFC8E9007560688C
:10963000401B60602068284420606068002800D0DB
:109640000120BDE8F08100002E2E5C2E2E5C2E2E17
:109650005C2E2E5C2E2E5C2E2E5C636F6D706F6EFA
:10966000656E74735C647269766572735F6E726640
:109670005C757362645C6E72665F6472765F75734C
:1096800062642E6300000000AC1900202DE9F04157
:10969000064690460D46086803F018F820B114A15C
:1096A00040F25220F9F75CF86C68214F404644457F
:1096B00000D90446402C04D90DA14FF41770F9F7D6
:1096C0004FF834B1224638462968F6F70BFF376069
:1096D00001E00020306074606868001B68602868E2
:1096E0002044286014B10120BDE8F0810020FBE790
:1096F0002E2E5C2E2E5C2E2E5C2E2E5C2E2E5C2EA4
:109700002E5C636F6D706F6E656E74735C647269EE
:10971000766572735F6E72665C757362645C6E729E
:10972000665F6472765F757362642E63000000008A
:10973000AC1900202DE9F041074616460C46086892
:1097400002F0C4FF20B90CA14FF4F570F9F708F846
:109750006568B54200D935462068C7E900056068EC
:10976000401B60602068284420606068002800D0AA
:109770000120BDE8F08100002E2E5C2E2E5C2E2EE6
:109780005C2E2E5C2E2E5C2E2E5C636F6D706F6EC9
:10979000656E74735C647269766572735F6E72660F
:1097A0005C757362645C6E72665F6472765F75731B
:1097B00062642E63000000002DE9F0410746164662
:1097C0000C46086802F082FF20B910A140F20B207D
:1097D000F8F7C6FF6568B54200D93546002D0FD0B1
:1097E000D4F80000C7E900056068A0EB05006060E0
:1097F00020682844206006D04FF00100BDE8F081C9
:109800004FF00000EEE74FF00000F7E72E2E5C2E41
:109810002E5C2E2E5C2E2E5C2E2E5C2E2E5C636F0C
:109820006D706F6E656E74735C6472697665727369
:109830005F6E72665C757362645C6E72665F6472A2
:10984000765F757362642E63000000002DE9F041BD
:1098500028B11E490A7822B10820BDE8F08107200E
:10986000FBE7486001200024087046024FEA040527
:1098700044F0800707F00F00082801D3314600E0CC
:1098800040213846FFF7C4FC3846FCF71DFB8573C2
:10989000641C0560E4B28560092CE9D35FF0000424
:1098A00004F00F00082801D3314600E04021204693
:1098B000FFF7AEFC2046FCF707FB8573641C0560D0
:1098C000E4B28560092CEBD30020C6E794010020A8
:1098D00003480078022801D3012070470020704718
:1098E0009401002002480078002800D00120704731
:1098F0009401002010B5FFF7EBFF28B12720F7F700
:10990000CDFB08B1012010BD002010BD01488078BA
:109910007047000094010020502002F097BD10B560
:10992000FFF74AFE58B1EFF3108472B64C2002F0F4
:109930008DFD4C2002F08AFD84F3108810BDBDE837
:1099400010404C2002F082BD0021016041601149AD
:10995000096801700F49091D096841700D490831F6
:1099600009680C4A0C32126841EA02214180094917
:1099700010310968074A1432126841EA02218180D5
:10998000044918310968034A1C32126841EA02216D
:10999000C180704780740240542002F057BD00001F
:1099A00070B5144C05462078022804D012A140F26C
:1099B000FD60F8F7D5FE002060701F4C15B9FFF769
:1099C000FBFD00B11D4C1E48C0F804431D49E020BA
:1099D00081F800041B49012280202339C1F880024C
:1099E000C1F8000118480260BFF36F8FBFF34F8FBB
:1099F00070BD0000940100202E2E5C2E2E5C2E2EB9
:109A00005C2E2E5C2E2E5C2E2E5C636F6D706F6E46
:109A1000656E74735C647269766572735F6E72668C
:109A20005C757362645C6E72665F6472765F757398
:109A300062642E63000000000714C0010714E001F7
:109A40000070024027E000E004750240104810B5A5
:109A50000078022804D00FA140F21C70F8F780FEB5
:109A60002720F7F71BFB002810D005F009FA194949
:109A700000200860BFF36F8FBFF34F8F164980201F
:109A8000C1F8800148171549C1F8080310BD00004E
:109A9000940100202E2E5C2E2E5C2E2E5C2E2E5C31
:109AA0002E2E5C2E2E5C636F6D706F6E656E747300
:109AB0005C647269766572735F6E72665C75736200
:109AC000645C6E72665F6472765F757362642E6347
:109AD000000000000475024004E000E00070024055
:109AE00010B500242046F8F757FD12484078B0B171
:109AF00005F0C6F910480168890510D40F49012204
:109B00000A60006882054FF0000001D5086006E099
:109B10000B4901240B680A4A14322BB11060002053
:109B2000F8F768FD204610BD49F275330B601060F0
:109B30000B60F4E794010020007402402C75024091
:109B400000EC064003490248C1F8080370470000D2
:109B500004148001007002402DE9F0410446000623
:109B600004D521A14FF40E60F8F7FAFDFFF724FDAC
:109B700001274FF000082C4D002804F00F06404646
:109B800012D0F8F709FD2046FCF76AF98740A8686B
:109B90002649B843A86040F2C57000EB4600086053
:109BA000091DC1F800801AE0F8F7F6FC2046FCF722
:109BB00057F98740A868B843A860082E0FD220063E
:109BC00004D51BA140F26240F8F7CAFD244A02EB1B
:109BD0008601C1F8A084BFF36F8FBFF34F8FBDE83C
:109BE000F0410020F8F706BD2E2E5C2E2E5C2E2EA6
:109BF0005C2E2E5C2E2E5C2E2E5C636F6D706F6E55
:109C0000656E74735C647269766572735F6E72669A
:109C10005C757362645C6E72665F6472765F7573A6
:109C200062642E630000000094010020007802406E
:109C30002E2E5C2E2E5C2E2E5C2E2E5C2E2E5C2E5E
:109C40002E5C6D6F64756C65735C6E7266785C68B3
:109C5000616C5C6E72665F757362642E68000000F2
:109C60000070024005480178012901D008207047A2
:109C700000214160017008467047000094010020F7
:109C800010B500242046F8F787FC0E48407868B1EC
:109C900002F0D4FB50B10C49002008600B490124AC
:109CA0000B680A4AC02014322BB110600020F8F76C
:109CB000A1FC204610BD49F275330B6010600B60AB
:109CC000F4E70000940100202C75024000EC0640EF
:109CD0000FB438B5040003D110A11C20F8F740FDE3
:109CE000606918B90DA11D20F8F73AFD206818B970
:109CF0000AA11E20F8F734FD606818B907A11F20DB
:109D0000F8F72EFD0599002905D006A800906A46AF
:109D1000204600F049F838BC5DF814FB2E2E5C2E6E
:109D20002E5C2E2E5C2E2E5C2E2E5C2E2E5C6578EC
:109D30007465726E616C5C667072696E74665C6E7E
:109D400072665F667072696E74662E630000000052
:109D500010B5040003D107A10B20F8F701FDA2689C
:109D6000002A05D0D4E90403216898470020A060A8
:109D700010BD00002E2E5C2E2E5C2E2E5C2E2E5C36
:109D80002E2E5C2E2E5C65787465726E616C5C663E
:109D90007072696E74665C6E72665F667072696E10
:109DA00074662E63000000002DE9FC4791460C46C6
:109DB0005FEA000804D183A14FF49F70F8F7D0FC4C
:109DC000D8F8140020B97FA14FF4A070F8F7C8FCB0
:109DD000D8F8000020B97BA140F24110F8F7C0FC90
:109DE000D8F8040020B977A14FF4A170F8F7B8FCB7
:109DF000002C76D014F8011B39B125290ED040462D
:109E0000F8F706FD20780028F4D198F80C00002817
:109E100067D04046BDE8FC47FFF79ABF002001220B
:109E200021782B291BD02D2902D0302908D102E01E
:109E300040F0010001E040F00200641C002AEFD174
:109E400000252A290ED02178A1F130020A2A11D248
:109E500005EB850201EB4205641C303DF1E740F063
:109E60000400EAE7D9F800100B1DC9F800300968B2
:109E7000641C0D44217800232E290BD114F8011FF6
:109E8000A1F130020A2A05D203EB830201EB42035F
:109E9000303BF3E76C290DD068290BD0692921D01C
:109EA0000BDC252918D0582931D063290ED064291C
:109EB00015D117E014F8011FECE7702969D0732958
:109EC00032D075291BD0782909D120E0D9F80000BB
:109ED000011DC9F8001001784046F8F799FC641C90
:109EE00090E76CE0D9F800100A1DC9F80020096855
:109EF000CDE900500A224046FCF722FEEFE7D9F8F0
:109F000000100A1DC9F8002009680A2206E0D9F8E5
:109F100000100A1DC9F8002009681022CDE9005080
:109F2000404604F021FDDAE7D9F8001000270A1DA9
:109F3000C9F800200E68C00705D112E04046761C23
:109F40007F1CF8F765FC31780029F7D104E0202167
:109F500040466D1EF8F75CFCBD42C0D9002DF6D11D
:109F6000BDE74EB13046F6F70BFB074604E0202173
:109F700040466D1EF8F74CFCBD4206D9002DF6D1C7
:109F800003E04046761CF8F743FC31780029F8D10D
:109F9000A5E7D9F80000011DC9F8001005683021B7
:109FA0004046F8F735FC78214046F8F731FC0820A8
:109FB0000021CDE90001034610222946B0E7BDE8A3
:109FC000FC8700002E2E5C2E2E5C2E2E5C2E2E5C2E
:109FD0002E2E5C2E2E5C65787465726E616C5C66EC
:109FE0007072696E74665C6E72665F667072696EBE
:109FF00074665F666F726D61742E63002DE9F84FB1
:10A000002E4D0400894628884FF0010C69689A4655
:10A0100016460CEB004025D02268002A2DD0002ED9
:10A0200035D062684FF010071268531E13EA090F0B
:10A0300012D1E046724349462046F7F72EF9002830
:10A040002FD0206853463246056901B04946204664
:10A05000AC46BDE8F04F604700292DD0184B19A23F
:10A06000009726E031B10E210091154B1FA221A1CE
:10A0700000F0DFFD0E20BDE8F88F31B1082100911E
:10A080000F4B27A21BA100F0D4FD0820F3E731B14C
:10A09000092100910A4B25A216A100F0CAFD092052
:10A0A000E9E7686840B100972988054B204A08EB2A
:10A0B000014010A100F0BDFD1020DCE73C050020B0
:10A0C000E7F80000616464725F69735F70616765DF
:10A0D0005F616C69676E656428705F66732C2070C1
:10A0E0006167655F6164647229000000705F667378
:10A0F00000000000257320636865636B206661695A
:10A100006C656420696E202573282920776974683E
:10A110002076616C756520307825782E000000006F
:10A12000705F66732D3E705F617069006C656E00D4
:10A13000640F0100F8B5030010484FF001064FF01E
:10A140000E054468008806EB004009D069B119602B
:10A150000C6801B0A446BDE8F040114618466047BF
:10A1600054B1074B07A2009503E02CB1044B07A2A2
:10A17000009508A100F05DFD0E20F8BD3C05002013
:10A180009CF80000705F667300000000705F6170F3
:10A1900069000000257320636865636B2066616950
:10A1A0006C656420696E202573282920776974689E
:10A1B0002076616C756520307825782E00000000CF
:10A1C00018B102680AB152691047002070470000B8
:10A1D0002DE9F84F414C05008B46208891464FF001
:10A1E0000106DDF828A0616898464FF00E0206EBE4
:10A1F00000401BD0B9F1000F1DD02A68002A23D0DF
:10A200000922B8F1000F29D06B685F68B8FBF7FC32
:10A2100007FB1C83002B27D029B1314B009231A2C0
:10A220003BA100F006FD0920BDE8F88F51B1009276
:10A230002B4B42A203E029B1294B009241A234A149
:10A2400000F0F7FC0E20EFE731B108210091244B1C
:10A250003EA22FA100F0EDFC0820E5E70029E2D0A6
:10A2600000921F4B3CA2DBE75846F7F710F8102787
:10A2700098B14846F7F70BF8C8B142465946284608
:10A28000F7F70BF8F8B1CDF800A0286843464A4626
:10A29000C46859462846A047C6E7606800281BD016
:10A2A000009720880E4B06EB00402CA207E0606868
:10A2B00090B1009720880A4B06EB00402DA214A114
:10A2C00000F0B7FC08E0606830B100972088044BCC
:10A2D00006EB004030A2F2E71020A5E73C05002085
:10A2E000D4F8000021286C656E202520705F66730D
:10A2F0002D3E705F666C6173685F696E666F2D3EA0
:10A3000070726F6772616D5F756E6974290000000D
:10A31000257320636865636B206661696C656420E2
:10A32000696E202573282920776974682076616C0E
:10A33000756520307825782E00000000705F667308
:10A3400000000000705F737263000000705F66734E
:10A350002D3E705F617069006C656E0061646472AF
:10A360005F69735F616C69676E6564333228646529
:10A3700073742900616464725F69735F616C6967FB
:10A380006E65643332282875696E7433325F7429C0
:10A39000705F737263290000616464725F69735F48
:10A3A00077697468696E5F626F756E647328705F39
:10A3B00066732C20646573742C206C656E29000014
:10A3C0002DE9FF411C46DDE90A7815460E46684630
:10A3D00000F0A8F846EA450141EA840141EA072273
:10A3E00042EA0841009A00EB8200C0F80017BDE87D
:10A3F000FF812DE9FF411C46DDE90A7815460E462E
:10A40000684600F0BFF846EA450141EA840141EAA6
:10A41000072242EA0841009A00EB8200C0F80017C8
:10A42000BDE8FF811CB5002100910B46012201917E
:10A43000FFF7C6FF1CBD1CB5002100910B46012291
:10A440000191FFF7D6FF1CBD1CB500220B46009200
:10A4500011460192FFF7B4FF1CBD1CB500220B464C
:10A46000009211460192FFF7C4FF1CBD1CB50021EC
:10A4700000910B46012201911146FFF7A1FF1CBD7F
:10A480001CB5002100910B46012201911146FFF7F6
:10A49000B0FF1CBD13B50C46684600F013F80099D8
:10A4A00000EB8101D1F8002722F44032C1F80027E7
:10A4B000009900EB8100D0F8001741EA0441C0F890
:10A4C00000171CBD10B504460068302804D308A14D
:10A4D00040F2A110F8F744F92068202802D24FF08A
:10A4E000A04010BD00F01F0020600D4810BD00000E
:10A4F0002E2E5C2E2E5C2E2E5C2E2E5C2E2E5C2E96
:10A500002E5C6D6F64756C65735C6E7266785C68EA
:10A51000616C2F6E72665F6770696F2E6800000055
:10A520000003005010B504460068302804D308A189
:10A5300040F2A110F8F714F92068202802D24FF059
:10A54000A04010BD00F01F0020600D4810BD0000AD
:10A550002E2E5C2E2E5C2E2E5C2E2E5C2E2E5C2E35
:10A560002E5C6D6F64756C65735C6E7266785C688A
:10A57000616C2F6E72665F6770696F2E68000000F5
:10A580000003005010B504460068302804D308A129
:10A5900040F2A110F8F7E4F82068202802D24FF02A
:10A5A000A04010BD00F01F0020600D4810BD00004D
:10A5B0002E2E5C2E2E5C2E2E5C2E2E5C2E2E5C2ED5
:10A5C0002E5C6D6F64756C65735C6E7266785C682A
:10A5D000616C2F6E72665F6770696F2E6800000095
:10A5E0000003005001B56846FFF79CFF009A012167
:10A5F0009140C0F8081508BD01B56846FFF7C2FFD5
:10A60000009A01219140C0F8081508BD7CB5154697
:10A6100004460C4A6618022ED2E90002CDE9000277
:10A6200004D909A140F2B920F8F79AF8694605E083
:10A6300051F82400D0F81005641C01C5A642F7D8D3
:10A640007CBD000044F400002E2E5C2E2E5C2E2ECD
:10A650005C2E2E5C2E2E5C2E2E5C6D6F64756C65F0
:10A66000735C6E7266785C68616C2F6E72665F6791
:10A6700070696F2E68000000034908B50844002186
:10A6800001600068009008BD006000400249405829
:10A69000012800D000207047006000402DE9F04103
:10A6A0000E461C4904460025D1F81024104609E046
:10A6B000037AAB4205D16D1C0A2DF7DB4FF0FF3555
:10A6C00025E040680028F3D1681C20D02572D1F81D
:10A6D000100440B140686060D1F810044460002765
:10A6E000DFF834800FE00020C1F810446060F6E726
:10A6F00008EBC700C279B24200D33246207A39460D
:10A7000000F090FB7F1C00F05DFBB842F0D82846BB
:10A71000BDE8F081D81F0020141C010038B5446941
:10A72000C0680022694600F06BFF002803D10021B9
:10A730002046F9F7C9F938BD10B544696068016869
:10A740008A680121904718B10420A168087010BDE3
:10A750000320FAE72DE9F34146690446B068007822
:10A7600004281ED0032807D0002501A9E06801F0C5
:10A770000BF985F0010709E00125F6E73946304677
:10A78000F9F7A2F901A9E06801F0FEF80028F5D177
:10A79000019800F040FC002D03D000213046F9F76D
:10A7A00093F9BDE8FC8100000148806802F070BEAA
:10A7B000C802002038B5002216491748FFF7BAFC36
:10A7C000164C012108B1217038BD022020701448B8
:10A7D0000025C0F8801101216068FCF719FC1149BF
:10A7E000486A0A8DCB6A61F39F200F49086090B2D6
:10A7F000C1E901030A4600950C2307482169FFF7C8
:10A80000E7FC20690C302061A068BDE838400121D8
:10A81000FCF7FEBB08F90000C0030020C8020020BE
:10A8200004E000E08CFA0000C81D002070B50B4C5D
:10A830000D46207801280FD0084600F0ECFB294691
:10A84000A068FCF7E7FE2078022805D1A068BDE8E3
:10A8500070400121FCF7DCBB70BD0000C802002085
:10A8600070B5074D01200023287006480122010B16
:10A8700009030C460448FFF7C1FB2C6170BD0000C2
:10A88000C80200208F2F0100C00300203EB50F49F1
:10A890000B0B0F491B0303F6FF72C1E9033201469C
:10A8A00000220B48FFF746FC04000DD1002500955F
:10A8B00002AA01A9684600F00FF80028F8D0054860
:10A8C00000990161057020463EBD00008F2F0100F8
:10A8D000C0030020C802002070B50D46016816466E
:10A8E000044611B91248010B090312482160FFF711
:10A8F00067FC68B1206828600C3030602868006808
:10A9000000F00301012905D0022907D0052070BD00
:10A91000062070BDC0F38310800002E0800D02F0BD
:10A92000F3FF21680C3008442060002070BD000057
:10A930008F2F0100C00300200148406802F0A8BD2D
:10A94000C80200207047000070B50E4C0D462078FC
:10A95000002815D1084600F05EFB29466068FCF728
:10A9600059FEA1690844A06104F10C00FCF74FFFF7
:10A97000002805D16068BDE870400021FCF748BBA5
:10A9800070BD0000C80200200A4A012902EBC00085
:10A9900007D0022907D0032907D0042907D00020B7
:10A9A0007047022070470420704700797047407953
:10A9B00070470000141C01002DE9FF5FF7F738FF16
:10A9C00018B1002004B0BDE8F09F874C0020C4F807
:10A9D0001804BFF34F8F60680090A6684FF000091D
:10A9E000304004EB800008E021680098814201D8E3
:10A9F0006160E6E7304004EB80000C306946FCF70C
:10AA0000A5F90028F0D101AAA046009901EA0604A0
:10AA100008EB8403491CDB6842F82030401C00919D
:10AA20000328F2D3019800F00300022802D0012885
:10AA300050D0BEE00198A022810D8A46B2EB905F13
:10AA400000D8A0210C4664F39F50C0F3C2070190C8
:10AA50000C31664800F096FA0500EAD000F0DBFA07
:10AA60004B460C2201A9284600F0F0FA009909F1A2
:10AA70000C0B3140701A8000001D844223D95A4EBD
:10AA80000C3630B1C2B208EB8101201A91460C316C
:10AA900004E03146E2B2002691463046C4B25B463D
:10AAA000284600F0D3FA0BEB09032EB122463146BB
:10AAB0004FEA050000F0CAFA00990AF1030001EB21
:10AAC000900000903DE008EB81015B46224628465D
:10AAD0000C31EFE70198C0F38310062800D306205D
:10AAE000019960F38911C1F38310C1F3C207C01C3F
:10AAF000019181003D4800F045FA050059D000F071
:10AB00008AFA4B460C2201A9284600F09FFA09F167
:10AB10000C0900240FE000984B460246304008EB39
:10AB20008001501C0090042228460C3100F08EFA5F
:10AB300009F10409641C0198C0F38310A042EAD80B
:10AB4000B5B3D8F81044D8F818044646F8B12846EA
:10AB500000F067FA42E0607A012817D1BDF80800DA
:10AB6000234A00EB400002EB8000217A806801EB71
:10AB70004101C84000F00700052F00D10327B8426B
:10AB800004D3226820462946126890476468002C46
:10AB9000E1D1284600F045FA0020F7F7FDFCD6F891
:10ABA000180408B9009870600020F7F723FD15E03D
:10ABB000FFE7D8F8104404E02168204689688847F8
:10ABC0006468002CF8D10B484168022906D300883C
:10ABD000022101EB004008A100F018F8F7F728FE69
:10ABE00080F00100EEE60000D81F0020901D01005B
:10ABF000D4030020840500204261636B656E64739A
:10AC000020666C75736865640000000000231A46B6
:10AC100003F0CEB908B5012300926A4603F0C8F9E3
:10AC200008BD1CB5CDE9002302236A4603F0C0F934
:10AC30001CBD3EB5069C8DE81C0003236A4603F04C
:10AC4000B7F93EBD7FB5DDE908458DE83C0004233A
:10AC50006A4603F0ADF97FBD70B586B00DF1280CE2
:10AC60009CE870008DE87C0005236A4603F0A0F99B
:10AC700006B070BD2DE9F0470E4680461C46924650
:10AC800008293ED894F80C900020207319461046ED
:10AC900002F094FB0025B54206D218F805201AA14F
:10ACA0002046FFF715F803E019A12046FFF710F83A
:10ACB0006D1C082DEFD317A12046FFF709F80025DA
:10ACC000B54210D218F80570F5F7B4FB0068C05D06
:10ACD00010F03E0F01D03A4600E02E220EA1204691
:10ACE000FEF7F6FF03E00DA12046FEF7F1FF6D1C15
:10ACF000082DE5D301222146504602F041FB84F89D
:10AD00000C90BDE8F087000020253032780000006C
:10AD1000202020007C0000002563000020000000AF
:10AD20002DE9F04705001FD0214C4FF00009FF200E
:10AD3000C4F80090C4E90190C4F81894C4F81494BD
:10AD400084F82094084600F00DF91A48C4F80C5411
:10AD500000F065F9002808D11749DFF86080A1EB01
:10AD60000800C70800241EE00720BDE8F087002681
:10AD700035460CE0AC4209D058F8340058F835108C
:10AD80001422F5F71BFC002800DD761C6D1CBD426B
:10AD9000F0D30B4904EB440001EB8000C0F80490B1
:10ADA00004804680641CBC42E1D30020DDE7000043
:10ADB000D81F0020901D01003C1D0100141C010043
:10ADC000D403002002480349401AC008704700001D
:10ADD0003C1D0100141C01007FB5054611460024EE
:10ADE00001A87BB1FCF740FCA0B901980B4900EB2E
:10ADF000400001EB800005EB45018068C84000F091
:10AE0000070407E0FCF730FC20B90548019900EB86
:10AE1000C100847904B0204670BD0000D403002036
:10AE2000141C010030B50F4B01EB410103EB810411
:10AE300000EB40000723A56803FA00F18D4302F000
:10AE400007018140294300252A46A16003FA02F048
:10AE50000840D040A84200D90546D21C0A2AF5D3A2
:10AE6000656030BDD403002013B56846FCF7FCFBD9
:10AE700008B100201CBD0248009950F831001CBDEB
:10AE8000141C010070B508480125D0F8104480F862
:10AE9000205405E065722168204649688847646847
:10AEA000002CF7D170BD0000D81F00202DE9FF470E
:10AEB00081460C9D00200C462F7B28739846164631
:10AEC0002946184602F07AFA072E42D2DFE806F049
:10AED00004090F161F2A360049462846FEF7F8FED9
:10AEE00037E0494628462268FEF7F2FE31E0D4E911
:10AEF000002349462846FEF7EBFE2AE0A0680090B2
:10AF0000D4E9002349462846FEF7E2FE21E0D4E9D1
:10AF10000201CDE90001D4E9002349462846FEF7A5
:10AF2000D7FE16E004F1080007C88DE80700D4E951
:10AF3000002349462846FEF7CBFE0AE004F108004C
:10AF40000FC88DE80F00D4E9002349462846FEF7D4
:10AF5000BFFE00222946404602F012FA2F73BDE8D8
:10AF6000FF870000054A0121054B516001E04008C0
:10AF700049009842FBD8C2E9000170473003002025
:10AF800040420F002DE9F041058B80462D1F4819E6
:10AF9000C01CB0FBF5F0C6B24046FCF763FC041ED3
:10AFA00019D00020207101206071E580002725461E
:10AFB000761EC4F800800BE04046FCF753FC60B1FD
:10AFC0006179491C6171286005467F1CC0F80080CA
:10AFD000B742F1D32046BDE8F081204600F002F8E8
:10AFE0000020F8E72DE9F041457901466B1E00226B
:10AFF00001E00968521C9A42FBD30F680146002603
:10B0000005E038460C68FCF793FC2146761CAE42FE
:10B01000F7D3BDE8F0810121001DFCF7FBBBFCF775
:10B02000CDBC10B504460121001DFCF714FC10F046
:10B03000FF0F04D12046BDE81040FFF7D3BF10BD7D
:10B0400038B501240094FCF79BFA38BD38B50024CC
:10B050000094FCF795FA38BD2DE9F84F834600F0CF
:10B0600091F90546DBF80800D0F84803C0F340002A
:10B0700030B15846BDE8F84F00221146FDF7BAB985
:10B080001C4803681CA208215846FDF755F91948C9
:10B09000001D03681DA208215846FDF74DF9DFF891
:10B0A0005480DFF8509008F10808002409F11009D5
:10B0B00008F1040A1AE00020F7F76EFAC8F8004019
:10B0C000D9F80070DAF800600020F7F793FA234609
:10B0D00013A2082158460096FDF72EF9234617A221
:10B0E000082158460097FDF727F9641CAC42E2D3CB
:10B0F000BDE8F88F90ED00E04D50555F5459504534
:10B100003A093078253038580D0A00004D50555F07
:10B110004354524C3A093078253038580D0A000013
:10B120000D0A4D50555F524241525B25755D3A09FB
:10B130003078253038580D0A000000004D50555F1A
:10B14000524153525B25755D3A09307825303858A5
:10B150000D0A00002DE9FC4107468068D0F848033D
:10B16000C0F3400038B102B03846BDE8F0410022DB
:10B170001146FDF73FB900F005F90646009030484A
:10B180000068C00701D02FA300E030A332A208213D
:10B190003846FDF7D1F800244EE00020F7F7FCF91F
:10B1A0002748001D046026480C300568001FD0F8B1
:10B1B00000800020F7F71EFAE807234633D032A2BA
:10B1C00008213846FDF7B8F8C5F344010120491CB1
:10B1D000884008EB0001491ECDE90010434630A22B
:10B1E00008213846FDF7A8F8284600F0D3F80346B2
:10B1F00037A208213846FDF79FF8284600F048F9A5
:10B20000034637A208213846FDF796F8284600F095
:10B21000FBF8034636A208213846FDF78DF8E80012
:10B2200003D538A302E038A201E03DA33DA20821E6
:10B230003846FDF781F8641CB442AED3BDE8FC810A
:10B2400094ED00E0456E61626C6564004469736171
:10B25000626C6564000000004D50552053746174A9
:10B26000653A2025732C20257520756E6966696501
:10B270006420726567696F6E732061766961626CC4
:10B28000652E0D0A0D0A0000526567696F6E202554
:10B29000753A20456E61626C65640D0A000000001D
:10B2A000092D204C6F636174696F6E3A09307825FF
:10B2B0003038582D307825303858202873697A6511
:10B2C0003A202575206279746573290D0A00000003
:10B2D000092D204163636573733A0925730D0A00D4
:10B2E000092D20547970653A090925730D0A00006B
:10B2F000092D2043616368696E673A0925730D0A59
:10B3000000000000584E0000526567696F6E2025EE
:10B31000753A2044697361626C65640D0A0000002F
:10B320002D2D0000092D20466C6167733A092573A5
:10B330000D0A0D0A0000000008B5012905D081683A
:10B34000D1F84813C1F3400129B10022BDE80840FB
:10B350001146FDF74FB851680091136802A202210F
:10B36000FCF7EAFF08BD000025733A20756E6B6E8E
:10B370006F776E20706172616D657465723A202519
:10B38000730D0A0002480068C0F3072070470000F0
:10B3900090ED00E0C0F30260082813D2DFE800F06F
:10B3A0000406080A0C0E101007A0704708A070478A
:10B3B00009A070470AA070470BA070470CA0704707
:10B3C0000DA070470EA070472D2D2F2D2D000000D1
:10B3D00052572F2D2D00000052572F524F000000C2
:10B3E00052572F52570000003F3F2F3F3F000000B1
:10B3F000524F2F2D2D000000524F2F524F000000B2
:10B40000556E6B6E6F776E0010B5C0F3C241C0F31E
:10B410004043C0F3004200F47C100404240C17D114
:10B420000014152814D2DFE800F00B0B0D0F0B0BE6
:10B430000B0B0B1313110B13130B0B1313130B0029
:10B440000A4810BD0AA010BD0BA010BD0CA010BD75
:10B45000042908D38807000F40EA43000B49104332
:10B4600051F8200010BD0148383010BDC8B30000AD
:10B4700057542F575400000057422F5742000000E6
:10B48000574257412F574257410000003C010020CE
:10B4900000F47C100104090C15D10114152912D2F5
:10B4A000DFE801F00B0D18180B0D16161811111806
:10B4B000161111160F1111110F0008A070470EA0E0
:10B4C000704712A07047C10C042905D3400301D571
:10B4D00010A0704714A0704715A070475374726F86
:10B4E0006E676C792D6F7264657265642C20536889
:10B4F00061726561626C65004465766963652C20E4
:10B50000536861726561626C65000000446576692C
:10B51000636500004E6F726D616C2C205368617220
:10B520006561626C650000004E6F726D616C0000B9
:10B530005265736572766564206F7220496D706C18
:10B54000656D656E746174696F6E20446566696EC1
:10B5500065640000094902220A60BFF36F8FBFF3E0
:10B560004F8F0A1D106006480268002AFCD0002098
:10B570000860BFF36F8FBFF34F8F704704E5014042
:10B5800000E4014070B50E4C01232360BFF36F8FC0
:10B59000BFF34F8F00230B4D08E000BF51F823602D
:10B5A00040F823602E68002EFCD05B1C9342F5D33C
:10B5B00000202060BFF36F8FBFF34F8F70BD00007E
:10B5C00004E5014000E4014000F1804108680022E8
:10B5D00010B101200A6070471046704770470000A4
:10B5E00010B5040004D105494FF4F670F7F7B8F828
:10B5F000204600F0BBFAA168081A10BD4CB8000044
:10B600002DE9F04190460D4604004FF0000703D1AC
:10B6100023A1B320F7F7A4F81DB921A1B420F7F7AF
:10B620009FF80020F6F7B8FF204600F0A1F830B1EF
:10B6300005270020F6F7DEFF3846BDE8F0812068D8
:10B640000668B8F1000F05D10168204600F046F900
:10B6500021680860E268012A0CD0022A0ED0042A70
:10B6600011D06068082A13D006FB02012846F4F7BF
:10B6700039FFDEE76068805D2870DAE7606830F8DF
:10B6800016002880D5E7606850F826002860D0E7CB
:10B6900000EBC601D1E90001C5E90001C9E70000DE
:10B6A0002E2E5C2E2E5C2E2E5C2E2E5C2E2E5C2ED4
:10B6B0002E5C636F6D706F6E656E74735C6C696227
:10B6C0007261726965735C71756575655C6E7266D1
:10B6D0005F71756575652E630000000070B51446D6
:10B6E0000E46050004D113A14FF4A170F7F738F806
:10B6F00026B910A140F24310F7F732F84FF00000DE
:10B70000002C12D0F6F748FF287C78B12846FFF7C6
:10B7100067FF844200D3044622463146284601F0A2
:10B7200008FF0020F6F766FF204670BDA868A0421B
:10B73000F2D8F0E72E2E5C2E2E5C2E2E5C2E2E5C88
:10B740002E2E5C2E2E5C636F6D706F6E656E747343
:10B750005C6C69627261726965735C71756575654F
:10B760005C6E72665F71756575652E630000000022
:10B7700010B5040004D107A14FF4F270F6F7F0FF02
:10B78000216808684968884201D1012010BD002065
:10B7900010BD00002E2E5C2E2E5C2E2E5C2E2E5CFC
:10B7A0002E2E5C2E2E5C636F6D706F6E656E7473E3
:10B7B0005C6C69627261726965735C7175657565EF
:10B7C0005C6E72665F71756575652E6300000000C2
:10B7D00070B5040003D108A16420F6F7C1FF20680A
:10B7E00005684168204600F079F8A84201D101209F
:10B7F00070BD002070BD00002E2E5C2E2E5C2E2E03
:10B800005C2E2E5C2E2E5C2E2E5C636F6D706F6E28
:10B81000656E74735C6C69627261726965735C7188
:10B82000756575655C6E72665F71756575652E63AD
:10B830000000000010B5040004D104A14FF4F97019
:10B84000F6F78EFF2068806810BD00002E2E5C2E5B
:10B850002E5C2E2E5C2E2E5C2E2E5C2E2E5C636FAC
:10B860006D706F6E656E74735C6C69627261726923
:10B8700065735C71756575655C6E72665F71756523
:10B8800075652E630000000010B5040004D104A10A
:10B890004FF4FC70F6F764FF21680020886010BD4B
:10B8A0002E2E5C2E2E5C2E2E5C2E2E5C2E2E5C2ED2
:10B8B0002E5C636F6D706F6E656E74735C6C696225
:10B8C0007261726965735C71756575655C6E7266CF
:10B8D0005F71756575652E630000000070B50C46DC
:10B8E000050003D105495120F6F73AFFA868A042A8
:10B8F00001D9601C70BD002070BD00004CB8000074
:10B9000070B514460D46060004D110A140F2AF10E8
:10B91000F6F726FF25B90DA14FF4D870F6F720FFF2
:10B920004FF00000002C10D0F6F736FE304601F044
:10B93000F4FD844200D3044622462946304601F0F5
:10B94000B9FD0020F6F756FE204670BD2E2E5C2E67
:10B950002E5C2E2E5C2E2E5C2E2E5C2E2E5C636FAB
:10B960006D706F6E656E74735C6C69627261726922
:10B9700065735C71756575655C6E72665F71756522
:10B9800075652E63000000002DE9F0410E460400AD
:10B990004FF0000803D12CA16F20F6F7E1FE1EB98D
:10B9A00029A17020F6F7DCFE0020F6F7F5FD204611
:10B9B000FFF70EFF070009D0207C38B14FF00408D4
:10B9C0000020F6F717FE4046BDE8F0812068456884
:10B9D00041682046FFF782FF2168486037B1206840
:10B9E00001682046FFF77AFF21680860E268012AB3
:10B9F00014D0022A16D0042A19D0082A1CD0606854
:10BA0000314605FB0200F4F76DFD204601F085FD8F
:10BA100021688A688242D3D28860D1E76168307831
:10BA20004855F2E76168308821F81500EDE7616854
:10BA3000306841F82500E8E7D6E90001626802EBCA
:10BA4000C502C2E90001E0E72E2E5C2E2E5C2E2EF0
:10BA50005C2E2E5C2E2E5C2E2E5C636F6D706F6ED6
:10BA6000656E74735C6C69627261726965735C7136
:10BA7000756575655C6E72665F71756575652E635B
:10BA8000000000002DE9F04F8046806889B0D0F8B2
:10BA90004803C0F3400038B109B04046BDE8F04F5C
:10BAA00000221146FCF7A6BC012907D909B040467F
:10BAB000BDE8F04F1FA20221FCF73EBC2249DFF88F
:10BAC0008CB0A1EB0B001C21B0FBF1F7002529E0A5
:10BAD000C5EBC5010BEB81042046D4E9026AFFF7F0
:10BAE000A9FE8146204600F041F8642209FB02F1DC
:10BAF0004243B1FBF6F1B2FBF6F26369247CB4B1C8
:10BB00000FF24C0CCDF81CC0CDF800A0CDE9059685
:10BB1000CDE90120CDE90361104A08214046FCF738
:10BB20000BFC6D1CBD42D3D309B0BDE8F08F0FF202
:10BB3000300CE7E742616420617267756D656E7471
:10BB400020636F756E740000541E0100AC1D01006F
:10BB50004E6F206F766572666C6F7700281001005B
:10BB60004F766572666C6F770000000010B50400B8
:10BB700004D108A140F2D710F6F7F2FD0020F6F745
:10BB80000BFD204601F0C9FC04460020F6F732FD0B
:10BB9000204610BD2E2E5C2E2E5C2E2E5C2E2E5C92
:10BBA0002E2E5C2E2E5C636F6D706F6E656E7473DF
:10BBB0005C6C69627261726965735C7175657565EB
:10BBC0005C6E72665F71756575652E6300000000BE
:10BBD0002DE9F0411F4615460E00044603D11D49CC
:10BBE0001520F6F7BDFD1DB91A491620F6F7B8FD68
:10BBF00037B1A068FBF70BFE10B11120BDE8F08152
:10BC0000A0686168D0E903C3ACEB0302481C824220
:10BC100007D10020286017B1A068FBF7EFFD0020D6
:10BC2000ECE70CEA010003EA0102904202D3091A90
:10BC3000491C01E0A3EB0C012B688B4200D2194692
:10BC40002960216808443060A0682A68C1681144EE
:10BC5000C160E4E7A41001002DE9F04117465FEA56
:10BC60000108054603D121499C20F6F779FD1FB94B
:10BC70001E499D20F6F774FDA868001DFBF7C7FD5F
:10BC800010B11120BDE8F081A868816800690C1A24
:10BC90003868A04200D204463C60AA68696810690E
:10BCA000926808400A40824201D9161A01E00E1A31
:10BCB000761CB44208D92968324608444146F4F754
:10BCC00011FCA41B0020B0442968224601444046D0
:10BCD000F4F708FCA8683A68016911440161A86892
:10BCE000001DFBF78BFD0020CCE70000A410010035
:10BCF0002DE9F04117465FEA0108054603D11E49C8
:10BD00004D20F6F72DFD1FB91B494E20F6F728FDF3
:10BD1000A868FBF77CFD10B11120BDE8F081A86890
:10BD200081680069081A69680C1A3868641CA042A6
:10BD300000D204463C60A8686968806808400E1A12
:10BD4000761CB44208D92968324608444146F4F7C3
:10BD5000C9FBA41B0020B044296822460844414680
:10BD6000F4F7C0FBA8683A68816811448160A8684C
:10BD7000FBF744FD0020D0E7A410010010B5826855
:10BD800094681369E41AA14201D9042010BD194432
:10BD90001161826851618068001DFBF72FFD002052
:10BDA00010BD00002DE9F0411E4614460F00054667
:10BDB00003D11D496D20F6F7D3FC1CB91A496E203A
:10BDC000F6F7CEFC3EB1A868001DFBF720FD10B1D0
:10BDD0001120BDE8F081A96888684969421A09D034
:10BDE0006B681940184088420DD9266896420AD9D6
:10BDF000226010E0002020601EB1A868001DFBF743
:10BE0000FDFC0020E5E7884205D8581A2268401C4E
:10BE1000824200D92060286808443860A8682268F7
:10BE2000416911444161ECE7A410010082680021DE
:10BE3000916082681161826851618268D160826814
:10BE4000516080680160704770B582684568946889
:10BE50001369E31AEB1A5B1C994201D9042070BDE7
:10BE6000214491608268D1608068FBF7CAFC08B108
:10BE7000002070BD082070BD70B50D46060003D1CE
:10BE80000BA11420F6F76CFC1DB909A11520F6F7DB
:10BE900067FC746804E0B2682946904718B12468CA
:10BEA00020680028F7D120682860256070BD000058
:10BEB0002E2E5C2E2E5C2E2E5C2E2E5C2E2E5C2EBC
:10BEC0002E5C636F6D706F6E656E74735C6C69620F
:10BED0007261726965735C736F72746C6973745CA0
:10BEE0006E72665F736F72746C6973742E63000098
:10BEF00010B5040003D103A13D20F6F731FC206802
:10BF000010BD00002E2E5C2E2E5C2E2E5C2E2E5C84
:10BF10002E2E5C2E2E5C636F6D706F6E656E74736B
:10BF20005C6C69627261726965735C736F72746C68
:10BF30006973745C6E72665F736F72746C6973742C
:10BF40002E63000010B5040003D103A13720F6F7DB
:10BF500007FC6068006810BD2E2E5C2E2E5C2E2E15
:10BF60005C2E2E5C2E2E5C2E2E5C636F6D706F6EC1
:10BF7000656E74735C6C69627261726965735C731F
:10BF80006F72746C6973745C6E72665F736F7274D7
:10BF90006C6973742E63000010B5040003D105A111
:10BFA0002B20F6F7DDFB61680868002801D00268E5
:10BFB0000A6010BD2E2E5C2E2E5C2E2E5C2E2E5C6A
:10BFC0002E2E5C2E2E5C636F6D706F6E656E7473BB
:10BFD0005C6C69627261726965735C736F72746CB8
:10BFE0006973745C6E72665F736F72746C6973747C
:10BFF0002E63000070B50C46050003D10BA1432051
:10C00000F6F7AEFB1CB909A14420F6F7A9FB002105
:10C01000686806E0A24203D121680160012103E0C3
:10C0200010460268002AF5D1084670BD2E2E5C2EFF
:10C030002E5C2E2E5C2E2E5C2E2E5C2E2E5C636FC4
:10C040006D706F6E656E74735C6C6962726172693B
:10C0500065735C736F72746C6973745C6E72665F27
:10C06000736F72746C6973742E6300000C4A10B5A0
:10C0700002F58C730EE0991AC91001EBD1714910C9
:10C0800002EBC1010C68844201D90B4602E005D2E3
:10C0900001F108029A42EED3002010BD486810BD9D
:10C0A00074F9000000B5FFF7E1FF002800D1014856
:10C0B00000BD000060F900004058002800D00120B9
:10C0C000704708B5002242504058009008BDD0F893
:10C0D0000403084000D0012070474058002800D0D9
:10C0E0000120704708B5002242504058009008BD1A
:10C0F00030B5050600F00F030E4C03EB830004EB94
:10C1000080000AD5082B03D30B480160001D09E00D
:10C11000C0F80016C0F8042630BD082B04D3074829
:10C120000160001D026030BDC0F80017C0F8042790
:10C1300030BD000000700240A0760240A0770240AF
:10C1400010B5044600F00F00092804D30BA140F2FB
:10C150009640F6F705FB21064FF0010004F00F02B0
:10C1600000FA02F001D5114901E01049091D0968E2
:10C17000014201D0012010BD002010BD2E2E5C2EEA
:10C180002E5C2E2E5C2E2E5C2E2E5C2E2E5C6D6F69
:10C1900064756C65735C6E7266785C68616C5C6E0D
:10C1A00072665F757362642E68000000107502404D
:10C1B00070B50446000604D415A140F29B30F6F792
:10C1C000CFFA04F00F00082804D311A14FF46770D0
:10C1D000F6F7C6FA200704D10DA140F29D30F6F71C
:10C1E000BFFA02F0D7FC2046F9F76EFE817B0125ED
:10C1F000032902D00068002809D12046F9F730FE53
:10C200008540E943BDE870401148FBF709BB70BDAC
:10C210002E2E5C2E2E5C2E2E5C2E2E5C2E2E5C2E58
:10C220002E5C636F6D706F6E656E74735C647269A3
:10C23000766572735F6E72665C757362645C6E7253
:10C24000665F6472765F757362642E63000000003F
:10C25000A001002038B50446000604D41B4940F272
:10C26000BB30F6F77DFA04F00F00082804D2174916
:10C270004FF46F70F6F774FA02F08CFC2046F9F771
:10C2800023FE817B0125032915D00068002811D1E8
:10C290002046F9F7E5FD8540E9430D48FBF7C0FA74
:10C2A0000C480B49806800900C398DF802404968B1
:10C2B0006846884738BD2046F9F7D2FD8540E943F6
:10C2C000BDE838400248FBF7ABBA0000E0EB0000E5
:10C2D000A001002060F3000038B50446000604D534
:10C2E0001FA14FF47F70F6F73BFA04F00F00082807
:10C2F00004D31BA140F2FD30F6F732FA200704D137
:10C3000017A140F2FE30F6F72BFA02F043FC20466C
:10C31000F9F7DAFD817B0125032902D0006848B1D5
:10C320001AE02046F9F79CFD8540E9431C48FBF7DD
:10C3300077FA11E02046F9F793FD8540E943184864
:10C34000FBF76EFA17481649006900900C398DF812
:10C350000240496868468847BDE8384002F060BC42
:10C360002E2E5C2E2E5C2E2E5C2E2E5C2E2E5C2E07
:10C370002E5C636F6D706F6E656E74735C64726952
:10C38000766572735F6E72665C757362645C6E7202
:10C39000665F6472765F757362642E6300000000EE
:10C3A000A001002060F3000070B50546000605F00E
:10C3B0000F0402D5092C09D301E0092C0BD30D4938
:10C3C00040F23E40F6F7CCF9280604D5094940F280
:10C3D0003F40F6F7C5F9082C05D307480068C103AC
:10C3E00000D5002070BD054901EB8400D0F8A00401
:10C3F00070BD0000309C0000C0740240007002401C
:10C4000002494058002800D00120704700700240C7
:10C410000449084400210160BFF36F8FBFF34F8FC1
:10C42000704700000070024003490860BFF36F8F3F
:10C43000BFF34F8F7047000000740240024800684D
:10C44000002800D0012070472C75024004490844A0
:10C4500001210160BFF36F8FBFF34F8F7047000062
:10C4600000700240084810B5007918B907A195205E
:10C47000F6F776F900F03AF912490120086002490E
:10C48000091F087010BD0000AC0100202E2E5C2E8C
:10C490002E5C2E2E5C2E2E5C2E2E5C2E2E5C6D6F56
:10C4A00064756C65735C6E7266785C6472697665DF
:10C4B00072735C7372635C6E7266785F636C6F63D9
:10C4C0006B2E630018050040084810B5007918B9B4
:10C4D00007A1D420F6F744F94FF48070FCF7BBFABB
:10C4E00001208107C1F80403086010BDAC010020E1
:10C4F0002E2E5C2E2E5C2E2E5C2E2E5C2E2E5C2E76
:10C500002E5C6D6F64756C65735C6E7266785C64CE
:10C510007269766572735C7372635C6E7266785F63
:10C52000636C6F636B2E630010B50A4C207918B9E9
:10C5300009A1DC20F6F714F9154901200860154916
:10C540004FF001100A6802F001128242FAD0002076
:10C55000607110BDAC0100202E2E5C2E2E5C2E2EA4
:10C560005C2E2E5C2E2E5C2E2E5C6D6F64756C65C1
:10C57000735C6E7266785C647269766572735C7304
:10C5800072635C6E7266785F636C6F636B2E6300C0
:10C59000040000400C04004010B5040003D108A1C1
:10C5A0007C20F6F7DDF8144900200A790AB18520CD
:10C5B00010BD01220C600A7100224A7110BD0000FA
:10C5C0002E2E5C2E2E5C2E2E5C2E2E5C2E2E5C2EA5
:10C5D0002E5C6D6F64756C65735C6E7266785C64FE
:10C5E0007269766572735C7372635C6E7266785F93
:10C5F000636C6F636B2E6300AC01002070B54FF469
:10C6000080763046FCF720FA114CB50560B1304613
:10C61000FCF721FA0120C5F80803607920B9012050
:10C6200060712168002088474FF482763046FCF71D
:10C630000BFA00280AD03046FCF70DFA0220C5F8A4
:10C6400008032168BDE870400120084770BD000064
:10C65000AC010020094810B5007918B908A1BF2025
:10C66000F6F77EF84FF48270FCF7F5F902204107E7
:10C67000C1F8040310490120086010BDAC0100207E
:10C680002E2E5C2E2E5C2E2E5C2E2E5C2E2E5C2EE4
:10C690002E5C6D6F64756C65735C6E7266785C643D
:10C6A0007269766572735C7372635C6E7266785FD2
:10C6B000636C6F636B2E630008000040002802D09B
:10C6C0000149800108477047A1F300000121B1EB47
:10C6D000507F01D101207047002070470121B1EB4C
:10C6E000507F01D101207047002070470748006843
:10C6F000012110F0010F08D14FF0E020E02280F876
:10C700000024C0F88012C0F80011704700E100E07A
:10C7100007480068012110F0010F08D14FF0E02018
:10C72000E02280F80024C0F88012C0F800117047A1
:10C7300000E100E070B5040003D10DA14620F6F73A
:10C740000FF8194D287808B1852070BD2078174959
:10C75000C0F34000086015492078083900F0010056
:10C760000860FFF7D5FF01202870002070BD000091
:10C770002E2E5C2E2E5C2E2E5C2E2E5C2E2E5C2EF3
:10C780002E5C6D6F64756C65735C6E7266785C644C
:10C790007269766572735C7372635C6E7266785FE1
:10C7A000706F7765722E6300B40100208005004031
:10C7B00070B54FF08040D0F80453324C68070CD568
:10C7C0004FF48470FEF700FF38B1606818B92EA1ED
:10C7D000E020F5F7C5FF60688047A8060DD54FF447
:10C7E0008A70FEF7F1FE40B1A06818B926A1E820D2
:10C7F000F5F7B6FFA1680020884768060DD54FF40D
:10C800008C70FEF7E1FE40B1A06818B91EA1EF20C0
:10C81000F5F7A6FFA1680120884728060DD54FF43B
:10C820008E70FEF7D1FE40B1E06818B916A1F8206D
:10C83000F5F796FFE16800208847E8050DD54FF42D
:10C840009070FEF7C1FE40B1E06818B90EA1FF205C
:10C85000F5F786FFE16801208847A80511D54FF458
:10C860009270FEF7B1FE00280BD0E06820B906A157
:10C870004FF48370F5F774FFE168BDE87040022063
:10C88000084770BDB40100202E2E5C2E2E5C2E2E8B
:10C890005C2E2E5C2E2E5C2E2E5C6D6F64756C658E
:10C8A000735C6E7266785C647269766572735C73D1
:10C8B00072635C6E7266785F706F7765722E63006C
:10C8C0004FF080414FF46070C1F8080370474FF09B
:10C8D00080414FF46070C1F804037047034900229F
:10C8E000CA600068002800D0C8607047B40100200A
:10C8F00001490020C8607047B401002070B50D46A2
:10C90000040003D10DA15120F5F72AFF204600F0C5
:10C91000B3FD04000FD00020F5F73EFE207920B1D2
:10C920000020F5F767FE112070BD01202560207101
:10C930000020F5F75FFE002070BD00002E2E5C2E5B
:10C940002E5C2E2E5C2E2E5C2E2E5C2E2E5C6D6FA1
:10C9500064756C65735C6E7266785C64726976652A
:10C9600072735C7372635C7072735C6E7266785F14
:10C970007072732E6300000010B5040003D106A18D
:10C980007520F5F7EDFE204600F076FD002802D078
:10C9900000210160017110BD2E2E5C2E2E5C2E2E0A
:10C9A0005C2E2E5C2E2E5C2E2E5C6D6F64756C657D
:10C9B000735C6E7266785C647269766572735C73C0
:10C9C00072635C7072735C6E7266785F7072732EE5
:10C9D000630000000149024801F098BE581A002087
:10C9E000002000402DE9F04117460D00064603D116
:10C9F0001AA18420F5F7B4FE3079264A00EB4001F5
:10CA000001EBC00102EB810494F82A1011B1082057
:10CA1000BDE8F081204951F820103068FFF76EFF23
:10CA200008B11120F4E729463046F5F723FE676088
:10CA3000286920601FB1297F3046FAF7D5F83068A1
:10CA40000421C0F800150020A061E06184F82900ED
:10CA500044F8140F0121A175DAE700002E2E5C2E98
:10CA60002E5C2E2E5C2E2E5C2E2E5C2E2E5C6D6F80
:10CA700064756C65735C6E7266785C647269766509
:10CA800072735C7372635C6E7266785F75617274E8
:10CA90002E630000581A00204CF400002DE9F05FCE
:10CAA000054600790F4600EB400101EBC00140480C
:10CAB000164600EB810494F82A00012804D03DA119
:10CAC00040F24310F5F74CFE4FF4A27A1FB939A19A
:10CAD0005046F5F745FE26B936A140F24510F5F768
:10CAE0003FFE616800204FF4017811B12A68C2F856
:10CAF0000883A1694FF0000969B1E06938B1606845
:10CB000010B12868C0F804831120BDE8F09F2761A8
:10CB10000120E66105E0C4F82490E760A661C4F84E
:10CB20001C9094F82910014302D1284600F08CFE95
:10CB300060680028286803D0C0F804830020E4E778
:10CB400056465146FFF7BDFAB2464FF4927B59461E
:10CB50002868FFF7B1FA06464FF484712868FFF79A
:10CB6000ABFA804651462868FFF7A6FA074648EA1E
:10CB700007003043EBD056EA070007D1214628686A
:10CB800000F032FE616AA0698842E0D8C4F81890CB
:10CB90000EB10320B9E70FB10F20B6E794F82910C2
:10CBA00001200029296801D00860C7E74860C5E76F
:10CBB000581A00202E2E5C2E2E5C2E2E5C2E2E5C03
:10CBC0002E2E5C2E2E5C6D6F64756C65735C6E72C0
:10CBD00066785C647269766572735C7372635C6EAE
:10CBE0007266785F756172742E63000001684FF49D
:10CBF0000172C1F8082300680121416070470000FC
:10CC00002DE9F047054600790F4600EB400101EBA6
:10CC1000C0002D49164601EB800494F82A00012833
:10CC200003D02AA1EF20F5F79BFD1FB927A1F02023
:10CC3000F5F796FD1EB925A1F120F5F791FD2846DF
:10CC400000F060F810B11120BDE8F0874FF0000847
:10CC5000C4F82080A760666184F828804FF48E763F
:10CC6000474631462868FFF72CFA28684FF001093B
:10CC7000C0F808902146286801F08CFC606808BB69
:10CC8000D5F800A00FE000BF94F8280008B10F27E6
:10CC900016E031465046FFF70FFA0028F4D021463F
:10CCA000504601F077FC216A60698142F1D3314638
:10CCB0002868FFF701FA0028F9D02868C0F80C901E
:10CCC000C4F814803846BFE7581A00202E2E5C2E78
:10CCD0002E5C2E2E5C2E2E5C2E2E5C2E2E5C6D6F0E
:10CCE00064756C65735C6E7266785C647269766597
:10CCF00072735C7372635C6E7266785F7561727476
:10CD00002E630000007900EB400101EBC0000449F4
:10CD100001EB80004069002800D00120704700002E
:10CD2000581A00202DE9F047044600794FF0000919
:10CD300000EB400101EBC000254901EB80072068B2
:10CD4000C0F80095786880B120682249C0F80813BF
:10CD500020680121000B40B200F01F029140400901
:10CD6000800000F1E020C0F880112068D0F80C2588
:10CD7000D0F81485D0F80865D0F810554FF0FF3181
:10CD8000C0F81415C0F80C152068C0F80815C0F8D4
:10CD90001015501C02D01046FDF744FBB8F1FF3FC0
:10CDA00002D04046FDF73EFB681C02D02846FDF746
:10CDB00039FB701C02D03046FDF734FB2068FFF7CA
:10CDC000DBFD87F82A90C7F80490BDE8F0870000E3
:10CDD000581A0020840202000149024801F042BDB5
:10CDE000841A0020002000402DE9F04117460D0074
:10CDF000064603D118A19620F5F7B2FC3079244AF3
:10CE000000EBC00102EB810494F8201011B108205E
:10CE1000BDE8F0811F4951F820103068FFF76EFD22
:10CE200008B11120F4E729463046F5F75EFC67604B
:10CE3000286920601FB1297F3046F9F729FF306843
:10CE40000821C0F800150020A061E06101216061A7
:10CE500084F82010DCE700002E2E5C2E2E5C2E2E97
:10CE60005C2E2E5C2E2E5C2E2E5C6D6F64756C65B8
:10CE7000735C6E7266785C647269766572735C73FB
:10CE800072635C6E7266785F75617274652E6300A2
:10CE9000841A002050F400002DE9F05F0446007968
:10CEA0000F46DFF834A100EBC0010AEB81051646FE
:10CEB00095F82000012804D048A140F23110F5F780
:10CEC0004FFC27B945A14FF49970F5F749FC26B9F5
:10CED00042A140F23310F5F743FC207910B9B6F5C2
:10CEE000803F04D33DA14FF49A70F5F739FC3846E2
:10CEF000FFF7F4FBB0B168684FF000084FF4047915
:10CF000010B12168C1F80893A8694FF0000B80B1F7
:10CF1000E86948B1686810B12068C0F8049311202E
:10CF2000BDE8F09F1020FBE72F614FF00108EE6194
:10CF300002E0EF60C5E9066B00254FF488712068B8
:10CF4000FFF7D0F84FF4A2712068FFF7CBF8206804
:10CF5000C0F83475C0F838652068B8F1000F12D0F9
:10CF6000D0F8001241F02001C0F800122079D0461C
:10CF700000EBC0010AEB8100406838B12168C1F8BC
:10CF800004932846CCE701210160EFE74FF4887A4B
:10CF90004FF4A27951462068FFF79FF807464946AB
:10CFA0002068FFF79AF806464FF492712068FFF761
:10CFB00094F8014647EA06000843EBD0227902EBD9
:10CFC000C20308EB8302C2F818B001B10325002E9A
:10CFD000D7D00F25D5E70000841A00202E2E5C2E16
:10CFE0002E5C2E2E5C2E2E5C2E2E5C2E2E5C6D6FFB
:10CFF00064756C65735C6E7266785C647269766584
:10D0000072735C7372635C6E7266785F7561727462
:10D01000652E630000680121416070472DE9F047EB
:10D0200004460F4600792D4900EBC00001EB800556
:10D03000164695F82000012803D029A1E720F5F72E
:10D040008FFB1FB926A1E820F5F78AFB1EB924A1A2
:10D05000E920F5F785FB207910B9B6F5803F03D3B9
:10D060001FA1EA20F5F77CFB3846FFF737FB30B10C
:10D07000204600F051F820B11120BDE8F0871020C3
:10D08000FBE7AF606E614FF4907600273146206871
:10D09000FFF728F84FF4AC7841462068FFF722F8F4
:10D0A0002068AA686969C0F84425C0F84815206856
:10D0B00001218160686878B9B14649462068FFF768
:10D0C0000CF8064641462068FFF707F80643F4D0FF
:10D0D00000B10F27002068613846CEE7841A00208F
:10D0E0002E2E5C2E2E5C2E2E5C2E2E5C2E2E5C2E7A
:10D0F0002E5C6D6F64756C65735C6E7266785C64D3
:10D100007269766572735C7372635C6E7266785F67
:10D1100075617274652E63000079054900EBC000EB
:10D1200001EB80004069002800D00120704700001A
:10D13000841A00202DE9F04704460079274900EBC6
:10D14000C00001EB800720684FF00009C0F800958F
:10D15000786880B120682249C0F80813206801214E
:10D16000000B40B200F01F0291404009800000F126
:10D17000E020C0F880112068D0F80C25D0F8148584
:10D18000D0F80865D0F810554FF0FF31C0F80C15F5
:10D19000C0F814152068C0F80815C0F81015501C08
:10D1A00002D01046FDF747F9B8F1FF3F02D04046E4
:10D1B000FDF741F9681C02D02846FDF73CF9701CC8
:10D1C00002D03046FDF737F92068FFF7D5FB87F826
:10D1D0002090C7F80490BDE8F0870000841A002072
:10D1E0001003020010B5124C606898B16068406985
:10D1F0004068042808D3606804214069008801EB76
:10D2000000400CA1FDF702FD606801F00BF8002062
:10D21000606010BD0A4841680229FAD300880221E3
:10D2200001EB0040BDE8104006A1FDF7EFBC000097
:10D23000CC010020436F6D7061726520455654002B
:10D24000DC040020436F6D70617265206576656E49
:10D250007420627574206E6F206163746976652036
:10D2600074696D65722028616C72656164792073E0
:10D27000746F707065643F290000000070B5164837
:10D280004168042906D30088042101EB004013A162
:10D29000FDF7BCFC1548416829B141684968406800
:10D2A00021F07F41416000F045FE040013D04FF0B3
:10D2B00080756068A84203D2204600F0B3FF03E007
:10D2C000606820F07F4060602046FEF711FE002875
:10D2D00001D00446EDE770BDDC0400204F76657296
:10D2E000666C6F772045565400000000CC0100208A
:10D2F0002DE9F84317460C0005462BD0DFF8708067
:10D300004646D8F80000F6F7D9FE384487B23068B0
:10D31000F6F7D4FEA968498A081AB0FBF7F086B27E
:10D320002046F6F7CBFEA968381A87B2088BB0FB07
:10D33000F6F206FB1202401C088382B123460DA2BE
:10D3400007212846FAF7F8FF39462846BDE8F84392
:10D35000F8F730BBA96800200883BDE8F883009483
:10D3600005A207212846D8F80030FAF7E5FFEBE7D9
:10D37000B8020020257300000D0A257325730000F4
:10D3800010B50C46017A052908D0407A38B1084812
:10D3900008A102682046FCF79BFC00E01AB106A138
:10D3A0002046FCF795FC2046BDE81040FCF7D0BCB9
:10D3B0004C030020257300000D0A000038B5C38817
:10D3C0000D46044633B116A0009017A218A12846B6
:10D3D000FCF77EFC217A052920D0607A48B1A0882C
:10D3E000FDF7D2FA184951F8202018A12846FCF779
:10D3F0006FFC2846216801F087F8A0880021FDF71E
:10D4000033FD03461049207A143951F8202001B029
:10D410002846BDE830400EA1FCF75ABC38BD0000DC
:10D420001B5B306D000000001B5B313B33316D0036
:10D4300025734C6F67732064726F70706564202869
:10D4400025642925730D0A004C0300202573000074
:10D450003C25733E2025733A20000000EFF3058041
:10D46000C005C00D01D001207047EFF3148040F3D8
:10D470000000401C704700000349884201D1034866
:10D48000704700207047000000200040C4010020C9
:10D4900008B500226946FEF7B3F8002806D1044813
:10D4A0008169491C81610098FDF7BBFD08BD000042
:10D4B000C80200202DE9F04104460068174688465E
:10D4C00005684068854201D8461B02E0A068461BFB
:10D4D000761CE2686068B74205FB02010CD87A430B
:10D4E0004046F2F7FFFFA168E819884200D9002002
:10D4F00021680860BDE8F08102FB06F52A46404637
:10D50000F2F7F0FFE268BE1B724308EB05006168AA
:10D51000F2F7E8FF20680660ECE701680A684968EE
:10D52000914201D3881A70478068801A0844401CD1
:10D5300070472DE9F047164689460446FEF750F835
:10D5400080462068A168426840688F1A6168E26876
:10D550007F1C00FB0210BE420FD872434946F2F70F
:10D56000C1FF20684168A2683144914202D84168F5
:10D57000314400E00021416018E002FB07F52A4633
:10D580004946F2F7AFFFE268F71B7A4309EB050162
:10D590006068F2F7A7FF20684760B04506D22068B0
:10D5A00041682046FEF79AF9216808602046FFF797
:10D5B000B4FF21688A68824200D28860BDE8F087A3
:10D5C0002DE9F0479246894604004BD02078212867
:10D5D00005D05E2803D000270126002035E0012772
:10D5E000641CF9E700262F2D02D05C2D04D00CE03E
:10D5F0004FF0FF30BDE8F0875FEACA7006D114F83B
:10D60000010B5146F9F767F8C5B25DB320782D28B4
:10D610002AD160785146F9F75EF810F0FF0023D068
:10D620005D2821D0A41C5C280AD15FEACA7107D109
:10D6300014F8010B5146F9F74EF810F0FF00D9D05D
:10D640004D4503DC814501DC0120804614F8010BC7
:10D650005146F9F740F8C5B25D2DC3D1002EC1D1B6
:10D66000B84504D10020C5E74D45EFD1ECE7204691
:10D67000C0E710B510461A46F2F734FF002010BD7F
:10D680000846704710B50446F8F7AFFA08B1FFF73F
:10D69000F5FD00212046F8F7C1F908B1FFF7A2FD1A
:10D6A000204600F059FE2046BDE81040AFF3008050
:10D6B0002DE9F047334C814600264FF0040800BFA7
:10D6C00000F038FC002854D0476860684068616802
:10D6D000C1B1616800294AD0B84248D96068007E6B
:10D6E00080B1606840694068042807D36068406979
:10D6F000018808EB014024A1FDF788FA61682748FA
:10D70000FEF7BAFB00F01CFC05464069416804299D
:10D7100006D301883A4608EB014021A1FDF77AFAC9
:10D720006A6818484FF47A7300210830F8F77EFAD7
:10D7300080B10D2811D021499C20F5F711F86869B6
:10D7400041680429BCD3018808EB01401CA1FDF706
:10D750005DFAB5E7606820B106E0284600F062FD9A
:10D76000EDE74846F8F746FA6560002EA8D1BDE817
:10D77000F08760680028FAD14846BDE8F047F8F71E
:10D7800047BA0000CC01002054696D6572207072A8
:10D7900065656D707465642E000000005CF4000027
:10D7A00041637469766174696E672074696D65722E
:10D7B000202843433A2564292E000000400401003C
:10D7C00054696D6572206578706972656420626560
:10D7D000666F7265207363686564756C6564207438
:10D7E0006F205254432E000070B5054688690C46E0
:10D7F00000284FF4847128460AD0FEF762FCD5F861
:10D800001805626AE1688854606A401C606270BDF5
:10D81000FEF757FCD5F8180570BD1FB501238DF82C
:10D820000030CDE90121D0E90012684690471FBDC4
:10D830001FB501238DF800308DF808100192D0E952
:10D840000012684690471FBD10B5044600684FF4AB
:10D850009271FEF736FC4FF484712068FEF731FCBC
:10D8600020680121016010BD7CB50546FF200090B5
:10D8700001236A4601A9E868FEF7AAF9040004D06A
:10D8800010A11A20F4F76CFF19E0009ABAB1686988
:10D890001C4C01990378D2B2E35C1BB1001DFFF769
:10D8A000FBFA02E00C30FFF7F9F8040007D1A86892
:10D8B0002A4640F6CD410068F3F708FE04462046AC
:10D8C0007CBD00002E2E5C2E2E5C2E2E5C2E2E5C3F
:10D8D0002E2E5C2E2E5C636F6D706F6E656E747392
:10D8E0005C6C69627261726965735C636C695C75BA
:10D8F0006172745C6E72665F636C695F756172748D
:10D900002E63000080010020342800D93420C01C80
:10D9100020F0030070470020704700002DE9FE430F
:10D9200008790C46012804D0022805D0032872D1BA
:10D9300072E01222404977E0B4F80700092800D9C4
:10D940000920814609264FF00008F3F7CDFF25E0B6
:10D95000686820B939A140F29720F4F701FF6868A0
:10D96000406820B935A14FF42670F4F7F9FE00277E
:10D97000009700E07F1C686801230022D0F804C0F3
:10D9800029466846E0470028F4D1297A3E4401EB55
:10D99000080000F0FF082846F4F70AF80500D7D180
:10D9A00002A8F4F79BF902990546894504D923A1F9
:10D9B00040F2AD20F4F7D4FE1F494A461231284602
:10D9C000F2F790FD85F804806E80F4F719F818B12D
:10D9D000E87940F02000E871F3F786FF0146264819
:10D9E00080E82202B4F80710C1600020F4F7D4FDEB
:10D9F000114980200839F4F701FA040005D10E49D5
:10DA000080201039F4F7C6F804460020F4F7F2FD40
:10DA10002046BDE8FE830DE0E078B4F80510F4F789
:10DA20008DFD010006D00A7803B0601CBDE8F0430C
:10DA3000F4F724B90620ECE7F4F400002E2E5C2E57
:10DA40002E5C2E2E5C2E2E5C2E2E5C2E2E5C636F9A
:10DA50006D706F6E656E74735C6C69627261726911
:10DA600065735C757362645C6170705F757362642A
:10DA70005F636F72652E6300FC1B002038B50D4696
:10DA80006846F4F72BF904460098022804D20CA14A
:10DA900040F26F20F4F764FE0020208020781749C0
:10DAA00040F00100207049784908C90702D040F0D1
:10DAB0000200207002222146681CF4F7DFF838BD0E
:10DAC0002E2E5C2E2E5C2E2E5C2E2E5C2E2E5C2E90
:10DAD0002E5C636F6D706F6E656E74735C6C6962E3
:10DAE0007261726965735C757362645C6170705FAA
:10DAF000757362645F636F72652E630014020020A9
:10DB0000F8B50C46070004D142A140F22930F4F7E1
:10DB100027FE24B93FA140F22A30F4F721FE6078B5
:10DB200010F0600F2AD10006494DA0784FF0000692
:10DB300026D520B1062808D008281FD10BE02146A1
:10DB40003846BDE8F840FFF799BF21463846BDE8A2
:10DB5000F840FFF7E3BE6846F4F7C0F801462878BE
:10DB6000052802D0042803D008E00120087000E056
:10DB70000E700122601CF4F781F8F8BD0620F8BD94
:10DB80000A28FBD2DFE800F0051E0513050605058F
:10DB9000052DF3E72878032803D0042801D00528B1
:10DBA00024D1F3F7DBFC042000F040FF15E0B4F8CB
:10DBB00003000128E2D1F3F723FF80B1687840F039
:10DBC000020009E0B4F803000128D7D1F3F718FFE9
:10DBD00028B1687820F0020068700020F8BD0F209E
:10DBE000F8BD2878052803D0042801D00820F8BD06
:10DBF000E07818B1012805D00720F8BDF3F7AEFC96
:10DC0000042002E0F3F7C2FC052000F00FFF3046CD
:10DC1000F8BD00002E2E5C2E2E5C2E2E5C2E2E5C6F
:10DC20002E2E5C2E2E5C636F6D706F6E656E74733E
:10DC30005C6C69627261726965735C757362645C65
:10DC40006170705F757362645F636F72652E6300ED
:10DC500014020020F8B50546407810F0600F31D16D
:10DC600020486C79A978007821B1012923D00329B3
:10DC700028D111E0052801D0200729D16846F4F702
:10DC80002DF806462046FBF729FB3080022231465C
:10DC9000681CF3F7F3FFF8BD04F00F01082911D257
:10DCA000B5F8031071B9052801D0200710D120461E
:10DCB000FBF7FAFA14E004F00F01082902D2B5F8D4
:10DCC000031009B10620F8BD052803D0200701D0B4
:10DCD0000820F8BD2046FBF7BDF92046FBF716FBF0
:10DCE0000020F8BD14020020FEB50C46050004D14A
:10DCF0002F494FF4D170F4F733FD24B92C4940F289
:10DD0000A310F4F72DFD60784FF00606010642D50A
:10DD1000C0F3411111B1012924D125E000F01F0009
:10DD200001281FD1A07806281CD10020019002A84C
:10DD3000F3F7D4FF064601A80090E2782179334634
:10DD40002846F3F771FD05280CD00198402803D32D
:10DD50001749A320F4F704FD3146601C019AF3F73C
:10DD60008DFFFEBD0620FEBD2846F5F731F9F4F71C
:10DD700081FDA178212903D1B4F80710072901D02A
:10DD80003046FEBD072200F10C0103B0601CBDE867
:10DD9000F040F3F773BFC0F341100028F0D0012822
:10DDA000E0D103B021462846BDE8F04000F046B877
:10DDB000CC040100F8B50B4651780646144611F024
:10DDC000600F25D11C480906A17800781ED511B135
:10DDD0000A291DD109E005281ED16846F3F77EFF08
:10DDE00001460020088002220CE0052814D1684674
:10DDF000F3F774FF054619463046F4F761FA2870C8
:10DE000001222946601CF3F739FFF8BD0B2901D028
:10DE10000620F8BD052801D00820F8BDB4F803009D
:10DE2000FF2801D90720F8BDD27819463046BDE851
:10DE3000F840F4F717BA000014020020F0B585B0DE
:10DE40000D460746F5F7C4F8F4F714FD0446A87824
:10DE50000026202802D022282FD12BE0B5F8070079
:10DE600007282AD13846F5F7B3F80446F4F702FD3F
:10DE7000A9780170E9794170811C019602960091A0
:10DE8000407801900020F4F787FB69460020F4F702
:10DE900001F8050008D11D4803A90068CDE9030475
:10DEA0000020F3F777FE05460020F4F7A3FB284691
:10DEB00005B0F0BDB5F8070008B10620F8E7207DF1
:10DEC000B5F8031000F0010001F00105A182A8429D
:10DED0001AD00DB1022100E00321384601F068F8A4
:10DEE00095B93846F7F77EFDFBF782F83846F7F725
:10DEF00082FDFBF77DF8A6612662E6662667666707
:10DF000004F12800A667A0660020D1E7B4F4000061
:10DF10000022CA604A60054A8A60052803D2044A82
:10DF200052F8200000E00020086070472CFB000041
:10DF3000140300200148FEF705B800005CF400005F
:10DF40000148FEF729B800005CF400002DE9F0411B
:10DF500007460025F6F7B2F886B2002F25D0002438
:10DF600020E000BFF2F766FA0168385D085CC00780
:10DF700016D0601C06E03A5C8A5CD20706D06D1CA5
:10DF8000ADB2401C80B2B042F5D309E045B13918BA
:10DF9000751B38196A1C401CF2F7A4FAAEB20025B2
:10DFA000641CA4B2701E8442DCDBBDE8F08100007A
:10DFB0002DE9F84FDFF8B0809246894606461F46A5
:10DFC000012269461846D8F80850F4F7DDFBE8B39B
:10DFD000009800210446C01C0AE000BF00EA0502C8
:10DFE0005AF821C008EB8202401C491CC2F80CC040
:10DFF000B942F3D3BA46370CF7F706FD8346FCF770
:10E00000E1FEB84204D8194940F28310F4F7A8FBA6
:10E01000601C284008EB800047EA0B41C160D8F83B
:10E020000C0447468047A11C294007EB81012C4086
:10E03000C86007EB8401C86866F3C5006AF38910FD
:10E0400069F39F2020F00300401C00E002E020F074
:10E050000400C86098F8200402E000BFFCF7ACFCA4
:10E060000028FBD1BDE8F88FD81F002084150100DF
:10E0700070B50C46050003D107A15420F4F770FBDE
:10E080001CB905A15520F4F76BFB21462846BDE8D5
:10E090007040F2F77CBA00002E2E5C2E2E5C2E2EE5
:10E0A0005C64656D6F5F636C695F636D64732E6341
:10E0B0000000000070B50C46050004D108A140F630
:10E0C0001410F4F74DFB24B905A140F61510F4F730
:10E0D00047FB21682868BDE87040F2F758BA000095
:10E0E0002E2E5C2E2E5C2E2E5C2E2E5C2E2E5C2E6A
:10E0F0002E5C636F6D706F6E656E74735C6C6962BD
:10E100007261726965735C636C695C6E72665F6391
:10E110006C692E630000000070B50546F4F722FA22
:10E12000124C06462078F4F71DFA86420AD028469B
:10E13000F4F718FA20B104F10C00FAF7D7FC01E06B
:10E14000FAF792FC2846F4F71AFA06462078F4F714
:10E1500016FA864208D02846F4F711FA10B1FAF7F9
:10E16000F9FD01E0FBF7EEFC257070BDF401002025
:10E170002DE9F04114460D00064604D11BA140F2E2
:10E180007A20F4F7EDFA24B918A140F27B20F4F7D5
:10E19000E7FA3046F7F73EFB78B9B068FA2107890D
:10E1A000B0F80C803046F7F705FCFA213046F7F757
:10E1B0007DFA3046F7F72EFB10B10620BDE8F0815E
:10E1C000B06800892880B068808920802888C01BBA
:10E1D00081B23046F7F7DCFA2188A1EB080081B262
:10E1E0003046F7F7F3FB0020E8E700002E2E5C2E08
:10E1F0002E5C2E2E5C2E2E5C2E2E5C2E2E5C636FE3
:10E200006D706F6E656E74735C6C69627261726959
:10E2100065735C636C695C6E72665F636C692E63C8
:10E220000000000070B50446C06818B90F496120AD
:10E23000F4F796FA0E4800250078A0B19CB1207E34
:10E2400088B1D4E903108847A06850B1217E41B15C
:10E2500061680844606021460648FDF70DFE01250F
:10E2600001E000202076284670BD00004004010037
:10E27000CC0100205CF400000948007800280ED092
:10E2800008480268521C026007484168032906D307
:10E290000088052101EB004004A1FCF7BBBC7047DE
:10E2A000000000200400002084050020636F756ECC
:10E2B000746572203D2025640D0A000010B50446E7
:10E2C0000020F2F739FC20B16068D0E9002100207D
:10E2D00090476068D0E9002101209047A06822465D
:10E2E00040F6CD410068F3F7F1F8002805D0BDE80D
:10E2F000104002A11B20F4F733BA10BD2E2E5C2E65
:10E300002E5C2E2E5C2E2E5C2E2E5C2E2E5C636FD1
:10E310006D706F6E656E74735C6C69627261726948
:10E3200065735C636C695C7274745C6E72665F6367
:10E330006C695F7274742E63000000004069054AC6
:10E340000178515C11B1001DFEF764BE0C30FEF780
:10E350004DBC0000800100202DE9F84F374D834669
:10E3600069462868F9F734FA04464FF00408002794
:10E370004FF00109324EDFF8CCA05BE0207820B1ED
:10E38000012828D002284CD138E06068017E00299D
:10E3900047D180F818905846F7F747FB0146606868
:10E3A0004268511A284A914203D9416821F07F41BD
:10E3B0004160224861680830FDF75EFD6168486988
:10E3C0004268042A2DD34A68018808EB01401FA146
:10E3D000FCF720FC25E061687068814200D177601D
:10E3E00016480830FDF706FE606840694168042958
:10E3F00017D3018808EB01401AA110E0FFF7A0FD38
:10E4000008B10776FAE786F80090DAF804100329D5
:10E4100007D3BAF80000032101EB004015A1FCF777
:10E42000F5FB69462868F9F7C8F969462868F9F7DD
:10E43000CFF90446002CA1D1BDE8F88F54F40000B8
:10E44000CC010020DC04002017FCFF005374617233
:10E45000742072657175657374202843433A25648E
:10E46000292E000053746F70207265717565737486
:10E470002E00000053746F7020616C6C2072657107
:10E48000756573742E000000F8B5114C0D460646F4
:10E4900069462068F9F786F9B8B1067045606946A3
:10E4A0002068F9F7A0F918B10A48F7F78DFB0AE0E0
:10E4B00009484168022906D30088022101EB004087
:10E4C00006A1FCF7A3FB0020F8BD0420F8BD000066
:10E4D00054F40000D4010020DC040020536368657C
:10E4E00064756C696E6720696E746572727570749C
:10E4F000656420616E6F746865722073636865641B
:10E50000756C696E672E0000FEB51A4A6FF0E00563
:10E510005368B1FBF3F411684FF46162B4FBF1F39B
:10E52000B3FBF2F2554303EB05153C23B5FBF3F3C4
:10E53000A3EB031605EB8606B4FBF1F501FB1544CE
:10E540004FF47A756543B5FBF1F504EB440C05FB1C
:10E5500001F7CCEBC414C7EBC4044FF47A777C43C7
:10E56000B4FBF1F10096CDE9015103A1FBF7B0FB3B
:10E57000FEBD0000300300205B253032643A2530B8
:10E5800032643A253032642E253033642C25303302
:10E59000645D200070B50C4605464FF48E71FDF7A2
:10E5A00090FD216AA068415C206A401C2062C5F889
:10E5B0001C1570BD1FB500228DF8002002918168E6
:10E5C00001914261D0E90012684690471FBD0000EA
:10E5D0007CB5FF260546009600780C46002835D00D
:10E5E000012819D0022802D02CA1652011E0297A37
:10E5F000E068FDF729FC28B1042803D027A13920C1
:10E60000F4F7AEF82046FFF72FF9002803D023A136
:10E610003B20F4F7A5F87CBD297AE068FDF714FCEF
:10E6200028B1042803D01DA14120F4F799F8287AD5
:10E6300020B16068D0E90021002090472046FFF714
:10E6400013F90028E7D015A14D20E2E7297A2069C7
:10E65000FDF794FB18B111A15320F4F781F800964F
:10E6600001236A4601A92069FDF79CFB18B10BA1A3
:10E670005620F4F775F8009848B1C2B26069019964
:10E68000FAF74CFB18B105A15B20F4F769F8606854
:10E69000D0E90021012090477CBD00002E2E5C2E89
:10E6A0002E5C2E2E5C2E2E5C2E2E5C2E2E5C636F2E
:10E6B0006D706F6E656E74735C6C696272617269A5
:10E6C00065735C636C695C756172745C6E72665FC5
:10E6D000636C695F756172742E6300001FB50A4632
:10E6E00001788DF8001041680191017A8DF80810C9
:10E6F000C0680390044850F82210083850F82220CF
:10E70000684690471FBD00008C0100202DE9FF479F
:10E710000C4605464FF40071FDF7D9FC01274FF474
:10E720000178002618B34FF4927949462846FDF740
:10E73000C3FCE0B149462846FDF7C3FCC5F8088391
:10E7400094F8290000B96F6002208DF80000D5F818
:10E750008004C5F880040390A0690290E0680190ED
:10E76000A661E661D4E900126846904728E00421DA
:10E770002846FDF7ACFC18B34FF484712846FDF72A
:10E780009BFCE8B121462846FFF72EF8616AA06994
:10E79000884215D1E06938B1E268616AA0612069F8
:10E7A000E6616662E06008E094F8290000B96F60F5
:10E7B000C5F80883A661E268616A2046FFF72DF874
:10E7C0004FF48E7841462846FDF776FC78B1206AF2
:10E7D0006169884202D294F8280020B34146284655
:10E7E000FDF76FFC616911B12046FFF7E3FE4FF4BE
:10E7F000A27841462846FDF75FFC002818D0414624
:10E800002846FDF75EFC94F8290000B12F60A0694E
:10E8100000280DD0A661E268616A04B02046BDE818
:10E82000F047FEF7FABF21462846FFF7B3FEDEE7C2
:10E83000BDE8FF871FB50A4601788DF800104168D2
:10E840000191017A8DF80810C0680390044850F8CF
:10E850002210083850F82220684690471FBD00005B
:10E860008C0100202DE9FF410C464FF492770546BC
:10E870003946FDF732FC0026C0B139462846FDF77F
:10E8800031FC02208DF80000D5F88004C5F8800422
:10E890000390D5F83C058DF80800E0680190A6616A
:10E8A000E661D4E900126846904723E04FF4887788
:10E8B00039462846FDF711FCE0B139462846FDF7F8
:10E8C00011FCD5F83C15A069884213D1E06960B10C
:10E8D000E268D5F8000220F02000C5F80002E069E7
:10E8E000A0612069E661E06001E0A661E26820467F
:10E8F000FEF79EFF4FF4A27739462846FDF7EDFB61
:10E9000060B139462846FDF7EDFBA06930B1A6613C
:10E91000D5F83C152046E268FEF78AFF4FF4907761
:10E9200039462846FDF7D9FB002813D0394628463A
:10E93000FDF7D8FB606900280CD0D5F84C058DF8A0
:10E9400000608DF80800A06801906661D4E90012AB
:10E9500068469047BDE8FF8110B50248F8F74EFFC2
:10E96000002010BDC40200202DE9F05F8346DDE9E0
:10E970000A4A994690460D460846012703E000BF23
:10E98000B0FBF8F07F1C4045FAD2B94500D94F469C
:10E990005FEACA7012D18CB15FEA8A7002D5B9F110
:10E9A000000F01D0202607E0302605E0314658460A
:10E9B000641EF3F72DFF0CB1A742F7D35FF00106F9
:10E9C000B9F1010F02D9A9F1010903E0B5FBF6F095
:10E9D000404502D306FB08F6F2E7DFF83C9000BFA3
:10E9E000B5FBF6F000FB165519F800105846F3F782
:10E9F0000FFFB6FBF8F6002EF2D15FEACA7009D01D
:10EA0000002C07D0A74205D220215846641EF3F7F8
:10EA1000FFFEF5E7BDE8F09F8CF8000002480068B3
:10EA2000002800D0012070471C02002007490A7806
:10EA3000824209D00870052803D0487820F00200EF
:10EA400048700348F3F740BA7047000014020020F2
:10EA5000E0F400002DE9FE4F8046486891464FF0F3
:10EA6000010A0C4628B92068F2F7A2FF08B9A0688D
:10EA700090B1B9F1400F04D937A140F27110F3F70A
:10EA80006FFE00260096FAF7ADFDE768834648461C
:10EA90004F4559D9074657E04FF0000AC8F800A083
:10EAA000C8F804A054E0A068B84201D93D4600E08F
:10EAB0000546616839B10BEB06002A46F1F712FDF5
:10EAC000002060600CE058B121680BEB06022B4679
:10EAD0004868D0F804C004F11000E047012000901D
:10EAE000A068A7EB0507411BA160E0682E44A0EBDE
:10EAF0000500E06005D1009818B12068F2F758FFD2
:10EB00002060E06810B1A068F0B902E04FF0000AA0
:10EB10001AE0206800284FF0000001D0019009E0C1
:10EB200060609EB14E4511D24FF0000A0EE0A06821
:10EB3000401CA0602168012300224868456801A8A4
:10EB4000A8470028F3D12061002FACD1C8E900B656
:10EB50005046BDE8FE8F00002E2E5C2E2E5C2E2E21
:10EB60005C2E2E5C2E2E5C2E2E5C636F6D706F6E95
:10EB7000656E74735C6C69627261726965735C75F1
:10EB80007362645C6170705F757362645F636F72FF
:10EB9000652E63000249002008600249C870704772
:10EBA0001C7C02409401002070B50446010600F070
:10EBB0000F0502D5092D09D301E0092D08D308A1BD
:10EBC00040F28920F3F7CCFD200601D5042000E0B7
:10EBD000282000EB8500BDE87040FDF737BC000041
:10EBE0002E2E5C2E2E5C2E2E5C2E2E5C2E2E5C2E5F
:10EBF0002E5C636F6D706F6E656E74735C647269AA
:10EC0000766572735F6E72665C757362645C6E7259
:10EC1000665F6472765F757362642E630000000045
:10EC20002DE9F04F514D89B0E878002846D1804653
:10EC30004FF001093EE000BF90FAA0F0B0FA80F674
:10EC40003046F3F798FD8346F7F73EF9044600682F
:10EC500020B947A140F23150F3F782FD5FEA0B6023
:10EC600007D5D4E90031A28902A89847002836D0F8
:10EC700037E05846FAF772FCD4E900718246034641
:10EC8000A28902A8B84707460298D0B10399514516
:10EC90001DD20220A07309FA06F0C14333480C309C
:10ECA000F8F7BEFD4248006B00908DF802B069682D
:10ECB00068468847D5E902100840BDD109B0BDE8D3
:10ECC000F08F039850B12AA140F24D5004E0514515
:10ECD00004D027A140F25C50F3F742FD0FB9C4F80D
:10ECE000008034498220086085F80390A96809FAF9
:10ECF00006F08143A960A06803990844A060DDE99B
:10ED000002125846FDF7F4F9FAF756FC18B32A4CEC
:10ED10004FF482752846FDF77BFB5846FFF744FF0A
:10ED20000220FDF7CBFC2846FDF76AFB0028F1D056
:10ED30001E2000E00220FDF7C1FC20688006F9D506
:10ED40000120FDF7BBFC5846FAF7F8FAFDF758FB2F
:10ED50000028DFD0B2E75846FFF726FF5846FAF7FB
:10ED6000EDFAFDF74DFB0028F8D0A7E7940100204D
:10ED70002E2E5C2E2E5C2E2E5C2E2E5C2E2E5C2ECD
:10ED80002E5C636F6D706F6E656E74735C64726918
:10ED9000766572735F6E72665C757362645C6E72C8
:10EDA000665F6472765F757362642E6300000000B4
:10EDB00060F300001C7C0240747402402DE9F843AB
:10EDC00007460020F3F7E8FB3846F7F77DF80646DC
:10EDD0003806294D4FF000084FF003094FF00104A9
:10EDE00038461ED4F7F73CF8E96804FA00F0884387
:10EDF00003D03846FAF7B0FE10E03846C6F8008077
:10EE0000F7F72EF8E96804FA00F081433846E96024
:10EE1000F7F726F88440A868A043A86086F80E900B
:10EE200024E0F7F71DF8D5E9022104FA00F061EAC1
:10EE3000020108421AD03846F7F712F8E96804FAD6
:10EE400000F081433846E960F7F70AF88440A86883
:10EE50000443AC600948C6F8008086F80E9000684C
:10EE600000908DF80270696868468847BDE8F843ED
:10EE70000020F3F7BFBB00009401002060F3000006
:10EE80002DE9F041104EB068040CF06824040443EE
:10EE9000012712E094FAA4F0B0FA80F52846F3F7BF
:10EEA0006AFC00F00F00082804D22846F3F763FC40
:10EEB000FFF784FF07FA05F08443002CEAD140F203
:10EEC000FF10B060BDE8F08194010020012238B548
:10EED0008A400C490C468B6813438B606168E46878
:10EEE000094B050602EA040203D5002A09D19A69F2
:10EEF00002E0002A05D1DA6900928DF80200684626
:10EF0000884738BD9401002060F300002DE9F041EE
:10EF10001148F3F7DFF918B1104ACF21F1F77AF968
:10EF20000F48F2F7EDFB18B10C4AD421F1F772F952
:10EF3000F3F790FA18B1094AD921F1F76BF9064EA7
:10EF40004FF47A747C3EA701751C3846A847641EAE
:10EF5000FAD1BDE8F08100009CF200009C3E000068
:10EF600028F8000002498020C1F800027047000024
:10EF700004E000E010B5082809D009280FD00A28BD
:10EF800011D00E2813D1BDE81040F2F7AFBEFAF74A
:10EF90009FFC00280BD1BDE81040F2F7D1BEBDE8C0
:10EFA0001040F3F7C1BABDE81040F3F785BA10BDC1
:10EFB00070B50C460546F4F70BF8C269002A04D078
:10EFC00021462846BDE87040104770BD0249496897
:10EFD000002900D008477047B01B00201CB500294D
:10EFE00013D08268D27D8A420FD008A3D3E90023D0
:10EFF000CDE9002301F12F028DF803208268D1753D
:10F0000000696A4603A1FAF763FE1CBD1B5B34006E
:10F010006D000000257300001CB5826899B1927DD7
:10F020008A420FD00CA2D2E90032CDE9003201F1C0
:10F030002F028DF805208268917500696A4608A143
:10F04000FAF746FE1CBD9175006902B0054ABDE89D
:10F05000104003A1FAF73CBE1B5B313B33006D004F
:10F0600025730000F0F7000010B50446F5F726F808
:10F07000002105E0625C3F2A06D02A2A04D0491C00
:10F080008142F7D3002010BD012010BD0020704741
:10F090002DE9FC4180461C4617460E460C48089D4B
:10F0A000F8F7B5FB10B11120BDE8FC81A208394684
:10F0B0003046FCF767FA0648F8F7A0FB33463A46B5
:10F0C00001214046CDE90045F7F718F90020EBE7AC
:10F0D000C402002060FC00003CFC000000000000B6
:10F0E000CD51000000000000ECF00000ACFC00007E
:10F0F0008CFC000000000000F5520000B0FC000095
:10F1000068FC000000000000315300000000000017
:10F11000000000000000000000000000B8FC00003B
:10F12000B8FC0000E4F0000039520000C0FC000010
:10F13000C0FC000000000000695300000000000057
:10F1400044F1000018FD0000E0FC00000000000099
:10F15000E148000020FD0000F8FC00000000000075
:10F160001949000010FD0000C8FC0000000000006C
:10F1700051490000000000000000000000000000F5
:10F18000000000004CFD000028FD00003CF10000E4
:10F19000D547000001000000755D00000000000080
:10F1A000A4F10000A4FE00007CFD000000000000AF
:10F1B000FD490000A8FE000054FD000094F100008D
:10F1C000994B0000B0FE000068FD000094F10000C3
:10F1D000654C0000B8FE000080FE0000000000004A
:10F1E000594D000000000000000000000000000079
:10F1F00000000000E4FE0000C0FE00009CF10000E2
:10F2000089490000240301002003010004030100D8
:10F2100020000020000000000000000000000000AE
:10F220000338FDD8704700002C030100A8F200004D
:10F2300024080020540000203C0000203C1D010058
:10F240000D00000038030100E0F20000BC0D0020BA
:10F25000A000002088000020581D01000D000000C3
:10F2600048030100FCF20000B4120020EC00002072
:10F27000D4000020741D01000A000000FFFFFFFF02
:10F28000FFFFFFFFFFFFFFFFFFFFFFFF000000008A
:10F29000000000000000D60107010000C91E0000A8
:10F2A00075EF00000000000048F800000401002095
:10F2B0006C000020100D00203F000000500D0020C9
:10F2C000680D00200F000000780D002000000000F5
:10F2D000002000400000000000200040000000006E
:10F2E00078F80000900D0020B0F20000C0F200009D
:10F2F000B4F20000CCF20000B80000205CF800007E
:10F30000A8120020F8F200000000000010F3000036
:10F3100094030100780301000000000059B00000D0
:10F320008C030100540301000000000055B10000EF
:10F3300000000000000000000000000000000000CD
:10F34000B80301009C03010008F3000039B300007A
:10F3500000000000000000000000000000000000AD
:10F360000600000301000000060000000600000087
:10F370000600000006000000060000000600000174
:10F38000050000000200000003000000040000006F
:10F390000600000200000000000000000000000065
:10F3A0000338FDD870470000DD62000015620000E0
:10F3B000A95F0000DD5F0000E35F0000E95F00007F
:10F3C000EF5F0000F55F0000FB5F000001600000E0
:10F3D00045610000076000000D6000006D600000E6
:10F3E00073600000796000007F60000085600000AD
:10F3F0008B6000009160000099600000D9610000FE
:10F400001962000061610000E560000008010C0164
:10F410001001140118011C01200124012C013001EC
:10F42000340138013C014001440148014C015001C4
:10F4300002030405060708090B0C0D0E0F1011122C
:10F44000131400000000005000030050D5C9000054
:10F45000D9CD0000DC010020000007000000000002
:10F46000F001002095550000800000000B81000095
:10F470008200000083000000840D0E030B000000DA
:10F480000C0008000000090000000A000000000055
:10F49000F1230000C91E0000000000000000000071
:10F4A0009928000031290000000000000000000041
:10F4B000000000005530000000000000452800005A
:10F4C0000000000045280000000000007D31000021
:10F4D00000000000000000000A0000000000000022
:10F4E0000F00000017D900000000000055EA0000DE
:10F4F000FC1B0020120100020000004015190F52F1
:10F5000000010102030109020000000100C0FA002D
:10F51000111A0000000000000000000000000000C0
:10F52000000000002402002010F50000010002038A
:10F5300000800000040309002A034E006F007200DF
:10F540006400690063002000530065006D006900DD
:10F5500063006F006E0064007500630074006F004C
:10F56000720026036E005200460035003200200073
:10F570005500530042002000430044004300200097
:10F58000440065006D006F001A0330003000300049
:10F5900030003000300030003000300030003000EB
:10F5A00030000E035500730065007200200031002A
:10F5B000000102030400000018FD00001C0501000A
:10F5C0000000000081530000B00901002C0501007B
:10F5D000000000003D4E0000540501003C05010004
:10F5E000000000006147000000000000F0F500008E
:10F5F000B00901008C050100000000007D4F0000F3
:10F60000600501006805010000000000A150000035
:10F6100000000000000000000000000000000000EA
:10F62000B0050100B8050100E8F500000000000089
:10F630000338FDD8704700000000000040F60000CD
:10F64000640B0100400B010000000000697A00001B
:10F6500000000000000000000000000000000000AA
:10F660006C0B0100740B010038F60000697A000091
:10F6700055A7000039A700001DA7000000000000EA
:10F6800084F60000540C01003C0C01000000000056
:10F690006D7F0000580C0100240C010000000000E8
:10F6A000977F000000000000000000000000000044
:10F6B0000000000000000000BCF60000540C010037
:10F6C0005C0C01000000000059800000580C010093
:10F6D000B80C010000000000838000000000000062
:10F6E000000000000000000000000000000000001A
:10F6F000F4F6000018FD0000F80C01000000000006
:10F70000E97D0000B8FE0000CC0C01000000000004
:10F71000197E000000000000000000000000000052
:10F7200000000000000000002CF70000680D010040
:10F73000480D01007CF60000A57E0000600D010070
:10F74000240D0100B4F60000C17F0000700D01001F
:10F75000380D0100ECF600007D7D00000000000087
:10F760000000000000000000000000000000000099
:10F7700074F70000BC0D0100780D010000000000CE
:10F78000AD8200000000000000000000000000004A
:10F7900000000000D40D0100C40D010000000000B5
:10F7A000F97B0000000E0100DC0D010024F70000D1
:10F7B000CD7C0000180E0100040E010000000000C6
:10F7C000AD800000C00E0100200E01006CF70000AB
:10F7D000898100000000000000000000000000001F
:10F7E0001B37001B38001B45002C20001B5B4A0008
:10F7F0001B5B6D00082008001B5B4B00202D2000C8
:10F800001B5B48001B5B366E001B5B324A0000002E
:10F810000338FDD870471B5B3F336C002D682C20EC
:10F820002D2D68656C700000141C0020A0F40000F1
:10F8300002000106010204828101000000000101B2
:10F84000810100009D31000069350000A9350000EC
:10F850005D350000AD3500007D350000F93C00004D
:10F86000813D0000A13C0000893D00001D3D0000DD
:10F870000338FDD870470000CD44000081450000EA
:10F8800061440000994500001945000030313233D1
:10F890003435363738394142434445466E72665FE7
:10F8A0006673746F726167655F696E6974006E720A
:10F8B000665F6673746F726167655F756E696E69A6
:10F8C00074006E72665F6673746F726167655F72F3
:10F8D000656164006E72665F6673746F72616765FE
:10F8E0005F7772697465006E72665F6673746F72BB
:10F8F0006167655F6572617365000000001000005C
:10F900000400000001000000356B000059E9000010
:10F9100073D6000091F00000615F000081D6000006
:10F920008DF00000A96D00000000000030F900001B
:10F93000640B0100FC0F01000000000085BA00000C
:10F9400000000000000000000000000000000000B7
:10F9500020100100740B010028F9000085BA000096
:10F96000556E6B6E6F776E206572726F7220636F6B
:10F970006465000000000000541401000100000054
:10F980001413010002000000081101000300000030
:10F990008813010004000000DC13010005000000D2
:10F9A000BC12010006000000581201000700000010
:10F9B000C413010008000000D0120100090000007B
:10F9C000341301000A0000003C1401000B00000089
:10F9D000F01001000C000000E81201000D00000012
:10F9E0008C1401000E000000B41301000F00000091
:10F9F000F0130100100000002414010011000000A9
:10FA0000A0140100800000007012010081000000BD
:10FA1000AC110100820000006C11010083000000A5
:10FA20004C110100840000008811010085000000D5
:10FA300094120100860000009C1301009000000059
:10FA400038120100910000002C110100920000000A
:10FA5000FC12010000820000041401000182000079
:10FA600050130100028200006C13010000840000AA
:10FA7000C81101000184000060140100028400002C
:10FA80001012010003840000EC1101002D2D2D2D1A
:10FA90002D2D2D2D2D2D2D43524153484C4F472DAB
:10FAA0002D2D2D2D2D2D2D2D2D2D2D0D0A00000050
:10FAB00029000000000000000000000049A900002B
:10FAC00045A9000039A900002DA80000B5A7000035
:10FAD000A9A7000000000000DCFA0000D40D01001E
:10FAE000CC1401000000000089630000B014010084
:10FAF000B81401000000000005640000640B010060
:10FB0000D81401000000000065640000000000003F
:10FB1000000000000000000000000000EC140100E4
:10FB2000F8140100D4FA00000000000001000000F9
:10FB30009D7600000100000011DF000000000000C1
:10FB400044FB0000DC160100681601002CFB0000DD
:10FB5000296E0000D4160100E415010034FB0000FA
:10FB6000296E000004170100E416010000000000E7
:10FB70000170000018170100F416010000000000D9
:10FB800009700000640B010008170100000000006C
:10FB9000597100000000000000000000000000009B
:10FBA0000000000020170100241701003CFB0000AA
:10FBB000D16D000000404040404040404040414145
:10FBC0004141414040404040404040404040404032
:10FBD00040404040400502020202020202020202CC
:10FBE00002020202022020202020202020202002C9
:10FBF0000202020202029090909090901010101059
:10FC000010101010101010101010101010101010F4
:10FC10000202020202028888888888880808080888
:10FC20000808080808080808080808080808080854
:10FC30000202020240000000B5FB00005072696E33
:10FC400074204E6F726469632053656D69636F6ED3
:10FC5000647563746F72206C6F676F2E0000000014
:10FC60006E6F7264696300005072696E7420656122
:10FC7000636820706172616D6574657220696E20C1
:10FC80006E6577206C696E652E0000005072696E9B
:10FC90007420616C6C20656E74657265642070619F
:10FCA00072616D65746572732E000000616C6C008A
:10FCB000706172616D0000007072696E7400000006
:10FCC000707974686F6E000053746F702073656391
:10FCD0006F6E647320636F756E7465722E00000022
:10FCE0005265736574207365636F6E647320636F10
:10FCF000756E7465722E00005374617274207365A2
:10FD0000636F6E647320636F756E7465722E00008E
:10FD100073746F70000000007265736574000000FA
:10FD20007374617274000000446973706C617920AF
:10FD30007365636F6E6473206F6E207465726D6996
:10FD40006E616C2073637265656E0000636F756E23
:10FD50007465720045786563757465206120636F12
:10FD60006D6D616E642E000052656D6F7665206169
:10FD700020636F6D6D616E642E000000416464202D
:10FD800061206E65772064796E616D696320636FB1
:10FD90006D6D616E642E0A4578616D706C652075BD
:10FDA000736167653A205B2064796E616D696320D9
:10FDB0006164642074657374205D2077696C6C20C5
:10FDC00061646420612064796E616D696320636F92
:10FDD0006D6D616E64202774657374272E0A496EF9
:10FDE0002074686973206578616D706C652C206380
:10FDF0006F6D6D616E64206E616D65206C656E6700
:10FE00007468206973206C696D6974656420746F0F
:10FE10002033322063686172732E20596F7520631E
:10FE2000616E2061646420757020746F2032302010
:10FE3000636F6D6D616E64732E20436F6D6D616EC7
:10FE4000647320617265206175746F6D617469639C
:10FE5000616C6C7920736F7274656420746F2065B7
:10FE60006E7375726520636F727265637420434CA4
:10FE70004920636F6D706C6574696F6E2E000000B1
:10FE800053686F7720616C6C2061646465642064E2
:10FE9000796E616D696320636F6D6D616E64732E41
:10FEA0000000000061646400657865637574650036
:10FEB00072656D6F7665000073686F7700000000F3
:10FEC00044656D6F6E7374726174652064796E61E0
:10FED0006D696320636F6D6D616E6420757361671A
:10FEE000652E000064796E616D6963000D0A202043
:10FEF000202020202020202020202E636F3A2E203A
:10FF000020202020202020202020202020202020F1
:10FF1000202027786F2C2020202020202020202027
:10FF20000D0A2020202020202020202E2C636F6C02
:10FF30006C6C6C632C2E2020202020202020202080
:10FF400020202027636B4F4F6F3A3A2C2E2E202013
:10FF5000202020200D0A2020202020202E3A6F6F04
:10FF60006F6F6F6C6C6C6C6C6C6C6C3A272E202015
:10FF70002020202E3B644F4F4F4F4F4F6F3A3A3A5D
:10FF80003B3B3B272E2020200D0A202020276F6B93
:10FF90007864646F6F6F6F6C6C6C6C6C6C6C6C6C99
:10FFA0006C6C6C3B27636B4F4F4F4F4F4F4F4F4F16
:10FFB0006F3A3A3A3B3B3B2C2C2C27200D0A202051
:10FFC000204F4F4F6B78646F6F6F6F6C6C6C6C6C05
:10FFD0006C6C6C6C6C6C6C6C6C6C6C64784F4F4FB4
:10FFE0004F4F4F4F6F3A3A3A3B3B3B2C2C2C272E2E
:10FFF0000D0A2020204F4F4F4F4F4F6B646F6F6C97
:020000040001F9
:100000006C6C6C6C6C6C6C6C6C6C6C6C6C6C6C6C30
:100010006C6C6C64784F4F4F6F3A3A3A3B3B3B2CD9
:100020002C2C272E0D0A2020204F4F4F4F4F4F4F83
:100030004F4F6B786F6C6C6C6C6C6C6C6C6C6C6C2C
:100040006C6C6C6C6C6C6C6363636C646C3A3A3AA9
:100050003B3B3B2C2C2C272E0D0A2020204F4F4FB2
:100060004F4F4F4F4F4F4F4F4F4F78646F6C6C6CEB
:100070006C6C6C6C6C6C6C6C6C6C6C6363636363ED
:100080003A3A3A3A3B3B3B2C2C2C272E0D0A2020A7
:10009000204F4F4F4F4F4F4F4F4F4F4F4F4F4F4F9F
:1000A0004F6B78646C6C6C6C6C6C6C6C6C6C6C63B3
:1000B000636363633A3A3A3A3B3B3B2C2C2C272E42
:1000C0000D0A2020206B4F4F4F4F4F4F4F4F4F4F38
:1000D0004F4F4F4F4F4F4F4F4F6B646F6C6C6C6C6B
:1000E0006C6C6C63636363633A3A3A3A3B3B3B2C18
:1000F0002C2C272E0D0A2020206B4F4F4F4F4F4F97
:100100004F4F4F4F4F4F4F4F4F4F4F4F4F4F4F4FFF
:100110004F78646C6C6C6C63636363633A3A3A3A2D
:100120003B3B3B2C2C2C272E0D0A2020206B4F4FC5
:100130004F4F4F4F4F4F4F4F4F4F4F4F4F4F4F4FCF
:100140004F4F4F4F4F4F4F4F6B786F6C63636363ED
:100150003A3A3A3A3B3B3B2C2C2C272E0D0A2020D6
:10016000206B4F4F4F4F4F4F4F4F4F4F4F4F4F4FB2
:100170004F4F4F4F4F4F4F4F4F4F4F4F4F4F4F4F8F
:100180006B646C633A3A3A3A3B3B3B2C2C2C272E5F
:100190000D0A202020784F4F4F4F4F4F4F4F4F4F5A
:1001A0004F78646B4F4F4F4F4F4F4F4F4F4F4F4F05
:1001B0004F4F4F4F4F4F4F4F786F633A3B3B3B2C66
:1001C0002C2C272E0D0A202020784F4F4F4F4F4FB9
:1001D0004F4F4F4F4F64633A3A6C646B4F4F4F4FE2
:1001E0004F4F4F4F4F4F4F4F4F4F4F4F4F4F4F6B03
:1001F00064633B2C2C2C27270D0A202020784F4F9E
:100200004F4F4F4F4F4F4F4F4F64633A3A3B3B2C4A
:100210003B63646B4F4F4F4F4F4F4F4F4F4F4F4FBD
:100220004F4F4F4F4F4F4F786C3B27270D0A2020E1
:10023000202E6C6B4F4F4F4F4F4F4F4F4F64633AD1
:100240003A3B3B2C2C27272E2E3B6F4F4F4F4F4FC7
:100250004F4F4F4F4F4F4F4F4F4F4F4F4F4F7827AD
:100260000D0A2020202020202E3B6F4F4F4F4F4F54
:100270004F64633A3A3B3B2C2E2020202020202044
:100280002E3A784F4F4F4F4F4F4F4F4F4F4F4F6476
:100290003B2E20200D0A202020202020202020205E
:1002A0002E3A784F4F64633A2C2E202020202020B5
:1002B000202020202020202027636B4F4F4F4F6BA2
:1002C0006C272020202020200D0A20202020202004
:1002D000202020202020202E6F6427202020202076
:1002E0002020202020202020202020202020202707
:1002F000786B2C2020202020202020200D0A0D0AA1
:100300000000000064756D6D79206F7074696F6E08
:100310002068656C7020737472696E67000000005D
:100320002D7400002D2D7465737400007573625F69
:10033000636C693A7E242000756172745F636C6936
:100340003A7E2420000000007274745F636C693A86
:100350007E2420005072696E7420696E666F726D23
:100360006174696F6E2061626F7574204D50552005
:1003700073746174652E000044756D70204D505586
:10038000207265676973746572732E00696E666F9B
:100390000000000064756D7000000000436F6D6D1B
:1003A000616E647320666F72204D5055206D616ED2
:1003B0006167656D656E74006D7075002D2D2F2D54
:1003C0002D000000574257412F2D2D0057422F2D51
:1003D0002D00000057542F2D2D0000002D2D2F57DC
:1003E00042574100574257412F57425741000000A2
:1003F00057422F574257410057542F5742574100F9
:100400002D2D2F5742000000574257412F574200D1
:1004100057422F574200000057542F574200000008
:100420002D2D2F5754000000574257412F5754008D
:1004300057422F575400000057542F5754000000C4
:100440002E2E5C2E2E5C2E2E5C2E2E5C2E2E5C2EE6
:100450002E5C636F6D706F6E656E74735C6C696239
:100460007261726965735C74696D65725C657870E0
:100470006572696D656E74616C5C6170705F7469E2
:100480006D6572322E6300002E2E5C2E2E5C2E2E99
:100490005C2E2E5C2E2E5C2E2E5C636F6D706F6E4C
:1004A000656E74735C6C69627261726965735C75A8
:1004B0007362645C6170705F757362645F636C61CA
:1004C00073735F626173652E680000002E2E5C2ED0
:1004D0002E5C2E2E5C2E2E5C2E2E5C2E2E5C636FE0
:1004E0006D706F6E656E74735C6C69627261726957
:1004F00065735C757362645C636C6173735C636485
:10050000635C61636D5C6170705F757362645F638F
:1005100064635F61636D2E63000000005379737440
:10052000656D2072657365742E00000054726967F2
:10053000676572206572726F722E00005072696E6C
:1005400074206170706C69636174696F6E20736987
:100550007A652E006170705F73697A650000000033
:100560007761726E696E67005761726E696E67209F
:100570006C6F67206D657373616765207769746858
:1005800020706172616D6574657273004572726F7F
:1005900072206C6F67206D65737361676520776982
:1005A000746820706172616D65746572730000001B
:1005B0006C6F675F6D73670054726967676572205F
:1005C0006C6F67206D657373616765207769746808
:1005D00020646563696D616C20617267756D656E1D
:1005E000747300002E2E5C2E2E5C2E2E5C2E2E5C44
:1005F0002E2E5C2E2E5C636F6D706F6E656E747345
:100600005C6C69627261726965735C74696D657254
:100610005C6578706572696D656E74616C5C64723E
:10062000765F7274632E6300446174612062757337
:10063000206572726F72202872657475726E206107
:1006400064647265737320696E20746865207374C6
:1006500061636B206672616D65206973206E6F74D3
:100660002072656C6174656420746F207468652005
:10067000696E737472756374696F6E2074686174E7
:100680002063617573656420746865206572726F9C
:100690007229000044617461206275732065727272
:1006A0006F72202850432076616C756520737461E9
:1006B000636B656420666F7220746865206578637B
:1006C000657074696F6E2072657475726E20706FDC
:1006D000696E747320746F2074686520696E73741A
:1006E00072756374696F6E207468617420636175DC
:1006F00073656420746865206661756C74290000F8
:1007000043617573653A204275734661756C742058
:100710006F6E206120766563746F72207461626C05
:1007200065207265616420647572696E6720657802
:1007300063657074696F6E2070726F63657373693F
:100740006E672E005468652070726F636573736FF7
:1007500072206861732065786563757465642061D3
:100760006E2053444956206F7220554449562069E3
:100770006E737472756374696F6E20776974682024
:10078000612064697669736F72206F6620300000A3
:100790005468652070726F636573736F722068614F
:1007A0007320617474656D7074656420746F206566
:1007B00078656375746520616E20696E73747275F7
:1007C0006374696F6E2074686174206D616B65730A
:1007D00020696C6C6567616C20757365206F66209D
:1007E000746865204550535200000000546865202D
:1007F00070726F636573736F7220686173206174C8
:1008000074656D7074656420616E20696C6C6567D9
:10081000616C206C6F6164206F66204558435F52A5
:10082000455455524E20746F207468652050432CF7
:10083000206173206120726573756C74206F66206F
:10084000616E20696E76616C696420636F6E746599
:1008500078742C206F7220616E20696E76616C69ED
:1008600064204558435F52455455524E2076616C82
:10087000756500005468652070726F636573736FEF
:100880007220617474656D707465642061206C6F92
:100890006164206F722073746F72652061742061CF
:1008A000206C6F636174696F6E207468617420647A
:1008B0006F6573206E6F74207065726D697420743B
:1008C0006865206F7065726174696F6E000000006A
:1008D00041204D656D4D616E616765206661756C87
:1008E00074206F6363757272656420647572696EDB
:1008F0006720666C6F6174696E672D706F696E74C6
:10090000206C617A792073746174652070726573EC
:100910006572766174696F6E000000004120627537
:1009200073206661756C74206F63637572726564A1
:1009300020647572696E6720666C6F6174696E679A
:100940002D706F696E74206C617A79207374617494
:100950006520707265736572766174696F6E0000F0
:100960005468652070726F636573736F722068617D
:100970007320617474656D7074656420746F206594
:1009800078656375746520616E20756E646566694F
:100990006E656420696E737472756374696F6E003E
:1009A000496E737472756374696F6E20627573201B
:1009B0006572726F720000005468652070726F6318
:1009C0006573736F722068617320617474656D70F4
:1009D00074656420746F20616363657373206120A4
:1009E000636F70726F636573736F7200556E7374AB
:1009F00061636B20666F7220616E2065786365703D
:100A000074696F6E2072657475726E2068617320F0
:100A1000636175736564206F6E65206F72206D6F02
:100A20007265206163636573732076696F6C6174AE
:100A3000696F6E7300000000537461636B696E67C9
:100A400020666F7220616E20657863657074696FCF
:100A50006E20656E747279206861732063617573AE
:100A60006564206F6E65206F72206D6F7265206106
:100A700063636573732076696F6C6174696F6E73FD
:100A8000000000005468652070726F636573736FB7
:100A90007220686173206D61646520616E20756EDF
:100AA000616C69676E6564206D656D6F7279206138
:100AB0006363657373000000556E737461636B202C
:100AC000666F7220616E20657863657074696F6E01
:100AD0002072657475726E2068617320636175732E
:100AE0006564206F6E65206F72206D6F72652042A5
:100AF00075734661756C7473000000005374616314
:100B00006B696E6720666F7220616E206578636521
:100B10007074696F6E20656E7472792068617320DD
:100B2000636175736564206F6E65206F72206D6FF1
:100B30007265204275734661756C74730000000025
:100B40005072696E7420737461747573206F6620BF
:100B500062616C6C6F6320696E7374616E63657340
:100B60002E000000737461747573000062616C6C18
:100B70006F630000436F6D6D616E647320666F720A
:100B80002042414C4C4F43206D616E6167656D653D
:100B90006E74000025730D0A092D20456C656D6586
:100BA0006E742073697A653A092564202B202564C8
:100BB000206279746573206F6620646562756720B2
:100BC000696E666F726D6174696F6E0D0A092D2012
:100BD00055736167653A09257525252028257520F7
:100BE0006F7574206F6620257520656C656D656E68
:100BF0007473290D0A092D204D6178696D756D3A60
:100C0000092575252520282575206F7574206F66A8
:100C100020257520656C656D656E7473290D0A0D50
:100C20000A000000456E61626C6520636F6C6F7234
:100C300065642073796E7461782E00004469736175
:100C4000626C6520636F6C6F7265642073796E747B
:100C500061782E006F6666006F6E000044697361F4
:100C6000626C6520434C49206563686F2E20417299
:100C7000726F777320616E6420627574746F6E7327
:100C80003A204261636B73706163652C2044656C2C
:100C90006574652C20456E642C20486F6D652C2092
:100CA000496E7365727420617265206E6F7420687E
:100CB000616E646C65642E00456E61626C652043F4
:100CC0004C49206563686F2E000000004765742062
:100CD000434C49207374617469737469637320664B
:100CE0006F7220746865204C6F67676572206D6F46
:100CF00064756C652E000000526573657420434C6A
:100D000049207374617469737469637320666F72C8
:100D100020746865204C6F67676572206D6F64751D
:100D20006C652E00546F67676C6520434C492065E5
:100D300063686F2E00000000434C49207374617497
:100D40006973746963732E00546F67676C65206301
:100D50006F6C6F7265642073796E7461782E000019
:100D60006563686F00000000636F6C6F7273000052
:100D70007374617473000000417373756D6520387E
:100D8000302063686172732073637265656E2077CB
:100D90006964746820616E642073656E6420746891
:100DA00069732073657474696E6720746F2074684A
:100DB00065207465726D696E616C2E006465666194
:100DC000756C7400436C6561722073637265656E47
:100DD0002E000000636C656172000000557365664B
:100DE000756C2C206E6F7420556E69782D6C696B54
:100DF0006520434C4920636F6D6D616E64732E00F6
:100E0000636C6900436F6D6D616E64206869737413
:100E10006F72792E00000000686973746F72790038
:100E2000436F6E736F6C65206765747320746572B1
:100E30006D696E616C2073637265656E2073697A8B
:100E400065206F7220617373756D65732038302073
:100E5000696E2063617365207468652072656164E2
:100E60006F7574206661696C732E204974206D75EE
:100E700073742062652065786563757465642061AC
:100E8000667465722065616368207465726D696E51
:100E9000616C207769647468206368616E6765209F
:100EA000746F20656E7375726520636F727265630F
:100EB00074207465787420646973706C61792E0095
:100EC000726573697A650000436F6D6D616E6420B1
:100ED00062756666657220697320746F6F2073682F
:100EE0006F727420746F20657870616E6420616C1D
:100EF0006C20636F6D6D616E6473206D61746368E7
:100F0000696E672077696C646361726420706174D4
:100F10007465726E0D0A0000202000002E2E5C2EDB
:100F20002E5C2E2E5C2E2E5C2E2E5C2E2E5C636F85
:100F30006D706F6E656E74735C6C696272617269FC
:100F400065735C636C695C6364635F61636D5C6E55
:100F500072665F636C695F6364635F61636D2E6378
:100F600000000000616464725F69735F7769746890
:100F7000696E5F626F756E647328705F66732C2094
:100F8000706167655F616464722C20286C656E20F7
:100F90002A20705F66732D3E705F666C6173685FB8
:100FA000696E666F2D3E65726173655F756E6974FB
:100FB000292900002E2E5C2E2E5C2E2E5C2E2E5CFF
:100FC0002E2E5C2E2E5C636F6D706F6E656E74736B
:100FD0005C6C69627261726965735C657870657278
:100FE000696D656E74616C5F6D656D6F626A5C6E74
:100FF00072665F6D656D6F626A2E63005072696E16
:101000007420737461747573206F662071756575D3
:101010006520696E7374616E6365732E0000000055
:10102000717565756500000025730D0A092D204551
:101030006C656D656E742073697A653A0925640D77
:101040000A092D2055736167653A09257525252004
:10105000282575206F7574206F6620257520656CB6
:10106000656D656E7473290D0A092D204D617869CF
:101070006D756D3A092575252520282575206F7514
:1010800074206F6620257520656C656D656E7473C0
:10109000290D0A092D204D6F64653A090925730D44
:1010A0000A0D0A002E2E5C2E2E5C2E2E5C2E2E5C3F
:1010B0002E2E5C2E2E5C636F6D706F6E656E74737A
:1010C0005C6C69627261726965735C657870657287
:1010D000696D656E74616C5F72696E676275665C7E
:1010E0006E72665F72696E676275662E63000000DD
:1010F0004E52465F4552524F525F494E56414C49FF
:10110000445F4441544100004E52465F4552524FA5
:10111000525F534F46544445564943455F4E4F54E2
:101120005F454E41424C4544000000004E52465F30
:101130004552524F525F464541545552455F4E4FBE
:10114000545F454E41424C45440000004E52465FBC
:101150004552524F525F4D555445585F554E4C4F76
:10116000434B5F4641494C45440000004E52465FA8
:101170004552524F525F4D555445585F4C4F434B6B
:101180005F4641494C4544004E52465F4552524FDE
:10119000525F4D555445585F434F4E445F494E4949
:1011A000545F4641494C4544000000004E52465FA2
:1011B0004552524F525F4D555445585F494E495420
:1011C0005F4641494C4544004E52465F4552524F9E
:1011D000525F424C455F495053505F52585F504BED
:1011E000545F5452554E4341544544004E52465F5D
:1011F0004552524F525F424C455F495053505F50E9
:101200004545525F52454A4543544544000000005D
:101210004E52465F4552524F525F424C455F4950D5
:1012200053505F4C494E4B5F444953434F4E4E45DC
:1012300043544544000000004E52465F4552524F11
:10124000525F4150495F4E4F545F494D504C454DA0
:10125000454E5445440000004E52465F4552524FA1
:10126000525F4E4F545F535550504F5254454400B7
:101270004E52465F4552524F525F4D4F44554C457A
:101280005F4E4F545F494E495449414C495A454479
:10129000000000004E52465F4552524F525F4D4F84
:1012A00044554C455F414C52454144595F494E4974
:1012B0005449414C495A4544000000004E52465F93
:1012C0004552524F525F4E4F545F464F554E440069
:1012D0004E52465F4552524F525F494E56414C491D
:1012E000445F5354415445004E52465F4552524F5D
:1012F000525F444154415F53495A45004E52465F44
:101300004552524F525F494F5F50454E44494E47F8
:10131000000000004E52465F4552524F525F5356F6
:10132000435F48414E444C45525F4D495353494EEB
:10133000470000004E52465F4552524F525F494EA1
:1013400056414C49445F4C454E475448000000000C
:101350004E52465F4552524F525F4452565F545769
:10136000495F4552525F414E41434B004E52465FEA
:101370004552524F525F4452565F5457495F45524F
:10138000525F444E41434B004E52465F4552524FCE
:10139000525F494E5445524E414C00004E52465FFA
:1013A0004552524F525F53544F524147455F465545
:1013B0004C4C00004E52465F4552524F525F4E55C4
:1013C0004C4C00004E52465F4552524F525F494EC0
:1013D00056414C49445F504152414D004E52465F88
:1013E0004552524F525F4E4F5F4D454D0000000039
:1013F0004E52465F4552524F525F464F5242494409
:1014000044454E004E52465F4552524F525F445241
:10141000565F5457495F4552525F4F564552525599
:101420004E0000004E52465F4552524F525F494EA9
:1014300056414C49445F4144445200004E52465F7D
:101440004552524F525F494E56414C49445F464CBB
:10145000414753004E52465F535543434553530053
:101460004E52465F4552524F525F424C455F495083
:1014700053505F4348414E4E454C5F414C524541AD
:1014800044595F4558495354530000004E52465F3B
:101490004552524F525F54494D454F55540000003C
:1014A0004E52465F4552524F525F425553590000CB
:1014B0007265616400000000526561642073746F9E
:1014C000726564206C6F67730000000052656D6F79
:1014D0007665206C6F677300466C617368206C6F73
:1014E000672073746174757300000000666C61732B
:1014F000686C6F6700000000436F6D6D616E647310
:1015000020666F722072656164696E67206C6F6718
:10151000732073746F72656420696E206E6F6E2D18
:10152000766F6C6174696C65206D656D6F727900A2
:101530002E2E5C2E2E5C2E2E5C2E2E5C2E2E5C2EE5
:101540002E5C636F6D706F6E656E74735C6C696238
:101550007261726965735C6578706572696D656EDC
:1015600074616C5F6C6F675C7372635C6E72665FF4
:101570006C6F675F6261636B656E645F666C6173FD
:10158000682E63002E2E5C2E2E5C2E2E5C2E2E5C82
:101590002E2E5C2E2E5C636F6D706F6E656E747395
:1015A0005C6C69627261726965735C6578706572A2
:1015B000696D656E74616C5F6C6F675C7372635CA0
:1015C0006E72665F6C6F675F66726F6E74656E6475
:1015D0002E6300006E6F6E6500000000646562752A
:1015E00067000000276C6F6720656E61626C652084
:1015F0003C6C6576656C3E203C6D6F64756C655F18
:10160000303E202E2E2E20203C6D6F64756C655F61
:101610006E3E2720656E61626C6573206C6F677328
:1016200020757020746F20676976656E206C657612
:10163000656C20696E2073706563696669656420F6
:101640006D6F64756C65732028616C6C2069662011
:101650006E6F206D6F64756C657320737065636960
:1016600066696564292E0000276C6F6720646973C2
:1016700061626C65203C6D6F64756C655F303E2007
:101680002E2E203C6D6F64756C655F6E3E27206466
:10169000697361626C6573206C6F677320696E207B
:1016A000737065636966696564206D6F64756C65E8
:1016B000732028616C6C206966206E6F206D6F64EA
:1016C000756C657320737065636966696564292E3E
:1016D00000000000656E61626C6500006469736102
:1016E000626C6500526573756D65206C6F67676924
:1016F0006E67000048616C74206C6F6767696E6785
:1017000000000000676F00004C6F67676572207310
:10171000746174757300000068616C7400000000EF
:101720006C6F6700436F6D6D616E647320666F72DE
:1017300020636F6E74726F6C6C696E67206C6F677C
:10174000676572001B5B313B33306D001B5B306D96
:10175000000000001B5B313B33316D001B5B313BF4
:1017600033326D001B5B313B33336D001B5B313B10
:1017700033346D001B5B313B33356D001B5B313BFC
:1017800033366D001B5B313B33376D006170705F2A
:1017900074696D65722E6D5F74696D65725F30007E
:1017A00071756575652E6D5F636C695F6364635FFA
:1017B00061636D5F6C6F675F6261636B656E645FD1
:1017C000717565756500000062616C6C6F632E6DEC
:1017D0005F636C695F6364635F61636D5F636D64C6
:1017E0005F686973745F6D656D6F626A0000000009
:1017F0006170705F74696D65722E6D5F636C695F97
:10180000756172745F7472616E73706F72745F74FD
:10181000696D65720000000071756575652E6D5FFC
:10182000636C695F756172745F6C6F675F6261633F
:101830006B656E645F7175657565000062616C6CE7
:101840006F632E6D5F636C695F756172745F636D4A
:10185000645F686973745F6D656D6F626A00000034
:101860006170705F74696D65722E6D5F636C695F26
:101870007274745F7472616E73706F72745F746986
:101880006D65720071756575652E6D5F636C695F5E
:101890007274745F6C6F675F6261636B656E645FC7
:1018A000717565756500000062616C6C6F632E6D0B
:1018B0005F636C695F7274745F636D645F686973A2
:1018C000745F6D656D6F626A000000006D5F636C30
:1018D000695F6364635F61636D5F6C6F675F6261C3
:1018E000636B656E645F7175657565006D5F636CD4
:1018F000695F756172745F6C6F675F6261636B656E
:101900006E645F7175657565000000006D5F636CE6
:10191000695F7274745F6C6F675F6261636B656E41
:10192000645F7175657565006D5F636C695F6364A5
:10193000635F61636D5F636D645F686973745F6D3E
:10194000656D6F626A0000006D5F636C695F756151
:1019500072745F636D645F686973745F6D656D6FEA
:10196000626A00006D5F636C695F7274745F636DBF
:10197000645F686973745F6D656D6F626A00000013
:101980006170705F74696D65722E6D5F6273705FF8
:101990006C6564735F746D72000000006170705F4D
:1019A00074696D65722E6D5F6273705F616C6572D4
:1019B000745F746D720000006170705F74696D65B2
:1019C000722E6D5F6273705F627574746F6E5F7498
:1019D0006D7200006E72665F6D7075007374616386
:1019E0006B5F677561726400636C6F636B0000000E
:1019F0005553424400000000434C4F434B0000004D
:101A00004750494F544500005052530055415254DD
:101A10000000000055415254450000006170705FA5
:101A200074696D65722E6D5F646574656374696F4A
:101A30006E5F64656C61795F74696D65725F69641E
:101A4000000000006170705F74696D6572000000D5
:101A500061746669666F2E6D5F7265715F66696637
:101A60006F0000006170705F7573626400000000B9
:101A70006364635F61636D006170705F757362645E
:101A80005F636F7265000000686172646661756C07
:101A90007400000071756575652E6D5F72785F71F9
:101AA00075657565000000006D5F72785F71756522
:101AB00075650000636C695F7561727400000000F9
:101AC0006E72665F6673746F726167650000000016
:101AD0007077725F6D676D7400000000736F7274D1
:101AE0006C6973740000000071756575652E6D5F1B
:101AF000666C6173686C6F675F7175657565000012
:101B000071756575652E6D5F63726173686C6F6763
:101B10005F717565756500006D5F666C6173686CFB
:101B20006F675F7175657565000000006D5F6372BA
:101B30006173686C6F675F717565756500000000A3
:101B400062616C6C6F632E6C6F675F6D656D706F3B
:101B50006F6C0000617070006C6F675F6D656D7019
:101B60006F6F6C00541E0100000000209005000003
:101B700028070000901F010090050020F840000099
:101B8000A011000000000000D4F0000000000000E0
:101B90001CF10000000000002CF10000000000001B
:101BA00084F1000000000000F4F1000000000000DB
:101BB00040F3000000000000B8F500000000000045
:101BC000C8F5000000000000D8F50000000000008B
:101BD00020F600000000000060F600000000000099
:101BE00094F7000000000000A4F7000000000000CF
:101BF000B4F7000000000000C4F70000000000007F
